:020000040800F2
:1000000038380020530500089D040008090304083F
:10001000A1040008A3040008A504000800000000D3
:10002000000000000000000000000000A70400081D
:10003000A904000800000000AB040008AD0400089B
:10004000AF040008B1040008B3040008B5040008B8
:10005000B7040008B9040008BB040008BD04000888
:10006000BF040008C1040008C3040008C504000858
:10007000C7040008C9040008CB040008CD04000828
:10008000CF040008D1040008D3040008D5040008F8
:10009000D7040008D9040008DB040008DD040008C8
:1000A000DF040008E1040008E3040008E504000898
:1000B000E7040008E9040008EB040008ED04000868
:1000C000EF040008F1040008F3040008F504000838
:1000D000F7040008F9040008FB040008FD04000808
:1000E000FF040008010500080305000805050008D5
:1000F00007050008090500080B0500080D050008A4
:100100000F05000811050008130500081505000873
:1001100017050008190500081B0500081D05000843
:100120001F05000821050008230500082505000813
:1001300027050008290500082B0500082D050008E3
:100140002F050008310500083305000835050008B3
:1001500037050008390500083B0500083D05000883
:100160003F05000841050008430500084505000853
:1001700047050008490500084B0500084D05000823
:080180004F05000851050008BD
:10020000DECEA5ED02003078463430370000000025
:10021000000000000000444D31365F3138303600B8
:100220000000000000004170706C69636174696FC8
:100230006E00000000000000000000000000000050
:100240000000000000000405BC00DAF7DECEA5EDDA
:100250000200307846343037000000000000000013
:10026000000053504C6174436F6E74726F6C6C6518
:1002700072004170706C69636174696F6E00000098
:10028000000000000000000000000000000000006E
:0802900000000000FE00DAF797
:100298000100040818000000A90104080300000078
:1002A800E507040806000000250D04080900000001
:1002B800C515040802000000D1160408100000004B
:1002C8008D180408FF000000B51F04080C0000008A
:1002D80021250408000000005D270408050000002F
:1002E8007150040818000000D550040812000000DE
:1002F8001D5404080A000000C95904080A00000037
:10030800896204081400000015670408080000004A
:100318002D6E040807000000E974040810000000AE
:10032800D178040813000000818A04081300000033
:1003380001B9040816000000151F05081600000082
:10034800C124050817000000E5280508180000006A
:100358001558050816000000D958050817000000B0
:08036800CD6D05081500000031
:100370002F49072291438D462E492F480A1A06D04D
:100380000722914381F30988022282F314882B48C3
:100390002B492C4A00F039F82B482C492C4A00F004
:1003A00034F82C482C492D4A00F02FF82C482D49C0
:1003B0002D4A00F02AF82D482D492E4A00F025F844
:1003C0002D482E492E4A00F020F82E482E490022B2
:1003D00000F026F82D482E49091A082903DB0022CF
:1003E0000260043001601F481F49884205D002683E
:1003F000043003B4904703BCF7E700208646EC4680
:1004000000200021234A9047FEE7884207D0521A75
:1004100005D0037801300B700131013AF9D17047F2
:10042000884202D002700130FAE770471A487047DC
:1004300038380020384000203838002070D40508B3
:10044000880100200C0200200000040800000408BD
:10045000E8A1050870D40508880100208801002063
:10046000AC050008AC050008AC050008AC050008A8
:10047000AC050008AC050008E8A10508E8A10508DE
:1004800070D405080C020020EC3400203835002020
:1004900038350020A5370408FFFFFFFFFEE7FEE721
:1004A000FEE7FEE7FEE7FEE7FEE7FEE7FEE7FEE724
:1004B000FEE7FEE7FEE7FEE7FEE7FEE7FEE7FEE714
:1004C000FEE7FEE7FEE7FEE7FEE7FEE7FEE7FEE704
:1004D000FEE7FEE7FEE7FEE7FEE7FEE7FEE7FEE7F4
:1004E000FEE7FEE7FEE7FEE7FEE7FEE7FEE7FEE7E4
:1004F000FEE7FEE7FEE7FEE7FEE7FEE7FEE7FEE7D4
:10050000FEE7FEE7FEE7FEE7FEE7FEE7FEE7FEE7C3
:10051000FEE7FEE7FEE7FEE7FEE7FEE7FEE7FEE7B3
:10052000FEE7FEE7FEE7FEE7FEE7FEE7FEE7FEE7A3
:10053000FEE7FEE7FEE7FEE7FEE7FEE7FEE7FEE793
:10054000FEE7FEE7FEE7FEE7FEE7FEE7FEE7FEE783
:10055000FEE71348854600F022F84EF68850CEF2AA
:100560000000016851F47001016000BF00BF00BFCE
:10057000F1EE100A50F04070E1EE100A4FF000006A
:1005800080F314884EF63C71CEF20001086850F0FA
:1005900040700860034804490160FFF7E9BE7047F6
:0C05A0000000022008ED00E00000000850
:020000040802F0
:1000000000000000000000000000000000000000F0
:1000100000000000000000000000000000000000E0
:100020000000000000000000000000000000016669
:100030000F018600003D8601003D680220830044D8
:10004000F430F4301E00000A83014E014413F531F0
:1000500083015AF5330000F4030066000000F40346
:10006000012B000000094A004AFF51004A004AFFE4
:1000700051089800000000AF00AF01AF02AF038F3E
:100080002F008F30008F31008F3200431142108FCC
:1000900021008F2EFF680020F406F402202E00AD10
:1000A000F407000064009A830154800098421142D2
:1000B000104AFF710044244AFF710844257000442F
:1000C0002270084423AE009626AE01962A45210CE4
:1000D000018200D50C4421F535F406F402452E606A
:1000E000002000EFF5358100EF0C018200EF0C4598
:1000F00021128100FFF40700006400DB80006669C4
:100100000020452F453155510045304532555108A5
:1001100045315F0045325F089433AF009437AF013B
:10012000943BAF02943FAF038000B11E0000648394
:10013000014E0145131281012B44131E00006483FC
:10014000014E01451312820139F53180012B7010E7
:100150004A0F52096E012080015A6001200163F5A7
:10016000390009F5390109210D2E15FFFFFFFFFFA9
:10017000FFFFFFFFFFFFFFFFFFFFFFFFFFFFFFFF8F
:10018000FFFFFFFFFFFFFFFFFFFFFFFFFFFFFFFF7F
:10019000FFFFFFFFFFFFFFFFFFFFFFFFFFFFFFFF6F
:1001A000FFFFFFFFFFFFFFFFFFFFFFFFFFFFFFFF5F
:020000040803EF
:020000040804EE
:1000000030B583B04FF0000400944FF0F80501952F
:1000100020464FF003014FF004024FF0010303F0BC
:100020006DF94FF00400294615F064FF4FF003000E
:10003000214640F2AD02C0F6040203F05DFF4FF02E
:10004000010040F2BD01C0F6040140F29D02C0F67D
:10005000040203F051FF4FF010004FF0110102466F
:1000600011F082FE20464FF005014FF0070201F02B
:100070001FF94FF47A7300934FF001004FF0030122
:100080004FF00702034612F0A9F94AF21C20C0F60D
:10009000050007F0A9FE03B030BD00BF08B519B9CF
:1000A0004FF0030016F05CFE08BD00BF08B5012943
:1000B00003D14FF0010016F053FE08BD08B54FF014
:1000C000120000F035FF08BD4AF23C23C0F60503DC
:1000D0001A684EF60C50CEF200000260FEE700BF38
:1000E00008B5FFF7F1FF00BF51E8002FBFF35F8FA6
:1000F00041E80003012B3FF4F7AF1046704700BF03
:1001000013461A462DE9F00F0B460C460D460E46D7
:100110000F46884689468A468B46092AC0F00780E2
:10012000A0E8F80FA2F10902092ABFF4F9AF4FF0D5
:10013000080303FB02F2144B1A44974600F020B860
:1001400000BF00BF046000F01BB800BF80E83000B3
:1001500000F016B880E8700000F012B880E8F000F7
:1001600000F00EB880E8F00100F00AB880E8F00373
:1001700000F006B880E8F00700F002B880E8F00F61
:10018000BDE8F00F704713463C010408EFF31180FF
:100190004FF0800181F3118870474FF0000000BFDD
:1001A00080F31188704700BF30B440F20003C0F6FE
:1001B000000340F28812C0F60002D01A4FEAA001F4
:1001C000B1F5C47F04D81346264A9A4201D324E0ED
:1001D000FEE7254D254C601B20F003054FF0000382
:1001E00040F20002C2F2000240F20001C0F600013B
:1001F00005F10400C5F380045D589D5003F104032C
:10020000834226D109E05C589C5003F104035C58FA
:10021000D45003F104038342F5D14EF60853CEF2D5
:10022000000340F20002C2F200021A604FF0B50172
:10023000CBF26B1143F23850C2F2000001604EF66F
:100240001453CEF200031A6842F01001196030BC5A
:100250007047002CD7D05C589C5003F104038342B4
:10026000D1D1DAE700000008040000088B01000883
:1002700030B4034600283FD002F1100440F20000E1
:10028000C2F2000040F82430002A0ADA12F10C0F02
:1002900036DB02F10C024EF61850CEF2000011547B
:1002A0002EE04EF20015CEF200054CB211EA240405
:1002B00038BF80244EF20041CEF200015454134660
:1002C000002AB8BF02F11F034FEA631005EB80015B
:1002D0004FF01F03C8F200031340002B05DA03F1AF
:1002E000FF3262F01F0303F1010358B24FF0010225
:1002F00002FA00F30B6003E0002AC7DB014DD4E7EC
:1003000030BC704780E100E01EF0040F0CBFEFF33B
:100310000880EFF3098020E9F00F00F001B800BF7A
:1003200010B5026843F2EC43C2F200031A60416860
:10033000596082689A60C168D96002691A6141692E
:10034000596182699A61C169D961026A1A62416A16
:100350005962826A9A62C16AD962026B1A63416BFE
:100360005963826B9A63C16BD96300F140001864D2
:100370004EF62850CEF2000002685A6419F0F4FEDE
:10038000002800F0FB814AF24020C0F6050019F079
:10039000F1FE4EF62C54CEF200042368002B05DA51
:1003A0004AF25020C0F6050019F0E4FE4EF62C513A
:1003B000CEF20001086810F0020F05D04AF260206A
:1003C000C0F6050019F0D6FE4EF62852CEF2000215
:1003D0005478002C72D04AF27820C0F6050019F04B
:1003E000C9FE4EF62853CEF20003597811F0010FE2
:1003F00005D04AF28820C0F6050019F0BBFE4EF683
:100400002850CEF20000427802F00204E3B22BB191
:100410004AF2A820C0F6050019F0ACFE4EF62851AD
:10042000CEF20001487800F00402D4B22CB14AF2B6
:10043000CC20C0F6050019F09DFE4EF62853CEF2F2
:100440000003597801F00800C2B22AB14AF2F02044
:10045000C0F6050019F08EFE4EF62854CEF20004C8
:10046000637803F01001C8B228B14AF21030C0F628
:10047000050019F07FFE4EF62852CEF200025478A5
:1004800004F02003D9B229B14AF23030C0F6050099
:1004900019F070FE4EF62850CEF20000427802F0BD
:1004A0008004E3B253B14EF63851CEF20001096830
:1004B0004AF25030C0F6050019F05CFE4EF62850A6
:1004C000CEF20000428894B2002C5ED04AF2703026
:1004D000C0F6050019F04EFE4EF62853CEF200038A
:1004E000598811F0010F05D04AF28030C0F605009E
:1004F00019F040FE4EF62850CEF20000428802F07D
:100500000204A3B22BB14AF2AC30C0F6050019F0D8
:1005100031FE4EF62851CEF20001488800F0040268
:1005200094B22CB14AF2D030C0F6050019F022FE88
:100530004EF62853CEF20003598801F0080082B22B
:100540002AB14AF21040C0F6050019F013FE4EF62B
:100550002854CEF20004638803F4807188B228B175
:100560004AF24040C0F6050019F004FE4EF628524B
:10057000CEF20002548804F4007399B229B14AF211
:100580005C40C0F6050019F0F5FD4EF62850CEF29D
:1005900000000278002A63D04AF27440C0F60500D9
:1005A00019F0E8FD4EF62854CEF20004237813F03B
:1005B000010F05D04AF28440C0F6050019F0DAFDBB
:1005C0004EF62851CEF20001087800F00202D4B2B3
:1005D0002CB14AF2A440C0F6050019F0CBFD4EF64E
:1005E0002853CEF20003197801F00800C2B22AB1F4
:1005F0004AF2BC40C0F6050019F0BCFD4EF6285486
:10060000CEF20004237803F01001C8B228B14AF2F8
:10061000E040C0F6050019F0ADFD4EF62852CEF2CE
:100620000002147804F02003D9B229B14AF2045030
:10063000C0F6050019F09EFD4EF62850CEF20000DF
:10064000027802F08004E3B253B14EF63451CEF298
:10065000000109684AF22450C0F6050019F08AFD2D
:1006600043F2EC44C2F20004216A4AF25050C0F650
:10067000050019F07FFD616A4AF26450C0F605007A
:1006800019F078FDA16A4AF27850C0F6050019F019
:1006900071FDE16A4AF28C50C0F6050019F06AFD5E
:1006A00021684AF2A050C0F6050019F063FD6168A8
:1006B0004AF2B450C0F6050019F05CFDA1684AF298
:1006C000C850C0F6050019F055FDE1684AF2DC504B
:1006D000C0F6050019F04EFD21694AF2F050C0F64F
:1006E000050019F047FD61694AF20460C0F6050093
:1006F00019F040FDA1694AF21860C0F6050019F032
:1007000039FDE1694AF22C60C0F6050019F032FDAE
:10071000216B4AF24060C0F6050019F02BFD216CF8
:100720004AF25460C0F6050019F024FD616B4AF2EC
:100730006860C0F6050019F01DFDA16B4AF28C60DF
:10074000C0F6050019F016FD43F23450C2F2000065
:1007500002684AF2B060C0F605001146126819F04E
:1007600009FD40F6D003C2F200031A684AF2C860DD
:10077000C0F605001146126819F0FCFCFFF7B0FC4A
:1007800010BD00BF00B506F06BFD002808BF5DF886
:1007900004FBEFF30981EFF3118221E9F40F5DF817
:1007A00004EB1EF0100F08BF21ED108A41F804ED94
:1007B0000B4C2268002A18BF516006F0CDFD22685C
:1007C000516851F804EB1EF0100F08BFB1EC108A0D
:1007D000B1E8F40F82F3118881F3098870470000B3
:1007E0003435002008B540F28570C0F604004FF0A3
:1007F000FF016FF00102FFF73BFD08BDF8B50746AA
:100800000C461E460799089D14F0030F00D0FEE722
:1008100022B1A4EB8500A0F1480401E004F14800F6
:10082000012D01D8A16205E02A4601F0A5FFA7EB42
:100830008507A7624FF0000363604FF01130E0625C
:100840004FF0223121634FF0333262634FF0443373
:10085000A3604FF05530E0604FF0663121614FF0FA
:10086000773262614FF08833A3614FF09930E061D5
:100870004FF0AA3121624FF0BB3262624FF0CC33AD
:10088000A363E663069820644FF0807161646FF0A3
:100890000202226005F11200F8BD00BF62B64EF6FA
:1008A0000453CEF200031A6842F08050186000BF73
:1008B00043F64003C4F202031A6861F35D721A60E2
:1008C000704700BF4FEA00104AF2E063C0F605032C
:1008D0001A584BF28821C0F6050151F822007047E2
:1008E0002DE9F04F8BB083468A46914698469DF994
:1008F00050709DF954609DF958509DF95C1000911D
:100900009DF960200192FFF7DDFF03684AF2E06184
:10091000C0F6050101EB0B1BDBF80420012A02D015
:10092000022A34D119E01C46C3F340310991C3F3C4
:1009300000310891C3F303210791C3F3811106919C
:10094000C3F3C2010591C3F380010491C3F34001D5
:10095000039103F00101029119E043F30F44C3F343
:1009600040710991C3F300710891C3F303610791CA
:10097000C3F381510691C3F3C2410591C3F3804192
:100980000491C3F340410391C3F300410291BAF1D2
:10099000000FA4BF0AF0010ACDF808A0B9F1000FBA
:1009A000A4BF09F00109CDF80C90B8F1000FA4BF65
:1009B00008F00108CDF81080002FA4BF07F007074A
:1009C0000597002EA4BF06F003060696002DA4BFCF
:1009D00005F00F05079500990029A4BF01F001015A
:1009E000089101990029A4BF01F001010991012A90
:1009F00002D0022A35D11AE0029A62F30004039968
:100A000061F34104049A62F38204059961F3C50419
:100A1000069A62F38714079961F30B24089A62F32C
:100A20000C34099961F34D3464F30F0319E0029A11
:100A300062F30004039961F34104049A62F38204AF
:100A4000059961F3C504069A62F38714079961F367
:100A50000B24089A62F30C34099961F34D3464F362
:100A60001F4303600BB0BDE8F08F00BF38B50446EC
:100A70000D46FFF727FF4AF2E063C0F6050303EBDC
:100A800004146168012902D0022903D101E08560C4
:100A900038BD456138BD00BF10B540F20401C4F255
:100AA00002010C684AF6E802C0F60502136824EA5F
:100AB00003044AF25873C0F60503186804430C6037
:100AC00040F20441C4F202010C68506824EA0004B8
:100AD000586804430C6040F60401C4F202010C683B
:100AE000906824EA0004986804430C6040F60441CE
:100AF000C4F202010C68D06824EA0004D8680443F8
:100B00000C6041F20401C4F202010868126920EA93
:100B100002001B6940EA03040C6041F20441C4F284
:100B200002010868086041F60403C4F202031A686F
:100B30001A6041F60444C4F202042168216042F2C2
:100B40000400C4F202000368036040F20C01C4F226
:100B500002010C684AF63812C0F60502106824EA51
:100B600000044AF65C13C0F60503186804430C60E1
:100B700040F20C41C4F202010C68506824EA0004FF
:100B8000586804430C6040F60C01C4F202010C6882
:100B9000906824EA0004986804430C6040F60C4115
:100BA000C4F202010C68D06824EA0004D868044347
:100BB0000C6041F20C01C4F202010868126920EADB
:100BC00002001B6940EA03040C6041F20C41C4F2CC
:100BD00002010868086041F60C03C4F202031A68B7
:100BE0001A6041F60C44C4F202042168216042F20A
:100BF0000C00C4F20200036803604AF6A004C0F6C9
:100C00000504226840F21401C4F202010A6060681F
:100C100040F21443C4F202031860A26840F61401C3
:100C2000C4F202010A60E06840F61443C4F2020311
:100C30001860246941F21402C4F2020214604FF0F9
:100C4000000141F21440C4F20200016041F61403B5
:100C5000C4F20203196041F61444C4F20204216094
:100C600042F21402C4F20202116040F20001C4F226
:100C700002010C684AF60C12C0F60502106824EA5C
:100C800000044AF6C403C0F60503186804430C6068
:100C900040F20041C4F202010C68506824EA0004EA
:100CA000586804430C6040F60001C4F202010C686D
:100CB000906824EA0004986804430C6040F6004100
:100CC000C4F202010C68D06824EA0004D86820430A
:100CD000086041F20001C4F202010868126920EACA
:100CE00002001B691843086041F20041C4F202018E
:100CF0000A680A6041F60003C4F20203186818602B
:100D000041F60041C4F202010A680A6042F200039F
:100D1000C4F20203186818604FF0010004F0ACFA46
:100D200010BD00BF08B543F63002C4F202021368DA
:100D30006FEA53206FEA4021116043F62003C4F2AA
:100D400001031A6842F001001860FFF7A5FE08BD14
:100D50002DE9F0019DF814709DF81860079D4AF286
:100D60008074C0F6050454F820004FEA4104FF2FB8
:100D700012D0D0F80C804AF2007CC0F6050C1CF8AA
:100D8000077007FA04FC4FF0030707FA04F728EA94
:100D900007074CEA0707C760FF2B10D0D0F804C044
:100DA0004AF64C07C0F60507FF5C07FA01F74FF05B
:100DB000010303FA01F32CEA03033B434360FF2ED4
:100DC0000FD087684AF64803C0F605039E5D06FA11
:100DD00004F64FF0030303FA04F327EA0303334353
:100DE0008360B5F1FF3F16D04FEAD10303F108034A
:100DF00050F8236001F007014FEA810105F00F056B
:100E000005FA01F54FF00F0707FA01F126EA010193
:100E1000294340F82310FF2A10D001684AF6341302
:100E2000C0F605039B5C03FA04F34FF0030202FAD9
:100E300004F421EA040143EA01040460BDE8F0017E
:100E4000704700BF2DE9F007079F089E099D4AF2F1
:100E50008074C0F6050454F820004FEA41044FEABC
:100E6000D10801F0070C4FEA8C0C6FB1D0F80C9050
:100E700029FA04FA0AF003094AF27C7AC0F6050A54
:100E80001AF8099087F8009053B1476827FA01F1E2
:100E900001F001014AF63017C0F60507795C1970B8
:100EA00056B1836823FA04F303F003034AF64401BE
:100EB000C0F60501CB5C337045B108F1080850F865
:100EC000281021FA0CFC0CF00F032B6052B10068C3
:100ED00020FA04F404F003044AF20471C0F6050198
:100EE0000B5D1370BDE8F007704700BF4AF2F47362
:100EF000C0F6050353F820100A684AF65003C0F6FE
:100F0000050353F820100A404AF68013C0F6050383
:100F100053F82000824214BF00200120704700BF18
:100F20004AF28073C0F6050353F820000069704749
:100F30004AF65003C0F6050353F820307BB139B1AF
:100F40004AF20871C0F6050151F82020136070477D
:100F50004AF2A472C0F6050252F8200003607047FE
:100F60003A2800F2938000EB80004AF6D413C0F6D2
:100F7000050353F8202002F1FF300D2800F286808F
:100F8000DFE800F0071019222B343D464F58616A04
:100F9000737C43F64400C4F20200036861F300036B
:100FA0000360704743F64003C4F202031A6861F31A
:100FB00000021A60704743F64003C4F20203186847
:100FC00061F341001860704743F64000C4F202002C
:100FD000026861F382020260704743F64000C4F287
:100FE0000200036861F3C3030360704743F64003E4
:100FF000C4F202031A6861F304121A60704743F6E0
:101000004003C4F20203186861F34510186070478A
:1010100043F64400C4F20200026861F34102026038
:10102000704743F64400C4F20200036861F31043C2
:101030000360704743F64403C4F202031A6861F385
:1010400051421A60704743F64403C4F20203186821
:1010500061F392401860704743F64000C4F202000A
:10106000026861F386120260704743F64000C4F2E2
:101070000200036861F3C7130360704743F640033F
:10108000C4F202031A6861F308221A60704700BFB5
:1010900000EB80004AF6D413C0F6050353F8202075
:1010A0004BF2CC21C0F6050151F82200704700BF79
:1010B0002DE9F84F04468A46914698469DF92870D6
:1010C0009DF92C609DF930503A2800F2B680FFF768
:1010D000DFFF04EB84024AF6D413C0F6050303EBEA
:1010E00082035A68022A94BF8369C369016A02F1C4
:1010F000FF3CBCF1030F2ED8DFE80CF002180218F9
:101100006FF30103BAF1000FC8BF6AF38203B9F1AC
:10111000000FC8BF69F3C303B8F1000FC8BF68F37D
:101120000613002F17DD67F3C71314E06FF30923CD
:10113000BAF1000FC8BF6AF38A23B9F1000FC8BF24
:1011400069F3CB23B8F1000FC8BF68F30E33002F4B
:10115000C8BF67F3CF3302F1FF37032F44D8DFE86E
:1011600007F002142638332C04D1002E06DD66F376
:10117000820103E0002EC8BF66F30001002DC8BF46
:1011800065F341016FF3C30130E0362C04D1002E2A
:1011900006DD66F3861103E0002EC8BF66F3041176
:1011A000002DC8BF65F345116FF3C7111EE0382C41
:1011B00004D1002E06DD66F38A2103E0002EC8BFAD
:1011C00066F30821002DC8BF65F349216FF3CB21D9
:1011D0000EE0002EC8BF66F30C31002DC8BF65F3CA
:1011E0004D316FF3CF3103E0022A01D8836100E073
:1011F000C361016204EB84044AF6D410C0F6050012
:1012000050F82430012B02D0082B16D10BE04AF6FF
:10121000D013C0F605031A6840F24401C4F201017C
:101220000A60BDE8F88F4AF6D012C0F605021168D0
:1012300040F24440C4F201000160BDE8F88F00BFF5
:1012400038B504460D46FFF723FF04EB84014AF648
:10125000D413C0F6050303EB8104626802F1FF3189
:1012600003290AD8DFE801F002040608456338BD07
:10127000856338BDC56338BD056438BD40F20C23B5
:10128000C2F2000318684FF000020261016801F029
:101290001003002B0CBF01204FF0FF3040F2102351
:1012A000C2F200031A8810FA82F188B218807047DF
:1012B0002DE9F04F89B0154640F20C23C2F200032D
:1012C0004FF000021A604FEA01104AF67064C0F64F
:1012D00005042458142900F2F480092C00F2F4804B
:1012E0004AF6D073C0F6050353F82430002B00F003
:1012F000EE804FEA05124AF67060C0F6050082588B
:10130000944240F0E78004F1FF36072E4DD8DFE825
:1013100006F03404101C284C4C4043F64007C4F23D
:101320000207386840F001023A604FF00006059667
:101330003EE043F64007C4F20207386840F002027C
:101340003A604FF00106059632E043F64007C4F2DA
:101350000207386840F004023A604FF00106059633
:1013600026E043F64007C4F20207386840F008025E
:101370003A604FF0000605961AE043F64407C4F2BF
:101380000207386840F001023A604FF00106059606
:101390000EE043F64407C4F20207386840F0020248
:1013A0003A604FF00106059602E04FF001070597FD
:1013B00040F20C208246C2F2000ACAF800304AF617
:1013C0007069C0F6050909EB011898F804B0D8F85F
:1013D000081004910DF11F0300934FF000060196D1
:1013E0000296584632460DF11E03FFF72BFD9DF87D
:1013F0001E309DF81F2000924FF003070197D8F888
:101400000C000290584604993A46FFF7A1FC09EBFC
:10141000051595F80490D5F808800DF11F0100918D
:10142000019602964846414632460DF11E03FFF7EB
:1014300009FD9DF81F3000930197EA680292484623
:1014400041463A463346FFF783FCDAF800104BF288
:101450000400C0F6050003680B604BF20002C0F602
:101460000502106888604AF6FC73C0F605031A6826
:101470008A610E626FF07F40C862059B93B14AF6A5
:10148000F872C0F605021068C86041F27D20C0F60F
:1014900004004FF00F014AF6C073C0F605031A5757
:1014A000FEF7E6FE40F20C21C2F2000108684FF0A0
:1014B00000028262036843F0010101604FF0010005
:1014C0000AE04FF0000007E04FF0000004E04FF0AA
:1014D000000001E04FF0000009B0BDE8F08F00BF50
:1014E00040F20C23C2F200031B689BB1A8B91A6832
:1014F0006FF300021A604FF00000586240F21021B2
:10150000C2F2000108801A6842F0010018604FF032
:10151000010070474FF0000070474FF00000704727
:1015200010B483B040F20C23C2F200031B6803B373
:1015300010BB40F21022C2F20002586A148840EA3E
:101540000440019000BF00BF00BF00BF00BF586A49
:10155000148840EA04400090019C00988442ECD139
:10156000DDED017AB8EEE70A81ED000A4FF00100E7
:1015700004E04FF0000001E04FF0000003B010BCA9
:10158000704700BF40F20C23C2F200031B689BB1FE
:10159000A8B91A686FF300021A6059624FEA114144
:1015A00040F21020C2F2000001801A6842F00101EE
:1015B00019604FF0010070474FF0000070474FF086
:1015C0000000704743F67403C4F20203186847F240
:1015D0000402C4F20002136840F21222C2F20002B6
:1015E0004FF00001117013F0010F04D010464FF0BE
:1015F000040202703EE04FEA106212F0600F07D062
:1016000040F21221C2F200014FF020030B7031E0D2
:1016100002F00401C9B239B140F21220C2F2000056
:101620004FF04002027025E0C3F3400343EAD0606C
:1016300010F0010F07D040F21221C2F200014FF06A
:1016400080030B7016E002F01001CBB23BB140F208
:101650001220C2F200004FF0010202700AE002F014
:101660000202D0B230B140F21221C2F200014FF0BA
:1016700002030B7043F67401C4F202010B6843F0DD
:101680008070086047F20001C4F200010A6842F06D
:1016900008030B6043F23450C2F20000016840F2CC
:1016A0001422C2F200021160704700BF40F2122300
:1016B000C2F200031878704708B547F61021C1F64A
:1016C000FF714FF00C0216F06FFF4FF00C0008BDD9
:1016D00010B542F20803CEF204031A6842F010007B
:1016E000186041F28970C0F604004FF00F014FF00E
:1016F0003602FEF7BDFD43F64001C4F202010C685C
:1017000044F010030B6041F20004C4F200044BF2F9
:101710000802C0F60502106820604BF29021C0F666
:101720000501886915F0FEFC15A3D3E9002315F027
:101730003DFF4FF000024FF00003C3F6F07315F0C9
:10174000EFFD15F05BFD41F22C03C4F2000318809D
:1017500041F22800C4F200004FF0000202804BF278
:101760000C01C0F60501086841F20C03C4F2000345
:101770001860228842F00101218010BDAFF3008083
:101780002D431CEBE2362A3F684620F007018D46C8
:1017900001B541F21003C4F200034FF000021A60D9
:1017A00006F078F8BDE801408546704770B50446FC
:1017B000B0F5CC7F2FD940F23233984216D940F29F
:1017C0006560844215D940F6CB418C4214D941F66C
:1017D0009712944213D943F22F36B44212D946F2EB
:1017E0005F639C4298BF06250ED90FE04FF00105BC
:1017F0000AE04FF0020507E04FF0030504E04FF068
:10180000040501E04FF00505072D06D1FEF768FC41
:101810004FF0070501E04FF00005FEF7B7FC064664
:1018200004EB84044FEAC4004BF21001C0F605013A
:1018300051F83520B0FBF2F39CB2012C05D9B4F578
:10184000805F04D3FEF74CFC01E04FF0020443F24A
:101850000000C4F2000045F2555101604BF2100245
:10186000C0F6050202EBC5052B7943F20401C4F270
:1018700000010B6043F20802C4F2000214604AF651
:10188000AA2303603046FEF78BFC70BD08B543F217
:101890000003C4F200034CF6CC421A604FF0C800BB
:1018A000FFF784FF08BD00BF43F20003C4F200034A
:1018B0004AF6AA221A60704710B5044643F2100394
:1018C000C4F20003186810F0010F74D04FF032001A
:1018D00007F09CFA43F21001C4F200010A6812F00A
:1018E000010F68D04FF0320007F090FA43F2100376
:1018F000C4F20003186810F0010F5CD04FF0320002
:1019000007F084FA43F21001C4F200010A6812F0F1
:10191000010F50D04FF0320007F078FA43F2100375
:10192000C4F20003186810F0010F44D04FF03200E9
:1019300007F06CFA43F21001C4F200010A6812F0D9
:10194000010F38D04FF0320007F060FA43F2100375
:10195000C4F20003186810F0010F2CD04FF03200D1
:1019600007F054FA43F21001C4F200010A6812F0C1
:10197000010F20D04FF0320007F048FA43F2100375
:10198000C4F20003186810F0010F14D04FF03200B9
:1019900007F03CFA43F21001C4F200010A6812F0A9
:1019A000010F08D04FF0320007F030FA43F2100375
:1019B000C4F200031B682046FFF7F8FE10BD00BF0D
:1019C00002469CF8043043B1DCF8000040B140F21C
:1019D000A421C2F2000141F82200DCF8000050B955
:1019E00040F2A423C2F2000353F8220049F6404219
:1019F000002808BF104670474FF0010303FA00F0BB
:101A0000C0F34000704700BF70B50D464BF2D403E1
:101A1000C0F6050353F82040002C45D000EB8000B1
:101A200040F21826C2F2000606EBC00630464FF020
:101A3000000104F0ABFE122D07D142F20431C4F2D2
:101A400001010A6842F480030B60606B65F30400D7
:101A50006063E36C4FF0050007F0D8F9A16841F02E
:101A60008042A260236813F0020FFBD0E46C122DB9
:101A700016D142F20430C4F2010001686FF39651AE
:101A8000016042F20002CEF2040213684FEA0350F2
:101A90004FEA105140F2194291420CBFA400640079
:101AA000304604F081FF01E04FF0FF34204670BD66
:101AB00038B52DED028B044608EE101A4BF248059E
:101AC000C0F6050505EB8005F7EE007AB4EEE78A6F
:101AD000F1EE10FA09DC084615F07AFF00289FEDB8
:101AE000260A18BFB0EE408A01E0B7EE008A2B78D4
:101AF000012B1CD16878FFF7CBFAD0ED0B1A6D786B
:101B0000B8EE612A62EE082A12EE900A15F0B0FBD8
:101B10004FF000024FF00003C3F6E07315F002FC33
:101B200015F06CFB01462846FFF78AFB18E0022BF4
:101B300016D16D78DFED110A28EE201A11EE100A89
:101B400015F096FB4FF000024FF00003C3F6E07370
:101B500015F0E8FB15F052FB01462846FEF786FF1C
:101B600040F29020C2F2000000EB840484ED008A71
:101B7000BDEC028B38BD00BF0000000000F07F45C7
:101B800010B54FF000044FF000002146FFF790FF22
:101B90004FF001002146FFF78BFF4FF00200214676
:101BA000FFF786FF4FF003002146FFF781FF4FF05C
:101BB00004002146FFF77CFF40F20C03C4F202034D
:101BC0001A681A6040F20C40C4F202000168016019
:101BD00040F60C03C4F202031A684BF28800C0F608
:101BE0000500816822EA01024BF25C00C0F60500A4
:101BF00081680A431A6040F60C43C4F202031A6873
:101C00001A6041F20C00C4F202000168016041F266
:101C10000C43C4F202031A681A6041F60C00C4F2C5
:101C200002000168016041F60C43C4F202031A6825
:101C30001A6042F20C00C4F202000168016040F236
:101C40000003C4F202031A681A6040F20040C4F2B2
:101C500002000168016040F60003C4F202031A6842
:101C60004BF2B000C0F60500816822EA01024BF297
:101C7000E400C0F6050081680A431A6040F600439C
:101C8000C4F202031A681A6041F20000C4F20200B2
:101C90000168016041F20043C4F202031A681A604D
:101CA00041F60000C4F202000168016041F6004301
:101CB000C4F202031A681A6042F20000C4F2020081
:101CC0000168016010BD00BF08B502280ED84BF2B4
:101CD0000C13C0F60503195CFF290AD04BF2E00291
:101CE000C0F60502105CFFF78FFE08BD4FF0FF3015
:101CF00008BD4FF0FF3008BD10B50446FFF7E4FF04
:101D000007EE900AB8EE677A4BF20C13C0F60503A3
:101D1000185D11280BD147F62A21C1F6FF710A88F8
:101D200001EE102AF8EEC11AC1EE870A03E09FED1A
:101D3000030AC7EE000A10EE900A10BD00F07F45BE
:101D400040F29023C2F2000303EB8000006870476A
:101D500038B50D46044600B30E2801D9FEF7C0F988
:101D60004BF29023C0F6050353F8240055B1B0FBA5
:101D7000F5F14FEA114202F10103B0FBF3F0B0FBC1
:101D8000F5F502E04FF000052A464BF2CC21C0F6F3
:101D9000050151F824309A62DD6238BD10B582B079
:101DA00000918DF80420052840F0E2804FF00000FB
:101DB000FFF722FE48B1EC464FF00000FFF700FEAF
:101DC00001464FF00000FFF7C3FF4FF00100FFF79F
:101DD00013FE48B1EC464FF00100FFF7F1FD01465C
:101DE0004FF00100FFF7B4FF4FF00200FFF704FED1
:101DF00048B1EC464FF00200FFF7E2FD01464FF01C
:101E00000200FFF7A5FF4FF00300FFF7F5FD48B113
:101E1000EC464FF00300FFF7D3FD01464FF00300FF
:101E2000FFF796FF4FF00400FFF7E6FD48B1EC46E0
:101E30004FF00400FFF7C4FD01464FF00400FFF728
:101E400087FF4FF00500FFF7D7FD48B1EC464FF094
:101E50000500FFF7B5FD01464FF00500FFF778FFDD
:101E60004FF00600FFF7C8FD48B1EC464FF0060002
:101E7000FFF7A6FD01464FF00600FFF769FF4FF0A0
:101E80000700FFF7B9FD48B1EC464FF00700FFF738
:101E900097FD01464FF00700FFF75AFF4FF008008B
:101EA000FFF7AAFD48B1EC464FF00800FFF788FDA8
:101EB00001464FF00800FFF74BFF4FF00900FFF716
:101EC0009BFD48B1EC464FF00900FFF779FD014654
:101ED0004FF00900FFF73CFF4FF00A00FFF78CFDC1
:101EE00048B1EC464FF00A00FFF76AFD01464FF09B
:101EF0000A00FFF72DFF4FF00B00FFF77DFD48B103
:101F0000EC464FF00B00FFF75BFD01464FF00B0076
:101F1000FFF71EFF4FF00C00FFF76EFD48B1EC46D7
:101F20004FF00C00FFF74CFD01464FF00C00FFF79F
:101F30000FFF4FF00D00FFF75FFD48B1EC464FF08B
:101F40000D00FFF73DFD01464FF00D00FFF700FFCC
:101F50004FF00E00FFF750FD48B3EC464FF00E0077
:101F6000FFF72EFD01464FF00E00FFF7F1FE1EE0D9
:101F70004BF24803C0F6050313F82010012916D1CF
:101F80004BF24802C0F6050202EB8000447804EBF5
:101F900084034AF6D411C0F6050151F82340EC46FB
:101FA0002046FFF70DFD01462046FFF7D1FE02B0A7
:101FB00010BD00BF70B586B040F21825C2F2000512
:101FC0004BF21814C0F605042846214604F0C6FB5F
:101FD00005F12800214604F0C1FB05F1500021461F
:101FE00004F0BCFB43F64403C4F202031A6842F453
:101FF00080701860196841F400761E604BF2AC05E1
:10200000C0F605052C6842F20433C4F201031C60DB
:102010004BF20812C0F60502106842F20401C4F245
:102020000101086042F20416C4F2010630604BF26E
:102030001415C0F605052C6842F20C03C4F2010326
:102040001C6042F20C12C4F2010214604BF28400D4
:10205000C0F60500016842F21006C4F201063160C4
:1020600042F21015C4F2010529604BF21C14C0F6AF
:102070000504236842F22C02C4F20102136042F20A
:102080002C10C4F2010003604BF21011C0F60501E0
:102090000E6842F20805C4F201052E6042F20814EF
:1020A000C4F2010426604FF034004FF00101FEF746
:1020B00057FF4FF037004FF00101FEF751FF4FF08F
:1020C00039004FF00101FEF74BFF4FF00004009480
:1020D0004FF00106019602944FF03400214632463B
:1020E0004FF00603FEF7E4FF4AF6D415C0F60505E7
:1020F00095F81C04D5F8201400940194D5F81834F0
:1021000002934FF003022346FEF722FE009401964D
:1021100002944FF03700214632464FF00603FEF797
:10212000C7FF95F85804D5F85C1400940194D5F8CD
:10213000542402924FF003022346FEF709FE009456
:10214000019602944FF03900214632464FF00603C3
:10215000FEF7AEFF95F88004D5F88414009401943E
:10216000D5F87C5402954FF003022346FEF7F0FDAC
:102170004FF0050021462246FFF710FE4FF0000504
:1021800020462946FFF794FC30462946FFF790FC8D
:102190004FF002002946FFF78BFC4FF00300294661
:1021A000FFF786FC4FF004002946FFF781FC30461C
:1021B000FFF722FC50B14BF2CC20C0F6050041687D
:1021C0004BF28004C0F6050423680B604FF0020058
:1021D000FFF712FC50B14BF2CC22C0F60502956815
:1021E0004BF28000C0F60500016829604FF0030043
:1021F000FFF702FC50B14BF2CC24C0F60504E368B3
:102200004BF28002C0F6050215681D604FF0040015
:10221000FFF7F2FB50B14BF2CC20C0F6050001698C
:102220004BF28004C0F6050423680B604FF00500F4
:10223000FFF7E2FB50B14BF2CC22C0F60502556924
:102240004BF28000C0F60500016829604FF00600DF
:10225000FFF7D2FB50B14BF2CC24C0F60504A369C2
:102260004BF28002C0F6050215681D604FF00700B2
:10227000FFF7C2FB50B14BF2CC20C0F60500C1699C
:102280004BF28004C0F6050423680B604FF0080091
:10229000FFF7B2FB50B14BF2CC22C0F60502156A33
:1022A0004BF28000C0F60500016829604FF009007C
:1022B000FFF7A2FB50B14BF2CC24C0F60504636AD1
:1022C0004BF28002C0F6050215681D604FF00A004F
:1022D000FFF792FB50B14BF2CC20C0F60500816AAB
:1022E0004BF28004C0F6050423680B604FF00B002E
:1022F000FFF782FB50B14BF2CC22C0F60502D56A43
:102300004BF28000C0F60500016829604FF00C0018
:10231000FFF772FB50B14BF2CC24C0F60504236BDF
:102320004BF28002C0F6050215681D604FF00D00EB
:10233000FFF762FB50B14BF2CC20C0F60500416BB9
:102340004BF28004C0F6050423680B604FF00E00CA
:10235000FFF752FB50B14BF2CC22C0F60502956B51
:102360004BF28000C0F60500016829604FF00000C4
:102370004FF00101FEF79CFA4FF000000146FEF716
:1023800075FB4FF0000400940194029403940494AC
:1023900020464FF001010A462346FEF7A1FA4AF211
:1023A000E065C0F60505287AE96800940194029476
:1023B0004FF002022346FEF7CBFC4FF0010001462E
:1023C000FEF776FA4FF001002146FEF74FFB00942E
:1023D00001940294039404944FF0010001460246D4
:1023E0002346FEF77DFA287EE96900940194029461
:1023F0004FF002022346FEF7ABFCFFF7C1FB06B02D
:1024000070BD00BF10B504464FF000004FF0110141
:10241000FFF7FAFA47F62A23C1F6FF73198807EE89
:10242000901AB8EE670A06EE900AB8EE667AC0EE29
:10243000070AC4ED000A4FF0010010BD00000000C3
:1024400010B504464FF000004FF01201FFF7DCFA20
:1024500007EE900AB8EE677A9FED0B0AC7EE000A06
:1024600010EE900A14F004FF05A3D3E9002315F041
:102470009DF814F019FF20604FF0010010BD00BF5F
:102480006666666666660A4000F07F45AFF30080C8
:1024900010B504464FF000004FF01001FFF7B4FAFA
:1024A00007EE900AB8EE677A9FED1B0AC7EE000AA6
:1024B00010EE900A14F0DCFE11A3D3E9002315F00E
:1024C00075F814F0F1FE14F0D3FE0FA3D3E9002346
:1024D00014F026FF0EA3D3E9002315F01DF94FF0E9
:1024E00000024FF00003C4F2390314F01BFF14F094
:1024F000DBFE20604FF0010010BD00BFAFF3008095
:102500006666666666660A4052B81E85EB51E83F0D
:102510007B14AE47E17A643F00F07F45AFF3008063
:1025200030B472B64BF23013C0F605031A684EF69B
:102530003470CEF2000002604BF23411C0F6050197
:102540000A684EF68853CEF200031A604BF2381038
:10255000C0F60500016842F20802CEF204021160E2
:102560004BF22013C0F60503186842F20C01CEF2BC
:102570000401086043F60003C4F202031A6842F43F
:102580008030186019460B6813F4003FFBD043F607
:102590004000C4F20200026842F08051016047F23C
:1025A0000003C4F20003186840F480421A604BF242
:1025B0002811C0F60501086843F60803C4F20203B7
:1025C00018604BF22C12C0F60502116843F6004069
:1025D000C4F2020001604BF22413C0F605031A682E
:1025E00043F60401C4F202010A6043F60000C4F29B
:1025F0000200036843F0807202600146086810F030
:10260000007FFBD043F60803C4F202031A684FF0C0
:10261000020161F301021A601846036803F00C021C
:10262000082AFAD143F64401C4F20201086840F4D2
:1026300080430B6043F63000C4F20200026842F4AB
:102640008011016047F20003C4F200031A6842F4EB
:102650008071196047F20403C4F200031A6842F45F
:1026600000711960036843F48022026043F614404D
:10267000C4F2020001684AF23823C0F605031B6861
:102680004BF23C12C0F6050210686FEA0002594096
:102690000A4206D04AF23820C0F605004178CC291B
:1026A00004D12A4B2A49994221D344E043F60841F8
:1026B000C4F2020142F63B20C0F61900086046F65B
:1026C0007F60C4F65D400860134043F61442C4F2D4
:1026D00002021360136843F00201116043F60C40DC
:1026E000C4F20200026812F4803FFBD1D9E7194C12
:1026F000194D281B20F003054FF0000340F20002A3
:10270000C1F200024DF2F441C0F6050105F10404E6
:10271000C5F380005D589D5003F10403A3420CD122
:1027200009E05858985003F104035858985003F1A1
:102730000403A342F5D130BC70470028F1D05858AB
:10274000985003F10403A342EBD1F4E7801106088B
:10275000F4D40508F8D405088311060843F63003BD
:10276000C4F202031A6842F400101860196841F4B8
:1027700080021A60704700BF2DE9F0011546002A5B
:1027800066D040F6E003C2F2000353E8002F02F1E6
:10279000010243E80024012CF7D04BF24012C0F6AE
:1027A0000502146846F20846C4F2020634604BF291
:1027B0004C17C0F605073A6846F22843C4F20203F4
:1027C0001A604FF6FF7846F2304CC4F2020C46F223
:1027D0003447C4F2020746F22C46C4F202061C46F5
:1027E000454534BF2B464346CCF800103860336073
:1027F000226842F001022260ED1A4FEA8303C918F1
:10280000C018226812F0010FFBD1002DE8D140F66C
:10281000E003C2F2000353E8002FA2F1010243E8F3
:102820000024012CF7D053E8002FB2F1004F0DD156
:102830004FF0000243E80024012CF4D04EF604507F
:10284000CEF20000016841F080510160BFF32F8F8C
:10285000BDE8F001704700BF70B41646002A37D0BB
:1028600046F21045C4F202052C6814F0010FFBD1AA
:102870004BF24812C0F60502146846F20842C4F250
:102880000202146046F21842C4F20202116046F2DB
:102890001C41C4F20201086046F21440C4F2020076
:1028A00006604BF24412C0F60502116846F2104071
:1028B000C4F202000160026842F0010101603BB114
:1028C00046F21040C4F20200036813F0010FFBD17E
:1028D00070BC704743F61043C4F202031868002826
:1028E0000DDA43F60441C4F2020140F22312C4F2AD
:1028F00067520A6048F6AB13CCF6EF530B6043F611
:102900001040C4F20200016801F00042002A14BF26
:1029100002200020704700BF43F61043C4F20203B8
:102920001868002807DB43F61041C4F202010A6868
:1029300042F000430B60704700F17840B0F5801F13
:102940002CBF0020012070472DE9F04F83B00646D0
:102950000D46FFF7F1FF002856D02846FFF7ECFFA1
:10296000002854D0AE4255D8FDF710FC0190FFF777
:10297000B1FF0446002841D106F178434FEA933075
:102980004BF25412C0F6050212F8008041F2883072
:10299000FEF792FF4FF0020943F6104BC4F2020B10
:1029A00043F60C47C4F202074BF29C1AC0F6050A24
:1029B000FEF77AFF494668F3C60169F3092141F43D
:1029C0008033CBF80030386810F4803FFBD15AF8E0
:1029D0002820B61808F101085FFA88F8B542E7D256
:1029E0004FF06400FEF768FF4BF29411C0F605014A
:1029F000086843F61043C4F202031860FFF78CFF27
:102A00000198FDF7CDFB07E04FF0020404E04FF022
:102A1000020401E04FF00204204603B0BDE8F08F4D
:102A20002DE9F04106460C4615460846FFF784FF9F
:102A3000002861D005F1FF302018FFF77DFF002846
:102A40005DD040F6E003C2F2000353E8002F02F12C
:102A5000010243E800210129F7D0FFF73BFF0746B9
:102A600030BB4BF29811C0F605010A6843F61040DE
:102A7000C4F2020002608DB106F1FF3843F60C4645
:102A8000C4F20206336813F4803FFBD118F8011F2B
:102A900004F8011BFEF708FF013DF3D14BF250147F
:102AA000C0F60504226843F61040C4F2020002603A
:102AB000FFF732FF40F6E003C2F2000353E8002FB5
:102AC000A2F1010243E80024012CF7D053E8002FC3
:102AD000B2F1004F0DD14FF0000243E80024012C69
:102AE000F4D04EF60450CEF20000016841F080515F
:102AF0000160BFF32F8F04E04FF0020701E04FF0B9
:102B000002073846BDE8F08140F2E823C2F2000334
:102B100018684BF27C22C0F60502116801604FF084
:102B2000000303604BF28022C0F605021168416089
:102B30004BF27823C0F605031A68C2614FF00D010D
:102B400001624BF28423C0F605031A6802607047E5
:102B500040F2E023C2F200031868704770B4856841
:102B6000C668446806FB05404118196040F2E02041
:102B7000C2F20000006881420CD2521890420CD37D
:102B800040F2E420C2F200000268891819604FF098
:102B9000010004E04FF0000001E04FF0000070BCC5
:102BA000704700BF40F28813C2F200034FF00002EA
:102BB0001A70704710B540F28813C2F200031878FB
:102BC00040B140F28814C2F2000404F0A3F9217865
:102BD0000029FAD140F28813C2F200034FF001023B
:102BE0001A7010BD2DE9F0410546FEF75DFE4FF06D
:102BF0001E044FF0000840F2E826C2F200064FF033
:102C00000107052D26D8DFE805F0030A0F14191E69
:102C10003268936983F00200C0F340011BE0306822
:102C2000416901F0010116E032685369C3F34001C4
:102C300011E030684169C1F3C0110CE0326853699A
:102C4000C3F3801107E03368986980F0010101F057
:102C5000010100E0414689B933685A6912F4807F66
:102C600010D1586910F4806F10D1384606F0CEF8B4
:102C7000013CC6D14FF00000BDE8F0814FF00100EB
:102C8000BDE8F0814FF00000BDE8F0814FF000009A
:102C9000BDE8F08138B5044640F2E823C2F20003F3
:102CA0001868816911F0020F7ED0FFF72DFF4FF0F9
:102CB0000000FFF797FF40F2E822C2F2000213681B
:102CC000986910F0020F6FD04DE040F2EC25C2F28F
:102CD00000052B78032B05D1FF2C06D9E4B24FF069
:102CE000A20204E04FF0A00201E04FF0A00240F287
:102CF000E825C2F20005286802614FF00200FFF7E4
:102D000071FF29688B6913F0010F08D04A6912F42A
:102D1000806F00F0CA820D6845F4007008604FF0C3
:102D2000050004F029F94FF0000518E0042B0CD140
:102D300040F2E821C2F200010B68C4F307221A61D5
:102D40004FF00300FFF74EFF38B140F2E820C2F227
:102D500000000168E4B20C6101E04FF00005281C9E
:102D600018BF012038BD4FF0000038BD4FF0000003
:102D700038BD4FF0000038BD4FF0000038BD4FF0B7
:102D8000000038BD4FF0000038BD4FF0000038BDE6
:102D90004FF0000038BD4FF0000038BD4FF000008C
:102DA00038BD4FF0000038BD40F2E821C2F200010A
:102DB0000B684FF0000058611A6860F349221A60EE
:102DC000196841F4807018604FF00100FFF70AFFA6
:102DD0000028CBD040F2EC25C2F200052B78032B63
:102DE00005D1FF2C06D9E4B24FF0A20204E04FF067
:102DF000A00201E04FF0A00240F2E825C2F2000577
:102E000029680A614FF00200FFF7ECFE2868836929
:102E100013F0010F08D0426912F4806F00F048826D
:102E2000016841F4007303604FF0050004F0A4F85A
:102E300040F2E820C2F2000003684FF0000159613F
:102E40001A6861F349221A60186840F480711960A9
:102E50004FF00100FFF7C6FE00288AD040F2EC25B3
:102E6000C2F200052B78032B05D1FF2C06D9E4B262
:102E70004FF0A20204E04FF0A00201E04FF0A002E8
:102E800040F2E825C2F20005286802614FF0020016
:102E9000FFF7A8FE29688B6913F0010F08D04A6973
:102EA00012F4806F00F00782086840F400730B6032
:102EB0004FF0050004F060F840F2E821C2F2000192
:102EC00008684FF000034361026863F3492202601F
:102ED000016841F4807303604FF00100FFF782FE48
:102EE00000283FF449AF40F2EC25C2F200052878F3
:102EF000032805D1FF2C06D9E4B24FF0A20204E06A
:102F00004FF0A00201E04FF0A00240F2E825C2F22B
:102F1000000529680A614FF00200FFF763FE2B6885
:102F2000986910F0010F08D05A6912F4806F00F010
:102F3000C581196841F4007018604FF0050004F075
:102F40001BF840F2E823C2F2000318684FF00001BA
:102F50004161026861F349220260036843F48071B1
:102F600001604FF00100FFF73DFE00283FF407AF7E
:102F700040F2EC25C2F200052878032805D1FF2C89
:102F800006D9E4B24FF0A20204E04FF0A00201E043
:102F90004FF0A00240F2E825C2F200052B681A614A
:102FA0004FF00200FFF71EFE2968886910F0010F3C
:102FB00008D04A6912F4806F00F083810B6843F4F3
:102FC000007008604FF0050003F0D6FF40F2E821E2
:102FD000C2F200010B684FF0000058611A6860F3FC
:102FE00049221A60196841F4807018604FF001009E
:102FF000FFF7F8FD00283FF4C5AE40F2EC25C2F221
:1030000000052B78032B05D1FF2C06D9E4B24FF035
:10301000A20204E04FF0A00201E04FF0A00240F253
:10302000E825C2F2000529680A614FF00200FFF7A7
:10303000D9FD2868836913F0010F08D0426912F4A2
:10304000806F00F04181016841F4007303604FF02C
:10305000050003F091FF40F2E820C2F2000003688F
:103060004FF0000159611A6861F349221A6018682B
:1030700040F4807119604FF00100FFF7B3FD0028A4
:103080003FF483AE40F2EC25C2F200052B78032B0F
:1030900005D1FF2C06D9E4B24FF0A20204E04FF0B4
:1030A000A00201E04FF0A00240F2E825C2F20005C4
:1030B000286802614FF00200FFF794FD29688B69D0
:1030C00013F0010F08D04A6912F4806F00F0FF80FE
:1030D000086840F400730B604FF0050003F04CFFEC
:1030E00040F2E821C2F2000108684FF0000343619A
:1030F000026863F349220260016841F4807303604F
:103100004FF00100FFF76EFD00283FF441AE40F2A2
:10311000EC25C2F200052878032805D1FF2C06D93A
:10312000E4B24FF0A20204E04FF0A00201E04FF041
:10313000A00240F2E825C2F2000529680A614FF0BA
:103140000200FFF74FFD2B68986910F0010F08D0BF
:103150005A6912F4806F00F0BD80196841F4007064
:1031600018604FF0050003F007FF40F2E823C2F2B9
:10317000000318684FF000014161026861F34922C1
:103180000260036843F4807101604FF00100FFF7B3
:1031900029FD00283FF4FFAD40F2EC25C2F2000506
:1031A0002878032805D1FF2C06D9E4B24FF0A202FB
:1031B00004E04FF0A00201E04FF0A00240F2E82549
:1031C000C2F200052B681A614FF00200FFF70AFDFA
:1031D0002968886910F0010F07D04A6912F4806FDE
:1031E0007BD00B6843F4007008604FF0050003F0DB
:1031F000C3FE40F2E821C2F200010B684FF000006C
:1032000058611A6860F349221A60196841F48070A5
:1032100018604FF00100FFF7E5FC00283FF4BEAD59
:1032200040F2EC25C2F200052B78032B05D1FF2CD0
:1032300006D9E4B24FF0A20204E04FF0A00201E090
:103240004FF0A00240F2E825C2F2000529680A61A9
:103250004FF00200FFF7C6FC2868836913F0010FE6
:1032600007D0426912F4806F3AD0016841F40073CC
:1032700003604FF0050003F07FFE40F2E820C2F249
:10328000000003684FF0000159611A6861F3492298
:103290001A60186840F4807119604FF00100FFF760
:1032A000A1FC00287FF411AD7BE54FF0010519E08A
:1032B0004FF00A0516E04FF0090513E04FF008053E
:1032C00010E04FF007050DE04FF006050AE04FF063
:1032D000050507E04FF0040504E04FF0030501E0A9
:1032E0004FF0020540F2EC21C2F200010B7803F12D
:1032F000FF32D0B201283FF619AD19E52DE9F041B2
:1033000084B014461D46072900F2B480072A00F253
:10331000B48001EB81024BF2CC13C0F6050303EB42
:103320008202137C002B40F0AB8004EB84024BF252
:10333000CC13C0F6050303EB8202137C012B40F093
:10334000A2804BF2CC13C0F6050301EB810653F8C3
:10335000262004EB840653F826309A4240F09680EB
:1033600040F2EC27C2F200073870022A15D0032A77
:1033700025D0012A34D143F64000C4F20200066889
:1033800046F40012026040F2E823C2F2000345F264
:103390000047C4F200071F6022E043F64000C4F279
:1033A0000200066846F48002026040F2E823C2F29E
:1033B000000345F60007C4F200071F6010E043F663
:1033C0004000C4F20200066846F40002026040F2C7
:1033D000E823C2F2000345F60047C4F200071F606D
:1033E0004BF2CC18C0F6050801EB810108EB810215
:1033F000107991684FF0000700974FF00106019691
:10340000D36802934FF003023B46FDF7A1FC04EBA7
:10341000840408EB84042079A16800970196E2688F
:1034200002924FF003023346FDF792FC4FF0060084
:1034300005F0ECFCFFF768FBBDB140F2E420C2F2FE
:1034400000000A99016040F2E022C2F200020B9BE8
:10345000136040F2F020C2F200004BF26C21C0F683
:1034600005012A463B4607F0ADFAFFF79BFB4FF0FC
:1034700001000DE04FF000000AE04FF0000007E00F
:103480004FF0000004E04FF0000001E04FF00000BA
:1034900004B0BDE8F08100BF2DE9F04F83B00446D1
:1034A00000920D46002975D0FFF784FB4FF003080A
:1034B0004FF0000A40F2E829C2F2000940F2EC2382
:1034C000C2F20003019301E0002E4CD00098FFF7F8
:1034D000E1FB00284AD0009A02F0070715F0010F1F
:1034E0005ED14046FFF77EFB002842D05046FFF7F2
:1034F00079FB072F1AD8DDB13CB1D9F8003014F8A8
:10350000012B6FEA0200186104E0D9F800604FF067
:10351000FF01316107F10107BB4605F1FF36354672
:103520004046FFF75FFB002857D122E02E4600E01F
:103530002E46D9F800100B6843F400720A60009818
:1035400000F1080020F0070100914FF00500FFF79F
:1035500049FB88B1019B1A78032AB5D14FF01900B5
:1035600003F00AFDB0E74FF0010407E04FF000045C
:1035700004E04FF0000401E04FF0000440F2E820C6
:10358000C2F2000001680B6843F400720A60FFF7A2
:1035900009FB01E04FF00104204603B0BDE8F08FC5
:1035A0004046FFF71FFB0028E3D05046FFF71AFB09
:1035B000072FBBD82CB9D9F800004FF0FF010161EB
:1035C00006E0D9F8003014F8012B6FEA0200186108
:1035D00007F1010705F1FF3583E75046FFF702FBCE
:1035E000072FA3D82CB9D9F800504FF0FF0129615B
:1035F00006E0D9F8003014F8012B6FEA02001861D8
:1036000007F1010706F1FF356BE700BF30B583B066
:1036100015461C461A4601ABFFF7A0FA48B12846EA
:103620002146019AFFF738FF00280CBF1820002020
:1036300001E04FF01F0003B030BD00BF2DE9F041A5
:1036400005460E461446002A00F08380FFF7B2FAC2
:103650002846FFF71FFB002873D04FF00300FFF749
:10366000C1FA00286DD04FF00000FFF7BBFA40F21E
:10367000E823C2F200031868026842F48071016016
:103680004FF00100FFF7AEFA00285AD04FF00000CB
:10369000FFF7A8FA40F2E823C2F20003186814F119
:1036A000FF3118BF0121026861F38A2202604FF0E6
:1036B000A10303614FF00200FFF794FA002840D005
:1036C00040F2E820C2F2000001688A6912F0010F9E
:1036D00037D04B6913F4806F33D14FF004074FF0AC
:1036E000000540F2E828C2F200083846FFF77AFAEF
:1036F00038B32846FFF776FA04F1FF34012C2CD1B9
:10370000FCF744FDD8F800100A696FEA020306F8D6
:10371000013B0A686FF38A220A60FCF741FDE4E787
:103720002B681B6902E04FF00406114D3046FFF78D
:1037300059FA0028F4D10E4B1868016841F4007260
:103740000260FFF72FFAD4F1010038BF0020BDE876
:10375000F0814FF00100BDE8F081D8F80000016968
:103760006FEA010206F8012B002CBED1DBE700BF97
:10377000E802002030B583B015461C461A4601AB5E
:10378000FFF7ECF948B1019829462246FFF756FFAA
:1037900000280CBF1820002001E04FF01F0003B0EC
:1037A00030BD00BF08B543F23850C2F2000043F606
:1037B0003802C2F20002131A4FF0FF314FEAA3029F
:1037C000FCF79EFC43F63800C2F2000044F23801D8
:1037D000C2F200010A1A4FEAA2024FF0FF31A2F131
:1037E0002002FCF78DFC02F0ADFB40F20030C2F28B
:1037F000000044F20001C4F202014FF480524FF085
:10380000030313F069FCFDF749F84FF0000008BD11
:10381000BFF36F8F704700BF4BF20833C0F605034C
:10382000185C00EB40014BF28442C0F6050252F8EE
:1038300021305B68704700BF38B54BF20833C0F6E3
:1038400005031B5C03EBC30440F21832C2F2000212
:1038500002EB840282F8211014693CB140F2183561
:10386000C2F200051346D2699B69A04738BD00BF6C
:10387000F8B506460F464BF20833C0F605031D5C4B
:1038800005EBC50040F21834C2F2000404EB8004DA
:10389000D4F810C0BCF1000F07D0E2698A4204D00E
:1038A00030464FF00001A369E047E76163695BB10F
:1038B00005EBC50040F21832C2F2000202EB8002B2
:1038C000304639469269984794F8201079B12769B3
:1038D0006FB105EBC50540F21833C2F2000303EBEC
:1038E0008505304694F82110E269AB69B847F8BD08
:1038F0004BF20833C0F60503185C00EB40014BF2B5
:103900008442C0F6050252F82130D86840F08001A8
:10391000D9607047F8B5044600EB40024BF284438F
:10392000C0F6050353F8226035686FEA0500306081
:1039300005F0010215F0020F1CBF42F00202D2B2E4
:1039400015F0040F18BF42F0080215F0080F18BF59
:1039500042F0040215F4807F05D0316911F4804FE4
:1039600018BF42F0100215F0200F00D1E2B104EBB5
:10397000C40740F21833C2F2000303EB87008768E4
:103980008FB1716804EBC40040F21833C2F2000337
:1039900003EB80034BF2B830C0F60500005DC9B2FE
:1039A0009B69B84700E07368F26812F0800F1CD082
:1039B00015F0800F19D0F1686FF3C711F16004EBB7
:1039C000C40040F21833C2F2000353F8203063B150
:1039D00040F21832C2F2000202EB80024BF2B83021
:1039E000C0F60500005D9169984715F0400F17D0AB
:1039F00004EBC40140F21833C2F2000303EB81026E
:103A000053686BB1084640F21831C2F2000101EB75
:103A100080024BF2B830C0F60500005D916998470E
:103A2000F8BD00BF684620F007018D4601B54FF094
:103A30000600FFF76FFFBDE801408546704700BFF5
:103A4000684620F007018D4601B54FF00500FFF7ED
:103A500061FFBDE801408546704700BF684620F021
:103A600007018D4601B54FF00400FFF753FFBDE895
:103A700001408546704700BF684620F007018D462B
:103A800001B54FF00300FFF745FFBDE80140854653
:103A9000704700BF684620F007018D4601B54FF022
:103AA0000200FFF737FFBDE801408546704700BFC1
:103AB000684620F007018D4601B54FF00100FFF781
:103AC00029FFBDE801408546704700BF10B582B0B0
:103AD0008DF807104BF20833C0F60503185C00EBB5
:103AE00040024BF28441C0F6050151F822402368A0
:103AF00013F0800FFBD002A911F8012D626000EBDA
:103B0000C00040F21834C2F2000404EB8004608C60
:103B10004FF0010205F092F9608404F1200402B034
:103B200010BD00BF70B582B08DF807104BF208339E
:103B3000C0F60503185C00EB40014BF28442C0F66E
:103B4000050252F82140256815F0800F1DBF9DF831
:103B5000075065600126002600EBC00340F21830D4
:103B6000C2F2000000EB8305688C0DF107014FF0F5
:103B7000010205F063F9688405F12005E16841F070
:103B80008002E260304602B070BD00BF2DE9F04710
:103B900007468A4691461D469DF820804BF2083321
:103BA000C0F605031C5C04EB44024BF28440C0F6F3
:103BB000050050F82260082D06D0072D02D1B9F17A
:103BC000000F01D1FCF78CFA08F1FF31CBB2012BC9
:103BD00001D9FCF785FA4BF26842C0F6050252F8AB
:103BE0002400B0FBFAF1B1F5803F39D29DF82420D2
:103BF000012A14BF00220122B1604FF0000362F3DA
:103C00008613B8F1010F04D0002A0CBF0220002057
:103C100001E04FF0000060F30D3362F38E33336147
:103C20004FF06C01B9F1020F14BF0022012262F3C0
:103C3000492119F1000918BF4FF0010969F38A21E0
:103C4000082D18BF4FF0000969F30C3141F4005200
:103C5000F2603846FFF7E0FD4FF00100BDE8F08765
:103C60004FF00000BDE8F087F0B585B00D461E4668
:103C70004BF20833C0F60503195C01EB41044BF22B
:103C80008447C0F6050757F824704BF26443C0F62A
:103C90000503185C00EB40014BF21C44C0F6050420
:103CA00004EBC1040AB1FCF71BFA75B9207B21694A
:103CB0009DF82C2000924FF001030193626902925B
:103CC0004FF003023346FDF743F8207861689DF812
:103CD000283000934FF001020192A36802934FF045
:103CE00003023346FDF734F84BF2D840C0F6050026
:103CF0000168012D14BF0025012565F3C301796119
:103D000005B0F0BD2DE9F04385B004464BF2083311
:103D1000C0F60503185C00EBC00240F21835C2F291
:103D2000000505EB82054BF28441C0F6050100EB6E
:103D300040064FEA860701EB070851F80790FCF7A9
:103D400025FA064695F82030BBB14FF00007C9F8B8
:103D50000C703846394698F90420FCF789FA204659
:103D60003946FFF769FDEB681BB12046E969AA698E
:103D700098474FF0000085F820004BF2C035C0F6A0
:103D8000050504EB84016A1815F801809578D77849
:103D900092F804904BF26443C0F605031C5D04EBFB
:103DA00044004BF2D431C0F6050101EBC004527857
:103DB0000AB1FCF795F9B8F1000F0CD1207B21690D
:103DC000CDF800904FF0010301934FF000020292F2
:103DD0002B46FCF7BDFF2078616800974FF0010289
:103DE00001924FF0000302932B46FCF7B1FF3046DF
:103DF000FCF7D6F905B0BDE8F08300BF2DE9F04F20
:103E000085B005468B46924699464BF20833C0F67C
:103E100005031E5C40F21838C2F2000806EBC60724
:103E20004FEA870708EB070406EB46004BF2844194
:103E3000C0F6050101EB8006FCF7A8F9039043F6F4
:103E40004003C4F2020318684BF2DC41C0F60501DE
:103E50000A6820EA020E4BF22032C0F60502106812
:103E60004EEA0000186043F64403C4F202031868E7
:103E7000496820EA01005268104318604BF20C3187
:103E8000C0F6050105EB8503C818C95C4278837844
:103E900090F803C0CDF800C0007901902846FFF7E4
:103EA000E3FE9DF8382000929DF83C1001912846D1
:103EB000594652464B46FFF769FE0546109B48F8A7
:103EC00007301298A060119A62601399E160149B08
:103ED000A361B0684FF00F0196F90420FCF7C8F910
:103EE0004FF0010084F820000398FCF759F92846A8
:103EF00005B0BDE8F08F00BF4BF20833C0F60503F4
:103F0000185C00EBC00340F21830C2F2000000EB76
:103F1000830319615A6170474BF26443C0F605038D
:103F2000185C00EB40014BF22832C0F6050202EBB0
:103F300001107047FA2884BF0530C0B2032812D898
:103F40004BF20833C0F60503185C00EBC00140F2E9
:103F50001832C2F2000202EB81034FF6FF70588460
:103F60004FF0010070474FF000007047FA2884BFFF
:103F70000530C0B203280ED84BF20833C0F6050353
:103F8000185C00EBC00140F21832C2F2000202EBF2
:103F90008103588C70474FF000007047082806D9FD
:103FA000102807D920288CBF4020202070474FF0D0
:103FB000080070474FF01000704700BF022809D07A
:103FC000032804D0012814BF0020012070474FF0BF
:103FD000030070474FF00200704700BF40F6001327
:103FE000C5F20003186840F60802C5F20002116825
:103FF000C1F34103022B12BF6FF30200032363F3EB
:10400000020040F400406FF3995040F60012C5F2F0
:104010000002106040F60401C5F200010B6843F491
:1040200080700860704700BF4BF27853C0F60503FC
:104030001A6840F61030C5F200000260704700BFF9
:1040400010B440F6A463C2F200031A5CE0B14FF072
:10405000000340F6A031C2F200014FF04C0404FB13
:104060000212D16821F0030202F1040262F312038A
:104070004FF0010161F3DC434BF2EC42C0F6050264
:1040800002EB401081690B6010BC704770B440F2C5
:104090002003C5F200031868C0F34342022A01D08E
:1040A000062A29D100F00F014BF29055C0F6050504
:1040B00055F82160C0F30A1505F1030398081BD0D9
:1040C00041F20001C5F2000100F1FF3404F00104E7
:1040D0000A68334672604FF0010282420ED10AE054
:1040E0000C6803F1040343F8044F0C685C6002F1B0
:1040F00002028242F4D1356070BC7047002CEFD0D0
:104100000C6803F104035C6002F101028242E7D112
:10411000F1E700BF70B44BF27C53C0F6050353F8CF
:1041200020603268002A3CD04BF2EC41C0F6050119
:1041300001EB401102F103024FEA9202CB691B68C6
:104140009A420CD940F63402C5F2000211684FF0D1
:10415000010303FA00F008431060184623E006F15B
:104160000403C2B102F1FF3000F00105086953F801
:10417000044B0460501E18D10DE00C691A4652F829
:10418000045B256000F1FF300C695B68236002F17D
:1041900004030138F1D14FF0000131604FF001000C
:1041A00001E04FF0000070BC7047002DE5D00A69B7
:1041B00053F8044B14600138DFD1ECE708B54FF039
:1041C000010303FA00F040F21642C2F20002138823
:1041D000184210D023EA000340F21640C2F2000059
:1041E0000380CA6B52B1086A4FF0000104F060F816
:1041F0004FF0000008BD4FF0000008BD4FF0010077
:1042000008BD00BF70B540F21403C5F200031C687E
:104210004BF26C50C0F6050001680C4200F0BB8107
:1042200040F69962C2F200021378012B40F2B3818A
:1042300040F21800C5F2000001684BF2E442C0F6FB
:1042400005021368194200F0A68140F61800C5F275
:104250000000016811F0010F56D040F60815C5F2B4
:1042600000052A6840F60830C5F2000003682A609D
:10427000036040F6A461C2F20001087840F6A03164
:10428000C2F200014FF04C0505FB001503F00100E0
:10429000E96A0143E962C3F3C000296B0143296362
:1042A00003F00803D8B258BBD2B212F0010F0ED0FF
:1042B0001DE0EA6A22B105F1100000F0B5FF2BE025
:1042C0002B6B002BF7D1686B0028F4D124E012F09F
:1042D000900FEED040F63403C5F20003186820F0CA
:1042E000010119604FF00000FFF714FFE1E76E6B6A
:1042F0004FF000002946FFF761FF30436863D8E7BD
:104300004FF00001E963CFE740F61802C5F2000262
:10431000136813F4803FA0D140F61801C5F20001E4
:104320000A6802F0020398B2002856D040F6281519
:10433000C5F200052A6840F62830C5F2000003687F
:104340002A60036040F6A461C2F20001487840F69A
:10435000A031C2F200014FF04C0505FB001503F03F
:104360000100E96A0143E962C3F3C000296B01431C
:10437000296303F00803D8B258BBD2B212F0010F80
:104380000ED01DE0EA6A22B105F1100000F04CFFEA
:104390002FE02B6B002BF7D1686B0028F4D128E0BD
:1043A00012F0900FEED040F63403C5F20003186807
:1043B00020F0020119604FF00100FFF7ABFEE1E7CA
:1043C0006E6B4FF001002946FFF7F8FE304368633B
:1043D000D8E74FF00001E963CFE740F61801C5F2D6
:1043E00000010A684FEA124303F0020081B200297B
:1043F0009CD140F61801C5F200010A6802F00403DE
:1044000098B2002856D040F64815C5F200052A6833
:1044100040F64830C5F2000003682A60036040F6A9
:10442000A461C2F20001887840F6A031C2F2000116
:104430004FF04C0505FB001503F00100E96A01434C
:10444000E962C3F3C000296B0143296303F0080349
:10445000D8B258BBD2B212F0010F0ED01DE0EA6AFA
:1044600022B105F1100000F0DFFE2FE02B6B002BD6
:10447000F7D1686B0028F4D128E012F0900FEED04D
:1044800040F63403C5F20003186820F004011960F7
:104490004FF00200FFF73EFEE1E76E6B4FF00200C7
:1044A0002946FFF78BFE30436863D8E74FF00001E1
:1044B000E963CFE740F61801C5F200010A684FEA48
:1044C000124303F0040081B200299CD140F6180188
:1044D000C5F200010A6802F0080398B258B940F624
:1044E0001801C5F200010A684FEA124303F0080000
:1044F00081B200294FD040F66815C5F200052A6840
:1045000040F66830C5F2000003682A60036040F698
:10451000A461C2F20001C87840F6A031C2F20001E5
:104520004FF04C0505FB001503F00100E96A01435B
:10453000E962C3F3C000296B0143296303F0080358
:10454000D8B210B14FF00001E963D2B212F0010FFE
:1045500008D06E6B4FF003002946FFF72FFE304363
:1045600068630EE012F0900F0BD040F63403C5F2F2
:104570000003186820F0080119604FF00300FFF7EE
:10458000C9FDEA6A1AB92B6B0BB9686B18B105F152
:10459000100000F049FE14F0100F01D0FFF776FD77
:1045A00014F4805F0DD040F67561C2F200014FF047
:1045B00001020A7040F66C63C2F20003186802F050
:1045C00045FB14F4005F01D0FFF708FD14F4006F01
:1045D00014D040F60060C2F200004FF001010170FB
:1045E00040F69863C2F200034FF000021A7040F6E2
:1045F0006C60C2F20000006802F028FB002C14DAA4
:1046000040F60061C2F200014FF000030B7040F66B
:104610009860C2F200004FF00102027040F66C6137
:10462000C2F20001086802F011FB40F21403C5F267
:1046300000031C6070BD00BF684620F007018D4676
:1046400089B500AFFFF7DEFDBD46BDE88940854670
:10465000704700BF2DE9F04140F6A036C2F20006D7
:104660004FF04C0303FB0066304650F8205F4BF2DE
:10467000EC48C0F605084FEA451708EB07044FF071
:1046800000014FF01C0213F0B3FF35624FF0010040
:10469000B06258F807204FF00003136061690B60A7
:1046A000A0684FF0FF02026061680B60A0690360C0
:1046B000E1680A604BF29052C0F6050252F82500FC
:1046C00003604BF27C51C0F6050151F825201360C0
:1046D000BDE8F08100B583B04FF00003019340F2D4
:1046E0001001C5F200010A68B0F1FF3F08BF1020B9
:1046F00060F3891242F0200040F21003C5F200037B
:104700001860194640F63F52C0F20302019800F1CA
:10471000010001900B6813F0200F02D00198904225
:10472000F4D94FF0030004F071FB03B000BD00BFEB
:104730002DE9F8434FF04C0303FB00F040F6A031A5
:10474000C2F200014418256A4FF0010606FA05F688
:104750004BF2EC42C0F6050202EB45174058002828
:1047600067D0A368FBB1D7F80080D8F8001011F427
:10477000004F18D1D8F80020914663F30A09007A57
:10478000FFF71CFC60F3934949F4004965F399591C
:1047900049F08050C0F3404363F39A60C8F80000CA
:1047A0002846FFF797FFE168F1B17A68106810F4C6
:1047B000004F19D12846FFF743FCD7F80480D8F8FA
:1047C0000070E36863F30A072168087AFFF7F6FBD5
:1047D00060F3934747F4004242F01047C7F340406C
:1047E00060F39A67C8F800704BF29053C0F6050367
:1047F00053F825104FF000020A60A06858B140F647
:104800001C03C5F20003196846EA010290B2196858
:1048100060F30F011960E3685BB140F61C00C5F25C
:104820000000026846EA1246B6B2016866F31F410C
:104830000160BDE8F88300BF70B582B04FF00002A0
:10484000019240F21003C5F20003196841F0010023
:10485000186001921A6812F0010F19D0019940F600
:104860003F53C0F20303994212D840F21000C5F240
:10487000000040F63F52C0F20302019901F101012C
:104880000191036813F0010F02D001999142F4D90C
:104890004FF0030004F0BAFA4FF00000019040F22C
:1048A0001002C5F200021368002B1DDB019940F6CF
:1048B0003F50C0F20300814216D84FF0030640F289
:1048C0001005C5F2000540F63F54C0F2030430461F
:1048D00004F09CFA019A02F1010201922B68002B6C
:1048E00002DB0199A142F2D902B070BD00B583B0DC
:1048F0004FF00003019340F21000C5F2000002687F
:1049000042F01001016040F63F52C0F20302019BE9
:1049100003F101030193016811F0100F02D0019B14
:104920009342F4D94FF0030004F070FA03B000BDD5
:1049300050B14BF27051C0F605010A6840F21803FD
:10494000C5F200031A6070474BF27453C0F60503BA
:104950001A6840F21800C5F200000260704700BFFC
:1049600038B54FF0000440F60063C5F200031C6048
:1049700040F60002C5F20002106840F0030164F343
:10498000820164F30A11116040F22405C5F20005AA
:104990002B684FF0400262F30F032B60204662F356
:1049A0001F40214662F31F4162F30F0140F22805C8
:1049B000C5F2000529604FF0800363F30F0040F259
:1049C0000412C5F2000210604FF0C00161F30F0045
:1049D00040F20815C5F2000528604FF4807363F3B8
:1049E0000F0040F20C12C5F2000210604FF0FF30D1
:1049F000FFF770FEFFF77AFF40F61000C5F20000E7
:104A0000046040F61401C5F200010C604FF0FF3560
:104A100040F61803C5F200031D6040F61C02C5F203
:104A2000000214602046FFF715FE4FF00100FFF76B
:104A300011FE4FF00200FFF70DFE4FF00300FFF7ED
:104A400009FE4FF00400FFF705FE4FF00500FFF7E9
:104A500001FE4FF00600FFF7FDFD4FF00700FFF7E6
:104A6000F9FD40F21800C5F20000046040F21401A4
:104A7000C5F200010D604FF00100FFF759FF38BD8E
:104A800040F21643C2F2000319884FF0010202FA05
:104A900000F0084000280CBF02200320704700BF30
:104AA00040F60013C5F200031B68C3F3076202F06F
:104AB0008000C1B209B143F0804343F4001040F6D6
:104AC0000012C5F200021060704700BF2DE9F843E4
:104AD000054616464BF2EC48C0F6050808EB4018B0
:104AE0004BF27C53C0F6050353F820704FF00109D8
:104AF00009FA00F90C46A9B9386840B940F21643E2
:104B0000C2F20003188819EA000F5AD10AE040F2F5
:104B10001641C2F200010A8819EA020F02D02846A3
:104B2000FFF7D8FD06F1030107F1040388081CD044
:104B300000F1FF3202F0010CA4F1040151F8042F3E
:104B400043F8042B01383ED10FE001F1040249681B
:104B50001C4644F8041B00F1FF3002F104015268C6
:104B60005A6004F104030138EFD13E6040F216436D
:104B7000C2F20003198849EA0109A3F8009065B957
:104B800040F61010C5F2000002684FF0010161F319
:104B9000D44266F30602026009E0D8F81400026805
:104BA0004FF0010363F3DC4266F312020260D8F8AF
:104BB0000030186840F004421A6016B12846FFF72A
:104BC000A9FABDE8F883BCF1000FBED051F8042F5C
:104BD00043F8042B0138B8D1C7E700BF70B50446CD
:104BE0004BF29053C0F6050353F82060334653F858
:104BF000045BAA4238BF1546084619462A4613F0F8
:104C0000D3FC4FF0000030602046FFF719FA4BF25A
:104C1000EC41C0F6050101EB441463681A6842F0E8
:104C200004401860284670BDF8B5054640F6A0332C
:104C3000C2F200031868002871D040F6A031C2F219
:104C40000001CA6C002A71D040F6A034C2F2000400
:104C5000D4F89860002E6DD040F6A037C2F200075D
:104C6000D7F8E430002B69D040F6A030C2F2000043
:104C7000D0F83011002965D040F6A032C2F200020F
:104C8000D2F87C41002C61D040F6A036C2F200067A
:104C9000D6F8C871002F5DD040F6A033C2F20003F1
:104CA000D3F81402002859D040F6A031C2F2000116
:104CB000D1F86022002A55D0464E4FF00807FBF786
:104CC0000FFA2C7A002C53D040F21442C2F20002A8
:104CD0001088014610F0020F55D04FF0010404F186
:104CE000010441FA04F212F0010FF8D14FF0010172
:104CF00001FA04F1084340F21443C2F200031880A1
:104D000044B96889FFF74AF9B060A889FFF746F906
:104D1000F06042E06A89B260A989F1603DE040F646
:104D2000A036C2F200064FF000071EE02A4E4FF0F8
:104D300001071AE0294E4FF0020716E0284E4FF007
:104D4000030712E0274E4FF004070EE0264E4FF007
:104D500005070AE0254E4FF0060706E0244E4FF007
:104D6000070702E01B4E4FF00807072FA9D9A6E757
:104D700040F21443C2F20003188840F00101198088
:104D80004FF00004BDE740F0020440F21443C2F2C9
:104D900000031C804FF00104BCE740F6A460C2F29F
:104DA00000000755374647F8205B38464FF00001B2
:104DB0004FF01C0213F01CFC34626B68B36306F105
:104DC00010004FF006012A683B4600F00DFA20461D
:104DD000F8BD00BF000E0020EC0B0020380C0020B6
:104DE000840C0020D00C00201C0D0020680D002039
:104DF000B40D0020022907D140F60003C5F20003DC
:104E00001A6860F30A121A60704700BF10B54FF0BD
:104E1000000440F63403C5F200031C6040F60400B1
:104E2000C5F20000026842F0010101602046FFF770
:104E300011FC4FF00100FFF70DFC4FF00200FFF7EF
:104E400009FC4FF00300FFF705FC4FF00400FFF7EB
:104E500001FC4FF00500FFF7FDFB4FF00600FFF7E8
:104E6000F9FB4FF00700FFF7F5FB4FF0FF30FFF7BE
:104E700031FC40F21643C2F200031C8040F61800D9
:104E8000C5F200004FF0FF3202604BF28C51C0F6C9
:104E90000501086840F61C03C5F2000318604BF2D8
:104EA000E842C0F60502116840F61400C5F20000A1
:104EB00001604BF2A053C0F605031A6840F61001DA
:104EC000C5F200010A6020464FF00201FFF792FF91
:104ED000FFF7AAF82046FFF72BFC4FF00100FFF781
:104EE00027FC4FF00200FFF723FC4FF00300FFF711
:104EF0001FFC4FF00400FFF71BFC4FF00500FFF70D
:104F000017FC4FF00600FFF713FC4FF00700FFF708
:104F10000FFC10BD08B5FFF779FF08BD704700BF53
:104F2000F0B585B0054641F28830FCF7C5FC002D90
:104F300062D043F63401C4F202010C6844F08006EA
:104F40000E604FF0000400944FF0030601964FF0FE
:104F50000A07029720464FF00B0132462346FBF723
:104F6000F7FE00940196029720464FF00C0132465E
:104F70002346FBF7EDFE40F20C06C5F2000633684F
:104F800043F040023260FFF757FC40F23800C5F2B0
:104F900000004FF40411016044F6206003F036FF76
:104FA000FCF782FC336843F0400064F3082064F3AC
:104FB00049204FF0050262F38D2064F35D7040F0EC
:104FC0008041316044F6206003F020FFFCF76CFC68
:104FD000FFF7C6FC40F20803C5F2000340F281105F
:104FE000186044F23960C0F604004FF00F014FF032
:104FF0004302FBF73DF913E04FF000004FF00F01C3
:105000004FF04302FBF734F94FF0000340F238024F
:10501000C5F20002136040F21800C5F20000036000
:105020002846FFF77BFF4FF06400FCF745FC05B016
:10503000F0BD00BF10B543F61404C4F202042368A7
:1050400043F0400020604FF0010003F0DFFE2168D4
:105050006FF3861121604FF0010003F0D7FE40F698
:105060000003C5F206031A6842F00400186010BD80
:1050700008B543F63403C4F202031A6842F0400054
:105080001860FFF7D7FF08BD08B540F60403C5F266
:105090000603186810F0660F05D0FFF7CBFF4FF03E
:1050A000640003F0B3FE08BD08B5FFF7EDFF40F65E
:1050B0000803C5F20603186808BD00BF08B5FFF76E
:1050C000E3FF40F60403C5F20603186800F0010090
:1050D00008BD00BF2DE9F04182B04BF2A457C0F6E5
:1050E000050745F2B516C0F6040640F28C15C2F26B
:1050F00000054FF00408CDF8008038464FF08001DD
:1051000032462B4601F0EEFE40F21844C2F2000493
:105110002060CDF8008038464FF08101324605EB23
:10512000080301F0DFFE6060CDF8008038464FF0E4
:105130008201324605F1080301F0D4FEA060CDF8EB
:10514000008038464FF08301324605F10C0301F030
:10515000C9FEE060CDF8008038464FF08401324649
:1051600005F1100301F0BEFE2061CDF80080384645
:105170004FF08501324605F1140301F0B3FE606182
:10518000CDF8008038464FF08601324605F118030D
:1051900001F0A8FEA061CDF8008038464FF08701ED
:1051A000324605F11C0301F09DFEE06102B0BDE84E
:1051B000F08100BF08B505464FF000060BE0FAF796
:1051C000E5FF2C68616829606660FAF7E9FF2268EC
:1051D0000AB1A06890472B6803F1FF3010F1030F6C
:1051E000EDD901F001FDF6E70260B3F1FF3F18BF12
:1051F0008360FF290ED143F23453C2F200031A68D0
:1052000022B192F829304FEA530101E04FF0070133
:105210000173704701F07F010173704710B14FF0C7
:1052200000020260704700BF38B50446FAF7AEFFCF
:105230000546BCB16368C3B9227B40F28C10C2F250
:10524000000050F82210616040F82240247B40F2B8
:105250001843C2F2000353F8240001F0F7FC4FF0AA
:10526000010404E04FF0000401E04FF00004284680
:10527000FAF796FF204638BD10B5044640F260604C
:10528000C2F200004FF000014FF0240213F0B0F919
:10529000D4B140F28040C2F200004FF000014FF064
:1052A000480213F0A5F940F22C50C2F200004FF072
:1052B00000014FF0240213F09BF940F22453C2F294
:1052C00000034FF002021A7010BD00BF38B54BF258
:1052D000F853C0F6050353F8205040F2CC41C2F217
:1052E000000151F820404BF25862C0F60502105CF4
:1052F000FBF716FE2840A04214BF0020012038BD55
:105300004BF25863C0F605031A5C40F22C51C2F20E
:10531000000151F822204BF2F853C0F6050353F870
:10532000200002420CBF00200120704770B440F6FC
:10533000E003C2F2000353E8002F02F1010243E848
:1053400000210129F7D04BF25862C0F60502155C26
:1053500040F26061C2F2000151F825404BF2F8566C
:10536000C0F6050656F8202024EA020041F8250080
:1053700053E8005FA5F1010543E80056012EF7D080
:1053800053E8005FB5F1004F0DD14FF0000543E841
:105390000056012EF4D04EF60450CEF20000016803
:1053A00041F080510160BFF32F8F14420CBF0020E9
:1053B000012070BC704700BF4BF27063C0F605035C
:1053C000185C704710B50446FBF7AAFD40F2AC1319
:1053D000C2F2000353F82410484010BD10B5044633
:1053E0004FF00100FFF748FF40F2C843C2F200034C
:1053F0001C704BF2B050C0F6050050F8342040F25B
:105400002851C2F200010A6000EBC404606840F257
:105410005453C2F20003186010BD00BF00B585B040
:105420004FF00000FFF7DAFF4FF00003009340F267
:105430005852C2F2000201924FF0400002904BF22B
:105440004C60C0F605004FF0020145F2F142C0F693
:10545000040201F033FC40F25C63C2F20003186006
:1054600005B000BD2DE9F001804600283CD04FF08A
:1054700000034FEA8302086850F823404D6855F84E
:10548000236086EA0407886850F8235084EA050CF4
:105490004CEA07076FEA070CC86850F8235026EA61
:1054A000050707EA0C0705EA0C0C66EA0C0635400E
:1054B00040F82350CD6855F82300384345F82300C1
:1054C0000D6955F82300384345F823004D690DB1A7
:1054D00045F8237048688558886885504868845026
:1054E00003F101034345C4D1BDE8F001704700BF9B
:1054F0002DE9F84340F22858C2F2000840F2505615
:10550000C2F2000640F23844C2F200044FF0000537
:1055100040F25457C2F20007D8F8000000EB8000B8
:1055200001F02AFD3368002B40F0F5812046294622
:105530004FF0240213F05CF8EDE14FF009004BF25C
:10554000E051C0F60501FFF78DFF40F22453C2F28F
:105550000003197859B101F1FF3040F22452C2F230
:105560000002107040F26063C2F200031D6040F25E
:105570002051C2F200010868E8B940F22052C2F29C
:105580000002156040F25863C2F20003197849B96D
:1055900040F22051C2F20001086860B1284606F0CE
:1055A000CFF808E040F22050C2F20000026842F05A
:1055B00000630360ECE740F22452C2F20002137869
:1055C0005BB103F1FF3140F22450C2F200000170E0
:1055D00040F26062C2F20002556040F22053C2F213
:1055E00000031968E9B940F22050C2F200000560DA
:1055F00040F25862C2F2000213784BB940F22053D5
:10560000C2F20003196861B1284606F099F808E073
:1056100040F22051C2F20001086840F000620A60C6
:10562000ECE740F22450C2F2000002785AB102F1D5
:10563000FF3340F22451C2F200010B7040F260606F
:10564000C2F20000856040F22052C2F200021368EC
:10565000EBB940F22051C2F200010D6040F25860F7
:10566000C2F2000002784AB940F22052C2F20002AF
:10567000136863B1284606F063F808E040F220534F
:10568000C2F20003196841F000601860ECE740F2D4
:105690002451C2F20001087858B100F1FF3340F202
:1056A0002452C2F20002137040F26061C2F20001A3
:1056B000CD6040F22050C2F200000368EBB940F226
:1056C0002052C2F20002156040F25861C2F200019D
:1056D000087848B940F22050C2F20000036863B174
:1056E000284606F02DF808E040F22053C2F20003ED
:1056F0001A6842F000611960ECE740F22452C2F2ED
:105700000002117859B101F1FF3040F22453C2F286
:105710000003187040F26062C2F20002156140F2AC
:105720002051C2F200010868E8B940F22053C2F2E9
:1057300000031D6040F25862C2F20002117849B9BC
:1057400040F22051C2F20001086860B1284605F01D
:10575000F7FF08E040F22050C2F20000036843F077
:1057600000620260ECE740F22453C2F200031A78B0
:105770005AB102F1FF3140F22450C2F20000017030
:1057800040F26063C2F200035D6140F22052C2F257
:1057900000021168E9B940F22050C2F20000056031
:1057A00040F25863C2F200031A784AB940F220521C
:1057B000C2F20002116861B1284605F0C1FF08E09D
:1057C00040F22051C2F20001086840F000630B6013
:1057D000ECE740F22450C2F2000003785BB103F121
:1057E000FF3140F22452C2F20002117040F26060B8
:1057F000C2F20000856140F22053C2F20003196832
:10580000E9B940F22052C2F20002156040F258603D
:10581000C2F2000003784BB940F22053C2F20003F9
:10582000196861B1284605F08BFF08E040F220516D
:10583000C2F200010A6842F000600860ECE740F242
:105840002452C2F20002107858B100F1FF3340F246
:105850002451C2F200010B7040F26062C2F20002F9
:10586000D56140F22050C2F200000368EBB940F26B
:105870002051C2F200010D6040F25862C2F20002F3
:10588000107848B940F22050C2F20000036863B1BA
:10589000284605F055FF08E040F22053C2F200030D
:1058A000196841F000621A60ECE740F22451C2F23C
:1058B00000010A785AB102F1FF3040F22453C2F2DB
:1058C0000003187040F26061C2F200010D6240F204
:1058D0002052C2F200021068D8B940F22053C2F23E
:1058E00000031D6040F25861C2F200010A783AB12B
:1058F00040F22050C2F20000036843F000610160F2
:1059000040F22052C2F20002106810B1284605F0A1
:1059100017FF356000E6D4F800902846FFF752FDE7
:1059200040EA09012160D4F804904FF00100FFF72C
:1059300049FD40EA09026260D4F808904FF0020085
:10594000FFF740FD40EA0900A060D4F80C904FF04A
:105950000300FFF737FD40EA0903E360D4F8109035
:105960004FF00400FFF72EFD40EA09012161D4F851
:1059700014904FF00500FFF725FD40EA090262612F
:10598000D4F818904FF00600FFF71CFD40EA09001C
:10599000A061D4F81C904FF00700FFF713FD40EA18
:1059A0000903E361D4F820904FF00800FFF70AFDE7
:1059B00040EA09012162306800F1010030603A6874
:1059C0009042FFF4A9ADB8E500B585B04FF00003F3
:1059D000009340F2D462C2F2000201924FF0400004
:1059E00002904BF28870C0F605004FF0060145F6B4
:1059F0000922C0F6040201F061F940F28463C2F2A8
:105A00000003186005B000BD2DE9F04F85B040F6E9
:105A100044031E46C2F2000640F2FC700746C2F282
:105A2000000740F2B061C2F20001019101F0DCF820
:105A30003268002AFAD061E1E359002B53D028469E
:105A4000FFF7C0FC01996258605090434BD0E35976
:105A500010EA030247D0039991F800E04BF29079E5
:105A6000C0F605094FEA451840F28861C2F200010C
:105A70004FF6FF7C4BF2886AC0F6050A40F2D87BED
:105A8000C2F2000B00957046C2F10003134022EAF7
:105A9000030218B954F80B502B4221D15FEA136E60
:105AA00004D01AF80E3003F118030EE01D0C04D0D8
:105AB0001AF8053003F1100307E05FEA132E1ABF4E
:105AC0001AF80E3008331AF80330434419F803501B
:105AD00031F815E0E6451CBF0EF1010E21F815E086
:105AE000002AD1D1009D05F1010504F10404092D1E
:105AF000A2D1029C621E029240F0F78003990878BE
:105B000000F10100C3B20B700B2B03D14FF0000466
:105B10000C7002E0002B40F0E58040F62002C2F25B
:105B20000002116891B16FEA01003B6803403B60DD
:105B300040F2D875C2F200052C682040286040F67B
:105B40002001C2F200014FF000020A6040F620007E
:105B5000C2F20000436893B16FEA03057C682C40F1
:105B60007C6040F2D872C2F2000251680D4055606C
:105B700040F62000C2F200004FF00003436040F600
:105B80002005C2F20005AC6894B16FEA0400BA685F
:105B90000240BA6040F2D873C2F20003996808402C
:105BA000986040F62005C2F200054FF00004AC609A
:105BB00040F62000C2F20000C26892B16FEA020310
:105BC000F9681940F96040F2D875C2F20005EC6836
:105BD0002340EB6040F62000C2F200004FF00002CC
:105BE000C26040F62003C2F20003196991B16FEA66
:105BF00001053C692C403C6140F2D870C2F20000C3
:105C000002691540056140F62003C2F200034FF01F
:105C10000001196140F62005C2F200056C6994B1DB
:105C20006FEA04007A6902407A6140F2D873C2F2E6
:105C3000000359690840586140F62005C2F200058A
:105C40004FF000046C6140F62000C2F2000082694F
:105C500092B16FEA0203B9691940B96140F2D8758F
:105C6000C2F20005AC692340AB6140F62000C2F2ED
:105C700000004FF00002826140F62003C2F20003F0
:105C8000D96991B16FEA0105FC692C40FC6140F2D1
:105C9000D870C2F20000C2691540C56140F6200309
:105CA000C2F200034FF00001D96140F62005C2F2B4
:105CB00000052C6A94B16FEA04003A6A02403A6225
:105CC00040F2D873C2F20003196A0840186240F625
:105CD0002005C2F200054FF000042C624FF4FA7068
:105CE000029002E04FF4FA7502954FF0010001F0C6
:105CF00043F93268002A3FF499AE07E04FF4FA7591
:105D0000029540F2D474C2F2000403944FF00004F0
:105D1000254691E610B54FF0000440F64403C2F268
:105D200000031C6040F2D870C2F2000021464FF020
:105D30000902FAF7E5F940F2FC70C2F200002146D0
:105D40004FF00902FAF7DCF940F62000C2F2000039
:105D500021464FF00902FAF7D3F940F2B060C2F2DF
:105D6000000021464FF00902FAF7CAF940F28860B4
:105D7000C2F2000021464FF0280212F039FC40F236
:105D8000D470C2F20000047010BD00BF70B54BF2B9
:105D90005863C0F605031B5C4BF2F852C0F60502CF
:105DA00052F8202040F64400C2F20000046840F29D
:105DB000FC75C2F2000555F82300104206D104F12B
:105DC000010640F64405C2F200052E6049B140F2DA
:105DD000D871C2F2000151F82350154341F8235005
:105DE00009E040F2D871C2F2000151F8235025EACF
:105DF000020541F82350104340F2FC71C2F2000149
:105E000041F8230040F62001C2F2000151F82300BE
:105E100020EA020241F8232034B940F28463C2F23E
:105E20000003186800F012FF70BD00BF30B44BF2E1
:105E30005863C0F605031B5C4BF2F852C0F605022E
:105E400052F8202040F2FC70C2F2000050F823000B
:105E5000104229D040F64404C2F20004256805F13E
:105E60000105256071B140F62001C2F2000151F830
:105E70002340144341F8234040F2D471C2F20001A0
:105E8000097889B96FEA020240F2D871C2F20001C2
:105E900051F82340144041F82340024040F2FC7086
:105EA000C2F2000040F8232030BC704730B40346F3
:105EB00040F6E002C2F2000252E8000F00F10100D9
:105EC00042E80004012CF7D040F28860C2F20000E2
:105ED00030F8132039B140F28861C2F200014FF06E
:105EE000000421F8134040F6E003C2F2000353E837
:105EF000004FA4F1010443E80045012DF7D053E819
:105F0000004FB4F1004F0DD14FF0000443E80045BD
:105F1000012DF4D04EF60450CEF20000016841F09D
:105F200080510160BFF32F8F104630BC704700BF17
:105F300040F2D473C2F200031878D0F1010038BFE8
:105F4000002070472DE9F84FDFF834814B4FC8EB44
:105F500007004FEAD00707F101074FF0000540F2B4
:105F6000982AC0F6000A40F27039C0F6000931E004
:105F700044464FF000066FEA060B0BEB070101F0F9
:105F8000010B58F8043CAB4229D135E054F8043CED
:105F9000AB4205D154F8080C8047FBF785FC0BE0B9
:105FA000FF2B09D9FF2D07D154F8040C4FF007013E
:105FB00054F8082C00F0A2FF06F1010604F10804D1
:105FC00054F8041CA94240D14CE005F10105B5F597
:105FD000807F02D0CA45CBD3F7E7BDE8F88FFF2B0F
:105FE0000FD9FF2D0DD158F8040C4FF0070158F8C8
:105FF000082C00F083FF04E058F8082C9047FBF7CA
:1060000053FC06F1010604F10804BE42DDD0BBF1E9
:10601000000FBBD054F8040CA8420AD0FF280DD9B9
:10602000FF2D0BD14FF0070154F8082C00F066FF4C
:1060300004E054F8081C8847FBF736FC06F101061B
:1060400004F10804BE42A1D1BFE7FF290FD9FF2DFB
:106050000DD154F8040C4FF0070154F8082C00F04F
:106060004DFF04E054F8082C9047FBF71DFC06F1A7
:10607000010604F10804BE4288D1A6E777030008B0
:10608000A0020008027840F6AD03C2F200031B78BC
:106090009A4206D34FF000020270087800F1010026
:1060A00008700A7840F6AE03C2F200031878824204
:1060B00024BF00200870704710B5A0F10803052B1D
:1060C0003DD8DFE803F01F3C2C3C038A40F64C002F
:1060D000C2F200004FF020014FF0540212F088FA93
:1060E00040F6A000C2F200004FF0FF314FF00C026A
:1060F00012F07EFA40F6B400C2F20000026802F12B
:10610000010202604FF0000140F64803C2F20003B2
:10611000197040F64900C2F2000001705DE040F6DF
:106120004801C2F200014FF000030B7040F6490035
:10613000C2F20000027802F10102027043E040F670
:106140004802C2F20002127840F64901C2F2000190
:106150000B7840F6AD01C2F20001097801FB032380
:1061600040F64C01C2F20001C95C814206D140F602
:10617000B001C2F20001097806291DD140F64C0495
:10618000C2F20004E0544FEA531040F6A001C2F2FC
:10619000000103F01F034FF0010404FA03F351F868
:1061A00020401C4341F8204040F6B400C2F20000F9
:1061B000016801F10101016002F1010240F64803AA
:1061C000C2F200031A7040F64800C2F2000040F626
:1061D0004901C2F20001FFF755FF4FF0000010BD6A
:1061E00070B4039D049C064628B140F6B000C2F28C
:1061F00000000078307029B140F6B800C2F200000B
:10620000007808702AB140F6AC01C2F200010878AB
:1062100010702BB140F6B902C2F200021178197069
:106220002DB140F64803C2F20003187828702CB153
:1062300040F64902C2F200021178217070BC70472A
:1062400007281DD8002808BF052040F6B003C2F279
:10625000000318704BF6B003C0F6050313F81010D6
:1062600040F6AD02C2F20002117003EB400041782B
:1062700040F6AE03C2F2000319704FF00100704700
:106280004FF00000704700BF08B540F6B803C2F2F7
:1062900000034FF001021A704FF00500FFF7D0FF26
:1062A0004FF00C004FF00001FFF706FF08BD00BFE4
:1062B00008B540F64802C2F20002107040F64903E9
:1062C000C2F20003197010461946FFF7DBFE08BD45
:1062D000034628B140F6AD00C2F200000078187005
:1062E00029B140F6AE03C2F20003187808702AB153
:1062F00040F6B401C2F200010B68136040F64C0096
:10630000C2F20000704700BF2DE9F00140F64C07D3
:10631000C2F200073F1853284BD8002A49D03B4609
:1063200007F1010702F1FF3257FA82F74FF000063A
:1063300040F6A004C2F200044FF001056FEA030C1E
:106340000CEB070202EA050C13F8018B01F1FF3197
:1063500011F8012F90452FD13DE013F801CB01F149
:10636000010049788C450ED003F8011C4FEA521108
:1063700002F01F0605FA06FC54F821604CEA0606F6
:1063800044F821602E4602F10102D2B2542A07D00D
:1063900013F801CB00F101014078844542D150E06F
:1063A0003EB140F6B403C2F20003196801F10101E5
:1063B0001960BDE8F001704703F8012C4FEA501650
:1063C00000F01F0805FA08F854F8262048EA0202EF
:1063D00044F826202E4600F10100C2B2542ADFD034
:1063E000BB42DDD0BCF1000FB7D013F801CB11F8E0
:1063F000010F84450ED003F8010C4FEA521002F051
:106400001F0605FA06FC54F820604CEA060644F81C
:1064100020602E4602F10102D2B2542AC0D0BB4203
:106420009BD1BDE703F8010C4FEA521002F01F06A2
:1064300005FA06FC54F820604CEA060644F8206091
:106440002E4602F10102D2B2542AA9D0BB4284D115
:10645000A6E700BF003018BF012040F6B803C2F223
:1064600000031870003118BF012140F6AC00C2F2E1
:1064700000000170003218BF012240F6B903C2F2D9
:1064800000031A70704700BF40F6AF03C2F200036A
:106490004FF000021A7070474FF05400704700BF71
:1064A00040F6AF03C2F200034FF001021A707047CA
:1064B000034628B10868834214BF002001207047BA
:1064C0004FF00000704700BF10B440F6E003C2F286
:1064D000000353E8002F02F1010243E800210129E3
:1064E000F7D00468C4B16268824202D192686260E7
:1064F00002E04368816899602368834202D15B6847
:10650000236002E0826841685160A26802F1FF31B5
:10651000A1604FF00004046040F6E003C2F2000303
:1065200053E8002FA2F1010243E80024012CF7D028
:1065300053E8002FB2F1004F0DD14FF0000243E8B5
:106540000024012CF4D04EF60450CEF20000016875
:1065500041F080510160BFF32F8F10BC704700BF26
:1065600038B504460D464FF000014FF0100212F00E
:106570003FF8E56038BD00BFF8B504460F46C66871
:106580008D192946FFF794FF00283CD140F6E0031F
:10659000C2F2000353E8002F02F1010243E8002198
:1065A0000129F7D04FF0000068606168A96001B16F
:1065B0004D60226802B925606560BC51A36803F193
:1065C0000103A36040F6E003C2F2000353E8002F8A
:1065D000A2F1010243E80024012CF7D053E8002F78
:1065E000B2F1004F0DD14FF0000243E80024012C1E
:1065F000F4D04EF60450CEF20000016841F0805114
:106600000160BFF32F8FF8BD2DE9F04104468846A5
:10661000C6688D199719C2B940F6E003C2F20003AB
:1066200053E8002F02F1010243E800210129F7D0CD
:1066300002686A6005604FF00000A860616809B9EF
:10664000656020E06B689D601DE03946FFF730FF14
:1066500000283FD02846FFF737FF40F6E003C2F29C
:10666000000353E8002F02F1010243E80021012951
:10667000F7D0B868A8606F60BD602168B9420EBFEE
:106680002560A9684D6048F80640A26802F1010241
:10669000A26040F6E003C2F2000353E8002FA2F12B
:1066A000010243E80024012CF7D053E8002FB2F197
:1066B000004F0DD14FF0000243E80024012CF4D02C
:1066C0004EF60450CEF20000016841F080510160A6
:1066D000BFF32F8FBDE8F081C368C918486808B1BF
:1066E000C01A70474FF00000704700BF036813B135
:1066F000C068181A70474FF00000704708B5C368AB
:10670000C918FFF7D5FE08BD08B5C0680818FFF71F
:10671000DBFE08BD08B540F6BC00C2F200004FF039
:106720001C01FFF71DFF08BD70B5054600F1080606
:106730003046FFF7DBFF0446686050B13046214623
:10674000FFF7E2FF4FF00100A861204600F07EFA5B
:1067500070BD4FF00003AB6170BD00BF38B504469B
:106760000D464FF000014FF0280211F041FF204686
:1067700040F8085B4FF01C01FFF7F2FE40F6BC004A
:10678000C2F200002146FFF7F7FE38BD2DE9F041C7
:106790000746884643F23453C2F2000318680028C3
:1067A00000F0FE8040F6E004C2F2000454E8002F3E
:1067B00002F1010244E800210129F7D0796831B1E2
:1067C00043F23452C2F20002136899422ED143F2CE
:1067D0003450C2F2000004687C60B96901F1010123
:1067E000B96140F6E003C2F2000353E8002FA2F1C2
:1067F000010243E80024012CF7D053E8002FB2F146
:10680000004F0DD14FF0000243E80024012CF4D0DA
:106810004EF60450CEF20000016841F08051016054
:10682000BFF32F8F4FF00100BDE8F081B8F1FF3FBB
:1068300024D140F6E003C2F2000353E8002FA2F196
:10684000010243E80024012CF7D053E8002FB2F1F5
:10685000004F0DD14FF0000243E80024012CF4D08A
:106860004EF60450CEF20000016841F08051016004
:10687000BFF32F8F4FF00000BDE8F08107F108054E
:106880002846FFF733FF0246F0B143F23456C2F216
:106890000006306892F8294090F829108C4208D9F7
:1068A00012E0336892F8290093F82940A04204D9F5
:1068B0000AE043F23456C2F2000628461146FFF7BA
:1068C0000BFF02460028ECD1284643F23451C2F2B5
:1068D00000010968FFF798FE40F6E006C2F20006E4
:1068E00056E8002FA2F1010246E80024012CF7D05F
:1068F00056E8002FB2F1004F0DD14FF0000246E8EC
:106900000024012CF4D04EF60450CEF200000168B1
:1069100041F080510160BFF32F8FB8F1000F04D018
:1069200008EB880000F028FB01E000F05DF940F67C
:10693000E004C2F2000454E8003F03F1010344E81C
:106940000032012AF7D043F23456C2F2000628463C
:106950003168FFF7D9FE54E8003FA3F1010344E892
:106960000032012AF7D054E8003FB3F1004F0DD1B7
:106970004FF0000344E80032012AF4D04EF60450F0
:10698000CEF20000016841F080510160BFF32F8F0B
:1069900078683268904214BF00200120BDE8F08181
:1069A0004FF00100BDE8F08110B5044643F23453C6
:1069B000C2F200031868002860D06268904201D0DB
:1069C000F9F78EFB40F6E003C2F2000353E8002F14
:1069D00002F1010243E800210129F7D0A16901F188
:1069E000FF30A06118B340F6E003C2F2000353E8A1
:1069F000002FA2F1010243E80024012CF7D053E854
:106A0000002FB2F1004F0DD14FF0000243E80024F7
:106A1000012CF4D04EF60450CEF20000016841F093
:106A200080510160BFF32F8F4FF0000010BD204652
:106A3000FFF77AFE40F6E003C2F2000353E8002FAE
:106A4000A2F1010243E80024012CF7D053E8002F03
:106A5000B2F1004F0DD14FF0000243E80024012CA9
:106A6000F4D04EF60450CEF20000016841F080519F
:106A70000160BFF32F8F4FF0010010BD4FF00100F8
:106A800010BD00BFF8B5054640F6E003C2F20003B2
:106A900053E8002F02F1010243E800210129F7D059
:106AA00040F6BC00C2F20000FFF720FE0446E0B151
:106AB00040F6BC07C2F200076068A84203D1204636
:106AC000FFF732FE0AE004F1080630462946FFF7D8
:106AD00015FE18B130462946FFF716FE3846214606
:106AE000FFF7FAFD04460028E6D140F6E003C2F2C3
:106AF000000353E8002FA2F1010243E80024012C17
:106B0000F7D053E8002FB2F1004F0DD14FF0000243
:106B100043E80024012CF4D04EF60450CEF20000DD
:106B2000016841F080510160BFF32F8FF8BD00BFB5
:106B300008B54BF6C003C0F60503195C012906D061
:106B400011B102290BD105E0FDF7E6F908BD02F00D
:106B50001DF908BDF9F7C4FA4FF0000008BD4FF069
:106B6000000008BD4EF60453CEF200031A6842F04E
:106B700080501860704700BF4FF0010280F8282055
:106B800040F6DC03C2F2000390F8291002FA01F289
:106B9000188802431A80704710B440F6D803C2F236
:106BA00000031A68C2B1904213D104E088420FD1A9
:106BB00002F1140203E040F6D802C2F20002436977
:106BC0001BB19C698169611899614369136003E095
:106BD0000A4651690029E9D14FF0000282614FF065
:106BE000FF31416110BC704710B5F9F7CFFA044688
:106BF00043F23453C2F20003186890F82820032AA5
:106C00001BD0F9F7C3FA43F23453C2F200031968F8
:106C10004FF0000281F8282091F82920096940F6F8
:106C2000CC13C2F2000343F82210F9F7B9FA204658
:106C3000F9F7B6FAFFF796FF10BD4FF0020180F8A2
:106C400028102046F9F7ACFA10BD00BF38B504464D
:106C500090B3036883B3F9F799FA054694F82800CE
:106C600010BB2046FFF788FF43F23451C2F2000107
:106C70000B6843B194F8292093F8290020F0010112
:106C8000531A002B15DA40F6E002C2F20002106837
:106C900038B140F0004140F6E003C2F20003196051
:106CA00007E0FFF75FFF04E0022804BF032084F839
:106CB00028002846F9F774FA38BD00BF2DE9F04FD7
:106CC00085B006460F46934698460F9DDDF84090E6
:106CD000F9F75CFA824640F62413C2F20003196801
:106CE000504881420FD240F20002C2F2020252F832
:106CF0002C4C54B14C4B1C468B4207D953F82C09F1
:106D00000028F8D102E0474C00E0464CA14206D1F1
:106D1000A1F12C0140F62412C2F2000211602046BB
:106D20004FF000014FF02C0211F062FC4FF0FF31E8
:106D300061611EB94BF6C416C0F605062660B8F1AF
:106D4000000F08D00E9B042B08D9184600F1030051
:106D50004FEA900604E04FF0000601E04FF0000615
:106D60000DBB44F23809C2F2000940F6CC05C2F26C
:106D70000005296847F2D910C0F604000090CDF84C
:106D80000480029648464FF000025B46F9F736FD54
:106D90002A68A260E0604FEA800153182B60C1EBC3
:106DA0000900606020E028464FF0FF314A46F9F7BD
:106DB000A7F94AF2ED52CDF6CE622A60E56005EB06
:106DC0008905656047F2D911C0F604010091CDF83C
:106DD00004800296284629464FF001025B46F9F7E7
:106DE0000DFDA5EB800363606FEA0702C2F3C011DB
:106DF00001EB470707F0FF0784F8297040F6E4032A
:106E0000C2F2000353F82700206143F827405046A0
:106E1000F9F7C6F92046FFF719FF204605B0BDE88F
:106E2000F08F00BFD4FF0120A8FF012030B585B04E
:106E30004FF0000143F23453C2F200031960284CB2
:106E400040F20005C2F202052A1B20464FEAA202C8
:106E5000F9F756F940F6CC00C2F200000460A5F143
:106E60002C0540F62411C2F200010D6043F63803F0
:106E7000C2F200034FF0B504CBF26B141C6003F1B7
:106E80004C004FF0FF3243F8042F43F8042F43F82F
:106E9000042F8342F9D14FF00004009440F62811EA
:106EA000C2F2000101914FF0280302934BF6D0107B
:106EB000C0F605004FF0070146F65972C0F604020D
:106EC0002346FFF7FBFE40F6C812C2F20002106034
:106ED00040F6E400C2F20000C46305B030BD00BF5C
:106EE0003C40002010B584B0069C00944FF0000494
:106EF00001940294FFF7E2FE04B010BD00B585B026
:106F00004FF00003009301930293FFF7D7FE05B003
:106F100000BD00BF38B543F23453C2F20003186815
:106F2000C0B1F9F733F9054643F23454C2F2000414
:106F30002068FFF721FE216891F82920086940F6B2
:106F4000CC13C2F2000343F822002846F9F728F9CF
:106F5000FFF708FE38BD00BF38B543F23455C2F222
:106F6000000540F6E404C2F200042B6822681A61AE
:106F7000FFF7D0FFF9E700BF38B543F23453C2F250
:106F800000031968002900F0918020B9FFF7C2FFC3
:106F90004FF001029AE0B0F1FF3F04D1FFF724FE69
:106FA0004FF0000292E040F6E004C2F2000454E820
:106FB000002F02F1010244E800210129F7D040F638
:106FC000D802C2F200021568002D7AD0AB6998424F
:106FD0006FD3C01A05F114016D691DB1AB6983420D
:106FE000F7D96AE043F23455C2F200052B68986184
:106FF000086858611846F9F777F840F6E004C2F2DD
:10700000000454E8003FA3F1010344E80032012AE0
:10701000F7D054E8003FB3F1004F0DD14FF000031B
:1070200044E80032012AF4D04EF60450CEF20000BB
:10703000016841F080510160BFF32F8FFFF7D4FD4D
:1070400054E8003F03F1010344E80032012AF7D07D
:1070500028684169B1F1FF3F04D0FFF79DFD4FF073
:10706000000201E04FF0010240F6E003C2F200032B
:1070700053E8004FA4F1010443E80045012DF7D087
:1070800053E8004FB4F1004F0DD14FF0000443E836
:107090000045012DF4D04EF60450CEF200000168F8
:1070A00041F080510160BFF32F8F0FE04FF00102DC
:1070B0000CE040F6D801C2F20001AC69221AAA61C4
:1070C00090E740F6D801C2F200018BE7104638BDC8
:1070D000F8B5044600287AD0F9F758F8064640F685
:1070E0002413C2F2000319683948814211D240F2D8
:1070F0000002C2F2020252F81C5CA54263D0354B7A
:107100001D468B4205D9A3F12C03D86BA042F7D1C1
:107110005AE094F8293040F6E402C2F2000252F834
:107120002300A04206D1016940F6E402C2F2000247
:1071300042F823102046FFF72FFD2046FFF7A2FC60
:1071400094F82900236940F6CC11C2F2000141F8FD
:10715000203043F23452C2F200021068A04229D01B
:10716000A06838B3E76800EB870540F6CC07C2F2A9
:1071700000073B685A1B29464FEAA2024FF0000362
:10718000FBF76AFBE1683868A0EB81033B6040F6DF
:107190002412C2F2000211680D4B99420AD29A6879
:1071A000954203D8E068A2EB80029A60A3F12C0319
:1071B0008B42F4D84FF00001216084F8281030464B
:1071C000F8F7EEFFF8BD024D21692961A1E7F8BD8E
:1071D000D4FF0120A8FF012000BFF04772B643F2A0
:1071E0003454C2F200042068FFF772FF4FF000032E
:1071F0002360F9F753FB00BF40F6D803C2F2000347
:10720000196849B1886950B100F1FF328A61D2F141
:10721000010038BF002070474FF0000070474FF06A
:107220000000704770B540F6D803C2F200031C6836
:10723000A4B1A06990B940F6D805C2F200054FF09C
:10724000FF3660692946F8F74FFF66612046FFF771
:10725000FDFC2C6814B1A1690029F2D070BD00BFFB
:107260002DE9F00172B640F6DC03C2F200031D887E
:107270002DB940F6C810C2F20000006867E04BF676
:10728000C408C0F6050840F6CC14C2F200044FF062
:10729000000C40F6E407C2F20007C5F100062E40DC
:1072A000300A1ABF18F80010083118F8061011F04B
:1072B000010F08D141F0010254F8220018B190F8F2
:1072C0002830012B3ED854F821200AB392F8280028
:1072D00030B140F6DC01C2F200010D80104636E00C
:1072E0001069824212D10CE090F828302BB140F6A0
:1072F000DC01C2F200010D8029E00369834204D160
:1073000000E01346C3F810C002E018460028EBD195
:1073100057F82100824207D1B543BED140F6DC02C6
:10732000C2F200021580A4E744F8210011F0010F19
:10733000C9D115EA4603C6D04FEA4606B6B241F0B7
:107340000101C0E740F6DC03C2F200031D8062B613
:10735000BDE8F001704700BF70B543F23453C2F28C
:1073600000031B6883420FD193F82820012A9CBF99
:10737000022283F8282093F8291040F6CC10C2F29C
:10738000000040F8213070BD40F6D002C2F2000289
:10739000136043F23451C2F20001086090F82920D2
:1073A00040F6CC13C2F2000343F8220090F82810F4
:1073B00001299CBF022180F828108268AAB9C168FF
:1073C0004AF2ED53CDF6CE630868984201D0F8F743
:1073D00087FE43F23452C2F2000211684868CB685B
:1073E00098427ED2F8F77CFE70BD40F6D403C2F21C
:1073F00000031B68984274D093B3586844F2380471
:10740000C2F20004251A4FEAA501D96043F63802FA
:10741000C2F2000290420AD34FF0B503CBF26B13D5
:1074200043F63800C2F2000004689C4201D0F8F72D
:1074300057FE40F6D405C2F200052A6840F6CC0497
:10744000C2F2000420685168D2684FF00003FBF7D5
:1074500003FA296823688B60C86803EB8002226006
:1074600043F23451C2F200010B6840F6D400C2F27C
:1074700000000360DA68002A33D0586899684FF03A
:107480000103FBF7E9F943F23456C2F2000635680E
:10749000A868EC6800EB840440F6CC06C2F2000653
:1074A0003268131B21464FEAA3024FF00003FBF79B
:1074B000D3F9E9683068A0EB8102326040F624130A
:1074C000C2F200031968074B99420AD29A689442A3
:1074D00003D8E868A2EB80029A60A3F12C038B42E8
:1074E000F4D870BDD4FF012000B585B040F66830F7
:1074F000C2F200004FF00001FFF732F840F6102012
:10750000C2F200004FF00001FFF72AF84FF000032D
:10751000009340F62822C2F2000201924FF0500080
:1075200002904BF6D810C0F60500194647F63D020A
:10753000C0F60402FFF7C2FB40F60C23C2F20003C0
:10754000186005B000BD00BF08B5FFF7CFF80346CF
:1075500048B1C06850B100F1FF31D960D1F10100EC
:1075600038BF002008BD4FF0000008BD4FF00000FC
:1075700008BD00BF70B505460E46144640F6E00350
:10758000C2F2000353E8002F02F1010243E8002198
:107590000129F7D0FFF7AAF80246002839D0C068C1
:1075A00084422DD3241A28461146FFF795F8024647
:1075B00000282ED0C068A042F4D921E040F6E003B4
:1075C000C2F2000353E8002FA2F1010243E80024B5
:1075D000012CF7D053E8002FB2F1004F0DD14FF03E
:1075E000000243E80024012CF4D04EF60450CEF201
:1075F0000000016841F080510160BFF32F8F70BD22
:10760000F460D1680B1BD36028463146FEF7FCFFBF
:10761000D4E7F46028463146FEF7AEFFCEE700BF60
:10762000F8B50646FFF762F80446F8B1C368EBB94F
:1076300030462146FFF750F80546F8F7A7FD074604
:1076400030462146FFF760F83846F8F7A9FD226971
:107650001AB130462146FFF78DFF04F11400FDF703
:10766000E3FD1DB12C46E8680028E1D0F8BD00BF5D
:1076700008B540F62423C2F200031A6802F10102A1
:107680001A6040F61020C2F20000FFF75DFF28B13B
:1076900040F61020C2F20000FFF7C2FF08BD00BF95
:1076A00008B5014640F66830C2F20000FFF726F840
:1076B00020B140F66830C2F2000008BD40F610204C
:1076C000C2F2000008BD00BF70B5044640F6E003FA
:1076D000C2F2000353E8002F02F1010243E8002147
:1076E0000129F7D0FFF7DCFF05462146FFF706F832
:1076F000002845D040F6E000C2F2000050E8002F1C
:1077000002F1010240E800210129F7D02846214674
:10771000FEF7E2FF18B1C168E2688B18C360F8F7A2
:1077200035FD064628462146FEF7EEFF3046F8F7BF
:1077300037FD4FF0FF35E56040F6E003C2F200038D
:1077400053E8002FA2F1010243E80025012DF7D0F4
:1077500053E8002FB2F1004F0DD14FF0000243E883
:107760000025012DF4D04EF60450CEF20000016841
:1077700041F080510160BFF32F8F4FF0010501E010
:107780004FF0000504F11400FDF748FD40F6E0035A
:10779000C2F2000353E8002FA2F1010243E80024E3
:1077A000012CF7D053E8002FB2F1004F0DD14FF06C
:1077B000000243E80024012CF4D04EF60450CEF22F
:1077C0000000016841F080510160BFF32F8F28460F
:1077D00070BD00BF2DE9F04105460F46144698469E
:1077E000FFF772FF064694B19DF82030002B14BFBE
:1077F00020460020286105F114004146069A079BA7
:10780000FDF7F2FC384629462246FFF7B3FE304624
:10781000BDE8F08170B584B00E4615460093089C13
:1078200001949DF82430029340F66831C2F20001C1
:1078300032462B46FFF7CEFF04B070BD00B583B0D3
:107840004FF0000300934FF00100019040F67830B4
:10785000C2F2000041F288314FF0FF0247F271633B
:10786000C0F60403FFF7D6FF40F66834C2F2000406
:10787000FFF7D8FC2046FFF7D3FEFFF7B5F9F7E78F
:1078800040F62023C2F2000318681A689042FBD128
:10789000704700BF10B540F62023C2F200031A68FB
:1078A00002F101021A60FFF7A7FC044640F66830B7
:1078B000C2F20000FFF748FE204310F0FF0F06D091
:1078C00040F60C20C2F200000068FFF7BFF910BDBF
:1078D00008B54BF6E410C0F605004FF0060147F678
:1078E0000D52C0F60402FFF709FB40F66C63C2F2CA
:1078F0000003186008BD00BF38B504460D4640F6C9
:10790000A033C2F20003586AA0420AD040F6A03168
:10791000C2F200014C620A681AB115B14948FDF77C
:1079200083FC40F6A033C2F20003186F84420AD0F1
:1079300040F6A031C2F200010C67CA6C1AB115B151
:107940004148FDF771FC40F6A033C2F20003D3F8C2
:10795000BC0084420CD040F6A031C2F20001C1F854
:10796000BC40D1F898201AB115B13848FDF75CFC3D
:1079700040F6A033C2F20003D3F8080184420CD0D1
:1079800040F6A031C2F20001C1F80841D1F8E4206C
:107990001AB115B12E48FDF747FC40F6A033C2F2EC
:1079A0000003D3F8540184420CD040F6A031C2F257
:1079B0000001C1F85441D1F830211AB115B1254860
:1079C000FDF732FC40F6A033C2F20003D3F8A00169
:1079D00084420CD040F6A031C2F20001C1F8A041AF
:1079E000D1F87C211AB115B11B48FDF71DFC40F6FA
:1079F000A033C2F20003D3F8EC0184420CD040F66D
:107A0000A031C2F20001C1F8EC41D1F8C8211AB18D
:107A100015B11248FDF708FC40F6A033C2F200038E
:107A2000D3F83802A0420CD040F6A031C2F20001D7
:107A3000C1F83842D1F814221AB115B10848FDF73F
:107A4000F3FB38BDB00B0020FC0B0020480C0020DD
:107A5000940C0020E00C00202C0D0020780D00205C
:107A6000C40D00202DE9F04707460D4691460898C1
:107A7000DDF828800C683E68D8F800108A19944216
:107A800002D80219964203D304192C60BDE8F0878E
:107A9000341B061BB14234BF8A46B246099931B144
:107AA000D9F8000008181919524610F07DFDD8F8D1
:107AB0000030CAEB0302C8F800203E6806EB0A015A
:107AC0003960D9F8000000EB0A03C9F800302E68CD
:107AD000A41954442C60BDE8F08700BF70B584B091
:107AE0009CF81960157A947B4FF007038CF81030DE
:107AF0004FF005028CF8112006F00F0260F3C71258
:107B00008CF812204FF0000065F301008CF8130090
:107B10004FF0000261F30A02ACF814208CF8164012
:107B2000DCF80C100093DCF804300193CDF808C0A9
:107B300001F104000CF108020CF11003FFF792FFB1
:107B400004B070BD2DE9F04F8FB007460591144683
:107B50004FF000030793136012896068131A8B4279
:107B600038BF05930599002900F0AA8040F670659A
:107B7000C2F200052D6815B34FEAC5054FF00002AB
:107B80004FF0FF01134640F67860C2F20000A5F105
:107B90000806C6F3C00E1658F6798E4240F095805E
:107BA00096E01658F6798E421CBF0133314602F139
:107BB00008028658F6798E4240F09F80A0E04FF090
:107BC000000303EB43024FEAC20000F110000890EB
:107BD0004FF48071ADF824104FF00402ADF8262068
:107BE0008DF828300DF129004FF000014FF0070209
:107BF00010F0FEFC04F1040B04944FF0100300930A
:107C0000019705A802905846214607AA08ABFFF73E
:107C100029FF0599002951D04FF001028DF821204C
:107C20000DF132004FF000014FF0060210F0E0FCC1
:107C300040F67063C2F20003186800283ED04FF08F
:107C4000FF014FF0000440F67869C2F200094BF6DC
:107C5000F818C0F6050840F6706AC2F2000A59F832
:107C60003450ED798D4223D08DF820404FEA05162F
:107C70000DF1220008EB06014FF0080210F094FC11
:107C800006F108010DF12A0041444FF0080210F0FE
:107C90008BFC4FF018020092019705AB02935846F7
:107CA000049907AA08ABFFF7DDFE059830B1294615
:107CB00004F10104DAF80020A242D0D8079801E0CC
:107CC0004FF0FF300FB0BDE8F08F03F101033146F4
:107CD00002F10802AA423FF474AFBEF1000F3FF474
:107CE00060AF1658F6798E421CBF0133314602F15F
:107CF0000802AA427FF455AF63E703F1010331465E
:107D000002F10802AA427FF44CAF5AE72DE9F04194
:107D10004FF00100FDF704F94BF68C20C0F605008A
:107D2000FCF782FF40F69963C2F200034FF00102B4
:107D30001A7040F66860C2F20000016841B940F66E
:107D40006864C2F20004FEF74FFF2568002DFAD0E8
:107D500040F67567C2F2000740F69964C2F200046B
:107D600040F60066C2F2000640F69865C2F20005D1
:107D700040F66468C2F200083B783BB14FF0000265
:107D80003A704FF002002070FDF7C4F8317859B115
:107D90004FF000033370227862F07F0020704FF0C4
:107DA00001000146FFF7A8FD297851B14FF000000E
:107DB0002870237803F07F0222704FF00101FFF753
:107DC0009BFD98F8000010B9FEF70EFFD4E740F6CF
:107DD0009961C2F200014FF002030B704FF00000F6
:107DE000FDF79EF8BDE8F08108B540F66863C2F281
:107DF0000003186040F66C60C2F200000068FEF7F5
:107E000025FF08BD70B505460E4640F69C33C2F20C
:107E100000031868032801D9F8F762F940F69C328C
:107E2000C2F20002116840F64464C2F2000444F851
:107E3000316004EBC104656001F10101116070BDA6
:107E400070B505460C461646032801D9F8F748F9DF
:107E500040F67863C2F2000353F8350008B1F8F732
:107E60003FF940F67861C2F2000141F8354001EB7C
:107E7000C5056E6040F67063C2F200031A6802F135
:107E800001021A60206930B1FCF7CEFE04F104044F
:107E900020690028F8D170BD08B540F6A033C2F2C1
:107EA0000003196881425AD040F6A032C2F20002A3
:107EB000D36C834234D040F6A031C2F20001D1F835
:107EC000982082422FD040F6A033C2F20003D3F8AC
:107ED000E41081422AD040F6A032C2F20002D2F869
:107EE0003031834225D040F6A031C2F20001D1F8F2
:107EF0007C21824220D040F6A033C2F20003D3F8A6
:107F0000C81181421BD040F6A032C2F20002D2F862
:107F10001432834216D0F8F7E3F84FF0080013E06C
:107F20004FF0010010E04FF002000DE04FF00300B1
:107F30000AE04FF0040007E04FF0050004E04FF0C6
:107F4000060001E04FF0070040F6A031C2F2000148
:107F50004FF04C0202FB001090F8200008BD4FF0DB
:107F60000000F1E72DE9F04F8FB0089007910A92D9
:107F70004FF0000309931360546813891B1B8B4255
:107F800038BF07930799002900F04A81082C69D867
:107F900040F67064C2F20004D4F800E040F69C356C
:107FA000C2F200052E680EEBCE0707EBC60404F103
:107FB00009044FF0000140F67867C2F20007CB5980
:107FC0008BB1DD68641903F110051B695BB15E8933
:107FD0000EB104F107049B890BB104F1070455F8B5
:107FE000043F002BF3D101F108012029E7D140F62D
:107FF0006861C2F200010D682F7E6E7EEB8A03F18C
:108000000103C3F347054FF000010C914FF0090342
:108010008DF82C304FF002018DF82D10ADF82E4068
:108020008DF830E04FF001018DF831104FF0000174
:1080300067F3451166F3861161F07F018DF8331007
:108040008DF834500093019007A8029002F10400CB
:10805000114609AA0BABFFF705FD079A002A00F0AD
:10806000DD80E0E04FF009001060DCE05BF83640B6
:10807000002C00F0CE80059D286800284BD07A683F
:10808000B2420CD04FF0000310F0010F3ED1DFE000
:1080900007EBC3025268B24240F0E38001E04FF0C8
:1080A000000357F83300D2B290F8048090F805C06E
:1080B00090F806E0C579016819B143F01000C3B229
:1080C00001E04FF000034FF008008DF82C004FF056
:1080D0000B018DF82D108DF82E208DF82F808DF846
:1080E00030C08DF831E08DF832508DF833300A9978
:1080F0000090089A019207AB029301F1040009AACB
:108100000BABFFF7AFFC079828B987E003F1010537
:108110002B468542BCD104F1100523697BB1294669
:108120004FF00002588908B102F101029B890BB19E
:1081300002F1010251F8043F002BF3D101E04FF0AE
:1081400000025FFA86FCD2B294F804E06079A1796B
:1081500023681BB146F02003DBB201E04FF00003BF
:108160008DF82CA04FF004088DF82D808DF82EC0CE
:108170004FF0000C8DF82FC08DF830208DF831E0D5
:108180008DF832008DF833108DF834300A99CDF81F
:1081900000A0089A019207A8029001EB080009AA22
:1081A0000BABFFF75FFC0799002937D0A3686BB1D1
:1081B0000A99E26800920898019007AA029201EBDE
:1081C000080009AAFFF74EFC079B3BB3246904B3E0
:1081D0004FF001084FF000092046FFF75DFE8DF8D3
:1081E0003500618939B10DF11C0C40462246FFF77C
:1081F00075FC079991B1A18939B10DF11C0C484664
:108200002246FFF76BFC079840B155F8044F002C4D
:10821000E2D106F10106042E7FF428AF099814E09C
:108220004FF0FF3011E04FF0000640F6786BC2F2DD
:10823000000B40F69C34C2F2000405944FF0090A8A
:1082400040F64467C2F2000710E70FB0BDE8F08FB8
:1082500003F1010307EBC3014A68B2427FF456AF52
:108260001FE705F1010307EBC3014A68B2427FF43F
:108270004DAF16E708B540F6A463C2F200031A5CDE
:1082800040F6A031C2F200014FF04C0000FB02109A
:10829000436AD3F1010238BF002242634FF000016C
:1082A000C1630164416400F11000FCF7BDFF08BD2B
:1082B0002DE9F84F81468A4640F6A463C2F20003D6
:1082C0001A5C40F6A030C2F200004FF04C0404FBF0
:1082D000020404F148064FF001084FF0000740F691
:1082E000B86BC2F2000B354640463146F7F7FCFE4C
:1082F00030B14FF002003146F7F7F6FEBDE8F88FD7
:10830000BAF1000F05D148464146FCF7B9FB0328F6
:1083100027D0256C75B15846A168E26BA847054681
:10832000B0F1FF3F14D06064484659462A46FCF736
:10833000CDFB0EE0616CA5688D4228BF0D46484616
:10834000E16B2A46FCF7C2FBE36B5A19E26300E0DB
:108350003D46606CA16888423CBFE7632764451BCB
:10836000656438463146F7F7BFFE0228BBD0BDE84A
:10837000F88F00BFF8B505460E46174640F6A463D1
:10838000C2F200031A5C40F6A030C2F200004FF0C7
:108390004C0404FB02044FF00000FCF7C9FAE76349
:1083A00026644FF00001616428464FF00101FFF799
:1083B0007FFF4FF00100FCF7BBFAF8BDF8B50546AA
:1083C0000F46164640F6A463C2F200031A5C40F65C
:1083D000A030C2F200004FF04C0404FB0204A1687C
:1083E000B1420DD243F63803C2F200039F4207D3D5
:1083F00044F23802C2F20002974201D2F7F770FE4F
:108400004FF00000FCF794FAE7634FF0000020649F
:10841000666428464FF00101FFF74AFF4FF0010064
:10842000FCF786FAF8BD00BF08B5FCF7D7FB08BD1E
:1084300070B586B005460C46164602A8F9F73CF919
:1084400001462EB102A82A46234600F0A9FD07E006
:108450004FF00103009302A82A46234600F052FE83
:1084600006B070BD70B58AB00378212B00F0938000
:1084700004D86BB1012B40F0D88186E0A12B00F02D
:10848000A781C02B00F0B481802B40F0CE8195E015
:108490004178052903D0092940F0CA8146E0408887
:1084A00040F69962C2F200021378022B02D0032B2D
:1084B00033D118E000F1FF318AB27E2A30D8C0B241
:1084C00040F6B463C2F2000318704FF00201FCF7EB
:1084D00091FC40F69960C2F200004FF00301017078
:1084E0004FF00100C3E170B940F6B462C2F200027D
:1084F000107040F69960C2F200004FF00203037062
:108500004FF00100B3E17F280DD840F6B461C2F20C
:10851000000108704FF00100A9E14FF00200A6E150
:108520004FF00200A3E14FF00200A0E1827840F694
:108530009963C2F200031978022923D972B940F66F
:108540009963C2F200034FF0030119704FF001006C
:108550000146FFF7D1F94FF0010088E1012A18BF69
:10856000022040F0848140F69960C2F200004FF092
:10857000040202704FF000000146FFF7BDF94FF012
:10858000010074E14FF0020071E140780B280CBF4C
:10859000012002206BE18388032B00F24C8140F61E
:1085A0007864C2F2000404EBC3035B68002B00F0A4
:1085B00045819847002808BF022058E142781AB147
:1085C000062A40F03E8121E0C18802291BD14FF0EC
:1085D0000000ADF8040040F66862C2F200021268C2
:1085E0000346517E61F30003ADF80430127E62F35E
:1085F00041030AA921F8243D4FF00202FFF7DEFEF5
:108600004FF0030033E14FF0020030E18278C1887F
:108610008CB2C378022B2ED0032B3DD0012B40F01F
:10862000D48040F60465C2F2000528464BF6782156
:10863000C0F605014FF012020FF0B6FF40F6686079
:10864000C2F2000001688A892A81CB896B81088A7D
:10865000A8818A7C2A71CB7C6B71097DA9714FF04E
:1086600000002946122C34BF22461222FFF7A6FE34
:108670004FF00300FBE040F6F862C2F20002118105
:108680004FF00000506047F66571C0F60401FFF737
:1086900071FE4FF00300EAE0D2B940F60464C2F282
:1086A000000404F102004BF6F411C0F605014FF08E
:1086B00002020FF079FF4FF0040222704FF0030521
:1086C00065704FF000002146FFF778FE2846CEE0A7
:1086D000012A06D140F66863C2F2000319680968EE
:1086E0002FE0022A06D140F66862C2F2000210684A
:1086F000416826E0032A06D140F66863C2F200030F
:10870000196889681DE002F00F0022F00F03102B9A
:1087100008D15A4B196888420EDA594A52F830008B
:1087200001680EE0202B07D1032805D8554951F8E0
:10873000300008B1016804E0EE2A04D04FF00200D6
:1087400095E009B93EE05049B1F1FF3F40F0888023
:1087500001A84FF020014FF00102FFF769FE0AADBA
:108760002A184FF0000002F8240C01A978E000F16B
:108770000206428003F10102134611F8015F5DB168
:1087800000F10400758002F1010311F8012F002AA5
:108790006FD101E04FF0000340F60461C2F2000126
:1087A0004FF003054D7003F101034FEA4303DAB2C2
:1087B0000A704FF00000A24228BF2246FFF7FEFDDC
:1087C000284654E04FF0020051E04FF002004EE026
:1087D0008388032B38D840F67864C2F2000404EB97
:1087E000C3035B689BB39847002808BF02203EE0A4
:1087F0004378212B2ED1C18840F6F863C2F20003E2
:1088000019814FF000025A608088042825D1104653
:1088100047F64531C0F6040140F6F862C2F20002A4
:10882000FFF7A8FD4FF0030021E04FF002001EE02B
:108830004FF002001BE04FF0020018E04FF0020082
:1088400015E04FF0020012E04FF002000FE04FF091
:1088500002000CE04FF0020009E04FF0020006E0D9
:108860000A78002A96D009484FF000037FE70AB043
:1088700070BD1E2B7FF47BAF8EE700BF9C0B0020EA
:10888000440E0020780E0020E8B90508040E0020F0
:1088900010B50446436993B14FF00000606140F6A3
:1088A0009961C2F200010A78032A08D140F6B46344
:1088B000C2F2000318784FF00301FCF79BFA20691D
:1088C00058B34FF000002061E06040F67461C2F2DE
:1088D0000001087040F69C61C2F200014FF00802EE
:1088E000FFF7A2FD082853D140F69C62C2F20002B5
:1088F000137813F0800F06D140F69C60C2F200009E
:10890000C188002944D140F69C60C2F200004FF0BB
:1089100000010A46FFF7A6FD2DE0E168002937D0E7
:108920004FF00000E06040F67462C2F2000213787B
:1089300040F60461C2F20001C3F14002FFF774FD8A
:10894000034628B340F67460C2F2000001785A185A
:10895000D2B2027040F69C63C2F20003D888904203
:1089600016D140F69C60C2F2000040F60461C2F2EB
:108970000001FFF777FD012804D0022808D1FCF799
:108980008FF810BD4FF0000001460246FFF716FDBC
:1089900010BD00BF08B540F60473C2F200031B69A6
:1089A0003BB14FF0000140F60472C2F2000252697E
:1089B000984740F60470C2F200004FF000010170C9
:1089C00041608160C1600161416108BD40F6047091
:1089D000C2F2000081614BF6AC21C0F605018A5C51
:1089E00042778377037F6FF3070303774FF000012C
:1089F00041624FF00100704730B583B040F6047417
:108A0000C2F200042070089D6560099DA5600A9D62
:108A1000E5600B9D25610C9D65619DF818400094F3
:108A20009DF81C400194FFF7D1FF4FF0010003B007
:108A300030BD00BF40F60473C2F200035B6AB3F1BD
:108A4000FF3F09D140F60471C2F200014FF000036C
:108A50004B624FF0010070473F2B0BD840F6047279
:108A6000C2F20002106AC15403F1010353624FF0D5
:108A7000010070474FF00000704700BF704700BF13
:108A800070B540F60474C2F2000404F118004BF60D
:108A90003C31C0F605014FF007020FF085FD4FF0A5
:108AA00000004BF6F821C0F60501FFF7ABF948F6D8
:108AB000F546C0F604064FF000004BF6E021C0F684
:108AC00005013246FFF7BCF94BF61035C0F6050537
:108AD0004FF0010029463246FFF7B2F92869FFF747
:108AE000DBF984F8280040F63070C2F200004FF045
:108AF000070148F60532C0F604024FF00003FCF708
:108B000073FB70BD38B540F6E473C2F200034FF05A
:108B100001021A7040F60474C2F2000494F82800AE
:108B20004FF000010A46FFF749FC606868B140F663
:108B30000474C2F200044FF0FF3565626368207868
:108B400061699847616A0029F7D040F60470C2F263
:108B500000004FF000024262836833B140F60471B6
:108B6000C2F2000108784969984738BD2DE9F04FF5
:108B700083B0804643680BB9806828B14FF000018C
:108B8000C8F80810FFF7BEFFD8F80C20002A45D01F
:108B90004FF00003C8F80C30D8F8000040F68071A0
:108BA000C2F200014FF04002FFF73EFC814640F662
:108BB0000470C2F20000C16800292FD0B9F1000F83
:108BC0002CD040F60474C2F2000440F68076C2F263
:108BD00000064FF0000509F1FF3B0BF0010B207878
:108BE000715D2A466369E768B84705F1010AD14516
:108BF00070D113E0207816F80A102A466369E768F6
:108C0000B8470AF1010A207816F80A102A46636963
:108C1000E768B8470AF1010AD145EBD1D8F814202A
:108C2000002A54D04FF0000440F6E473C2F200036F
:108C30001C70C8F8144040F6C070C2F20000FEF785
:108C400043FD40F60470C2F200004462416800290E
:108C500036D040F60475C2F2000540F64074C2F208
:108C600000042C622C46656A62682078616990472E
:108C7000636A9D42F7D11DB3D8F8000040F64071F9
:108C8000C2F200012A46FFF799FB4FF00000009066
:108C9000019040F6C070C2F200004FF04B014FF05F
:108CA000FF0248F60533C0F60403FEF7B3FD0EE0FD
:108CB00040F60472C2F2000210785169984706E04B
:108CC00040F60471C2F200018B68002BF0D103B0B2
:108CD000BDE8F08FBBF1000F8CD0207816F80A1099
:108CE0002A466369E768B8470AF1010AD14581D18C
:108CF00094E700BF10B544780378212B02D0A12B54
:108D00001BD10EE0202C04D0222C14BF0020012007
:108D100010BD072A14D10D480FF046FC4FF001009A
:108D200010BD212C0FD14FF0000008494FF0070271
:108D3000FFF744FB4FF0030010BD4FF0000010BDE3
:108D40004FF0020010BD4FF0000010BD1C0F0020BE
:108D500008B540F6E473C2F20003187870B940F623
:108D60000471C2F200014A6A72B940F60473C2F299
:108D7000000393F82800FFF77DFA08BD40F6307035
:108D8000C2F20000FCF750FA08BD00BF4BF6B0205D
:108D9000C0F60500704700BF70B4037801298CBF8E
:108DA0004478002402298CBF85780025DCF8000077
:108DB00048B34FEA93064BF67C40C0F60500365C9C
:108DC00016704FEA031343EA141303F03F031B5CCE
:108DD0005370012907D94FEA840444EA951303F03C
:108DE0003F04205C01E04FF03D009070022907D95C
:108DF00005F03F054BF67C43C0F60503E95C01E056
:108E00004FF03D01D17070BC704700BF82B04FF091
:108E100015010CE00191019B03F1FF32019233B186
:108E200000BF019B03F1FF320192002BF8D100F14A
:108E3000FF30B0F1FF3FEDD102B0704770B4C4B263
:108E40004FEA10204BF61056C0F605064BF67C355F
:108E5000C0F6050511F8013B1AB94BB944EA0020E8
:108E60000BE06340F45C4440E85C013AF2D1F5E782
:108E70006340F45C4440E85CECE770BC704700BFC2
:108E800010B444F6FB43C0F2861311F8014B02B94B
:108E9000ACB380EA04404FEA400010F0807F18BF76
:108EA00058404FEA400010F0807F18BF58404FEA0A
:108EB000400010F0807F18BF58404FEA400010F08B
:108EC000807F18BF58404FEA400010F0807F18BFE5
:108ED00058404FEA400010F0807F18BF58404FEADA
:108EE000400010F0807F18BF58404FEA400010F05B
:108EF000807F18BF5840002AC7D0013AC5D120F062
:108F00007F4010BC704700BF82B001909DF80630D2
:108F10004FF0000063F307009DF8052062F30F2077
:108F20009DF8042062F317409DF8072012F0800F8F
:108F300014BF63F07F0103F07F0161F307004FEA84
:108F40004201CAB262F31F6013F0800F18BF42F0F3
:108F5000010262F31F6002B0704700BF84B0C0F32B
:108F600007438DF80C30C0F307228DF80D20C3B2F3
:108F70004FEA10604FEA500210F0010F14BF63F087
:108F80007F0103F07F018DF80E1013F0800F18BFE2
:108F900062F07F028DF80F20039804B0704700BF85
:108FA0002DE9F04F83B005460F4614461E46019248
:108FB00001F1FF3313F1050F44D8032E43D9A6F175
:108FC0000400C0F380080DF1040C2846FFF7E4FE0E
:108FD00005F10305A7F1030104F10404A6F1040659
:108FE000A7F1040717F1050F67D92CE00DF1040C68
:108FF000284639462246FFF7CFFE05F1030B5D46B2
:10900000A7F1030104F1040A5446A6F104094E46EF
:10901000A7F1040717F1050F15D80F460DF1040C41
:1090200058465246FFF7B8FE0BF10305A7F10301BE
:109030000AF10404A9F10406A7F1040818F1050FC8
:1090400059D900E0FFE799B396B30DF1040C284617
:109050006A46FFF7A1FE022E11D0032E02D0012E88
:1090600026D11AE0019929B19DF8002022704FF015
:10907000010301E04FF0000304F1010401E04FF0AF
:109080000003019830B102A9CA1812F8080C207028
:1090900003F1010304F1010401E04FF00003019921
:1090A00021B102AAD31813F8080C207004F10104AE
:1090B0000199601A03B0BDE8F08F0F46032EC2D9A4
:1090C000B8F1000F92D00DF1040C28462246FFF7AC
:1090D00063FE05F10305A7F1030104F10404A6F101
:1090E0000406A7F1040717F1050FACD80F46032EAD
:1090F0003FF67CAFA7E7A7F10307032E3FF676AF55
:10910000A1E700BFF0B49DF81040ECB14FEA410771
:109110009F421CD2DD1B1DD056194FF030046FEA60
:109120000203F31803F0010302F8014BB24240F0CE
:10913000928007E0134603F8014B547003F10102DB
:10914000B242F7D13B4607E04FF0000504E04FF094
:10915000000501E04FF0000500293CD003F1FF3489
:10916000002B3AD000F1010341182846521B04F1AC
:10917000FF3515F0020F10D032E0A4F1020603F122
:1091800001031F46012C29D03446B44613F8016C64
:109190004FEA1616092E42D944E01E4613F8015C28
:1091A0004FEA1515092D8CBF37353035155414B9D4
:1091B00000F1010012E013F8016C06F00F05092D13
:1091C0008CBF373530351618757000F1020528460A
:1091D0008B42D2D102E0284600E02846F0BC70471E
:1091E0001E4613F8015C4FEA1515092D94BF303562
:1091F00037351554002CDBD013F8016C06F00F0541
:10920000092D94BF303537351618757000F10200FE
:109210008B42E3D003F10103A4F10204BDE706F1A0
:10922000300601E006F137065655BCF1000FBFD0FD
:1092300013F8016C06F00F06092E94BF303637364E
:109240001018467005F102008F42C7D003F10103E8
:10925000A4F10204A1E7002B3FF46CAF02F8014B2C
:10926000B2427FF467AF6DE7DCF8143093F8452025
:1092700083F84420DCF8141091F8463081F845302A
:10928000DCF8141091F8472081F84620DCF81430FF
:1092900083F84700704700BFDCF8143093F84700AC
:1092A00093F8462083F84720DCF8141091F84530F5
:1092B00081F84630DCF8141091F8442081F84520FC
:1092C000704700BF43F2B812C2F20002136840F2C6
:1092D0000001C0F60201C85CC918497803F1020315
:1092E000136041EA00207047DCF80430DCF8082005
:1092F00002EBD300CCF8080003F007014FF00103A4
:1093000003FA01F2CCF80420704700BF2DE9F04FBA
:1093100083B004468A4693461E46CDF804C04FF0FB
:109320000007B846B9463DE025463046D0470346DB
:1093300000283DD0B9F1000F0CD1202829D00928F0
:1093400029D00A2829D00D2829D0022D4FF0010953
:1093500088BF0225A3F13002D1B2092910D9A3F1A7
:109360004100C1B2052903D8A3F13703D9B207E000
:10937000A3F16102D0B205281AD8A3F15703D9B2DC
:109380004FEA0717FCB241EA040708F101082C462E
:1093900006E02C4604E02C4602E02C4600E02C4679
:1093A0003046D847FF2CBFD004F1FF35002CBCD18C
:1093B000DDF804C03846FFF757FF019B5A69D8F122
:1093C000010838BF4FF0000882F8508003B0BDE8B4
:1093D000F08F00BF43F26403C2F200031B684B63CB
:1093E0004BB19A68824209D0DB684B631BB19A6823
:1093F0008242F9D102E04FF01E0070474FF00000AA
:10940000704700BF884204D8884234BF0220002041
:1094100070474FF001007047D0F80431D0F80021B8
:10942000934214BFC05C0020704700BFD0F80431E5
:10943000FF2B14BF01330023C0F80431704700BF75
:1094400010B4DCF81420D16C0B46044658B14FEA36
:10945000016343EA116301F47F4043EA002301F40E
:109460007F0143EA1123DCF8040030B199B24FEADE
:10947000134060F30F0361F31F435CB94FEA0361CC
:1094800041EA136103F47F4041EA002103F47F03C2
:1094900041EA1323D36410BC704700BFDCF80030EE
:1094A000B3F5005F05D240F6E872C2F20002D05C6C
:1094B00070474FF000007047DCF8003003F1010303
:1094C000CCF80030DCF8140090F8512002F10102D1
:1094D00080F85120704700BF70B404460846A1B11F
:1094E00099188C4211D22518AA420ED294423ABF42
:1094F000C4EB0206F6B20026A94205D20019821A70
:10950000D31AF118C8B200E0304670BC704700BFF3
:10951000F0B583B043F23C03C2F200034FF01402F3
:109520001A7043F22000C2F2000004683CB31546F2
:1095300043F23C07C2F200074FF0000621680B68B7
:1095400073B10DF107000DF1060198479DF8070072
:109550009DF8061032463B78FFF7BEFF4519EDB285
:109560006468002CEAD143F23C02C2F20002107897
:10957000A84204D243F23C01C2F200010D7043F252
:109580003C03C2F200034FF010025A7043F254043D
:10959000C2F2000424683CB3154643F23C07C2F211
:1095A00000074FF000062068036873B10DF1070053
:1095B0000DF1060198479DF807009DF80610324608
:1095C0007B78FFF789FF4519EDB26468002CEAD17A
:1095D00043F23C01C2F200014A78AA4204D243F2AB
:1095E0003C00C2F20000457043F23C03C2F20003AB
:1095F0004FF00201997043F23404C2F2000424686F
:109600003CB30D4643F23C07C2F200074FF00006A0
:109610002268136873B10DF107000DF10601984738
:109620009DF807009DF806103246BB78FFF754FFFF
:109630004519EDB26468002CEAD143F23C00C2F255
:1096400000008178A94204D243F23C02C2F2000237
:10965000957043F23C03C2F200034FF00100D87052
:1096600043F21804C2F2000424683CB3054643F2F6
:109670003C07C2F200074FF0000621680A6872B189
:109680000DF107000DF1060190479DF807009DF8C8
:1096900006103246FB78FFF71FFF4519EDB26468EC
:1096A000002CEAD143F23C03C2F20003D878A8426E
:1096B00004D243F23C01C2F20001CD7003B0F0BD10
:1096C00043F28C13C2F20003196840F20000C0F6A6
:1096D0000400401A704700BF034610B182688A42F6
:1096E00018D043F23803C2F20003186860B18268F0
:1096F0008A4203D10BE083688B420AD0406800287D
:10970000F9D14FF0000305E04FF0000302E00346FB
:1097100000E003461846704710B540F2A064C1F25D
:1097200000044FF4117303FB0044D4F80811B1F1A5
:10973000FF3F03D0D4F8042191420DD123689A6AE7
:109740004FF0FF019047002834D0D4F8080100F111
:109750000100C4F8080110BD91422BD86318197993
:1097600043F2CC12C2F2000213787BB9FD290FD963
:1097700023689A6A4FF0FE019047D8B143F2CC10AB
:10978000C2F200004FF00101017010BD6FEA01014B
:109790002268936AC9B2984760B1D4F8080100F111
:1097A0000100C4F8080143F2CC11C2F200014FF0ED
:1097B00000020A7010BD00BF70B5064640F2A065F9
:1097C000C1F200054FF4117404FB00F42B194FF0A3
:1097D0000101C3F80C112A59936998472859016A65
:1097E0003046884770BD00BF38B540F2A061C1F275
:1097F00000014FF4117202FB00F28C18D4F808310A
:10980000D4F80451AB420DD08958E3188A6A19790B
:10981000904738B1D4F80801FF2814BF0130002068
:10982000C4F8080138BD00BF38B540F2A064C1F2E9
:1098300000044FF4117202FB00F2A318D3F8045194
:10984000D3F808118D4206D14FF00001C3F80C1176
:10985000A2589369984738BD10B440F2A063C1F292
:1098600000034FF4117202FB003000F58870D0F84D
:109870000031FF2B14BF5A1C0022D0F80441A24231
:109880001CBFC154C0F8002110BC7047F8B543F2AA
:109890008C14C2F2000424688568C768466807FB18
:1098A00005604518611911D2CE180B48864210D8B0
:1098B000012B04D1635D13704FF00000F8BD10461A
:1098C0001A460EF071FE4FF00000F8BD4FF01F0079
:1098D000F8BD4FF01F00F8BD0100040810B543F2B9
:1098E0002803C2F200031A8840F2A060C1F200000F
:1098F0004FF4117404FB0204F6F748FC4FF0FF31FB
:10990000C4F810124FF00003C4F8183204F588743C
:10991000F6F746FC10BD00BFF8B506464FF002034F
:10992000037044F20000C0F60000C28B4FF6FF71D6
:109930008A4221D03F4C404BA34222D203F1100374
:109940003E4DEF1A4FEA17124FF6FF7502F1010074
:1099500002F001071C46D98BA9424FD115E01C46E5
:10996000D98BA94211D002F1010203F110031C4668
:10997000D98BA94257D108E044F20004C0F6000494
:1099800003E044F20004C0F600044FF6FF702146E5
:109990004FF00D02FFF752FA4FF6FF73984208BFDF
:1099A0000020E28982421BD0A4F1100544F200009D
:1099B000C0F6000085421AD34FF6FF7029464FF0DB
:1099C0000D02FFF73BFA4FF6FF71884208BF0020F7
:1099D00034F8024C84420AD12C464FF0010201E0D7
:1099E0004FF00002607BFF2806D1327004E04FF098
:1099F000020333704FF000042046F8BD4FF0000220
:109A000002F1010203F110038242BED0002FA6D062
:109A10001C46D98BA942B8D002F1010203F1100310
:109A200082429CD1B1E702F1010203F110038242AC
:109A300095D1AAE700800008004000080F800008C8
:109A400070B5C0B005460E4620F0FF0468462146BA
:109A50004FF04002F8F790FE00AB53FA85F0314624
:109A60004FF010020EF0A0FD684621464FF48072C0
:109A7000F8F7D6FF40B070BD38B5054640F2A06497
:109A8000C1F200044FF4117303FB0044D4F81C022C
:109A9000FDF71EFB43F22800C2F200000188A94234
:109AA00006D143F22803C2F200034FF6FF721A8078
:109AB0004FF00000C4F81C0238BD00BF10B54FF0D5
:109AC0000000FBF7D9FB43F22003C2F200031C683D
:109AD00034B12068016901B188476468002CF8D16D
:109AE00010BD00BF10B50446072827D8032894BF2F
:109AF0004FF4FA73322303FB01F140F2A063C1F289
:109B0000000303EBC000C0F8141969B1FDF7B8FEFB
:109B1000002808BF012040F2A063C1F2000303EB5C
:109B2000C404C4F8100910BD40F2A061C1F20001E4
:109B300001EBC4044FF00002C4F8102910BD00BFAF
:109B400038B50446072851D840F2A063C1F200039B
:109B500003EBC000D0F8145935B340F2A061C1F254
:109B6000000101EBC402D2F81039EBB1FDF788FE19
:109B7000002808BF012040F2A061C1F2000101EB02
:109B8000C402D2F81039C01A85420CD240F2A06546
:109B9000C1F2000505EBC4014FF00005C1F81459EE
:109BA000C1F8105900E02D1A05F104054CF6CD421C
:109BB000CCF6CC42A2FB05234FEA9300032C0AD833
:109BC00000F1630348F21F51C5F2EB11A1FB033210
:109BD0004FEA521038BD00F109014CF6CD42CCF6E7
:109BE000CC42A2FB01304FEAD00038BD4FF000005C
:109BF00038BD00BF70B506466446DCF814305D6AB7
:109C0000FDF73EFE6169CA6A0AB9C86208E0801AB7
:109C100005EB850506FB05F6B04224BF0020C862AF
:109C20006369D96AD1F1010038BF002070BD00BF5F
:109C300010B540F2A063C1F200034FF4117404FBAD
:109C4000003303F58873D3F80841002C5FD15AB173
:109C50004FF0FF31C3F8001143F2CD13C2F20003FD
:109C60004FF00000187010BDD3F80021B2F1FF3F93
:109C700006D1FF294BD14FF00002C3F8002110BDDF
:109C8000FF291ED143F2CD11C2F200014FF00004B2
:109C90000C70012A10D94FF00102C3F8082140F2DC
:109CA000A063C1F200034FF4117101FB0030D0F842
:109CB0001C02FCF7CBFF10BD4FF00000C3F8000101
:109CC00010BDFE2907D143F2CD13C2F200034FF0BD
:109CD0000101197010BD43F2CD10C2F200000078EE
:109CE00048B16FEA0101C9B243F2CD10C2F20000DF
:109CF0004FF000040470FF2A05D8995402F10102C4
:109D0000C3F8002110BD4FF0FF32C3F8002110BD91
:109D100008B540F2A063C1F200034FF4117202FBD8
:109D20000030D0F80811D0F8043100F10400994255
:109D30000AD94FF00002C0F8002143F26800C2F2D5
:109D400000004068FCF782FF08BD00BFF8B565461B
:109D500043F22403C2F200031A7802F00804E7B2C7
:109D600027B1DCF8146096F8516007E012F0110F8B
:109D700006BFDCF8147097F85260002601EB8004EF
:109D800011F8203003F0070302F02002D7B23FB1F0
:109D900011F8202002F00807FAB20AB14FEA430393
:109DA00011F820704FEA9712012A08D0022A10D128
:109DB00011F82000C0F3011101FB06670BE06F6989
:109DC00097F8517011F82020C2F3011000FB0777BB
:109DD00001E04FF00007042B50D8DFE813F0C60174
:109DE00040003B002200050043F2B811C2F200011E
:109DF0000B6840F20007C0F60207FA1892F802E07A
:109E0000D0784FEA006040EA0E40527840EA0220E3
:109E1000FF5C03F104030B603843FFF79FF86860B1
:109E20002CE043F2B812C2F20002136840F20000C4
:109E3000C0F60200C11891F801C0C05C4FEA0040B2
:109E400040EA0C208978084303F1030313603F18AC
:109E50006F6013E0FFF736FAC2196A600EE043F252
:109E6000B813C2F20003186840F20001C0F6020104
:109E70000A5CBF186F6000F101001860637803F09E
:109E8000070343F22400C2F20000017801F020022F
:109E9000D7B237B1607800F00801CAB20AB14FEA10
:109EA000430367784FEA9710012807D002280ED1A4
:109EB0006178C1F3011202FB06670AE06F6997F847
:109EC00051006178C1F3011202FB000701E04FF07D
:109ED0000007042B50D8DFE813F0480140003B0096
:109EE0002200050043F2B811C2F200010B6840F2F3
:109EF0000007C0F60207FA1892F802E0D0784FEA9D
:109F0000006040EA0E40527840EA0220FF5C03F114
:109F100004030B603843FFF721F8A8602CE043F2FC
:109F2000B812C2F20002136840F20000C0F602004C
:109F3000C11891F801C0C05C4FEA004040EA0C2013
:109F40008978084303F1030313603F18AF6013E0FF
:109F5000FFF7B8F9C219AA600EE043F2B813C2F2D3
:109F60000003186840F20001C0F602010A5CBF1845
:109F7000AF6000F101001860A37803F0070343F21B
:109F80002400C2F20000017801F02002D7B237B1FC
:109F9000A07800F00801CAB20AB14FEA4303A778DB
:109FA0004FEA9710012807D002280ED1A178C1F3FB
:109FB000011202FB06670AE06F6997F85100A17869
:109FC000C1F3011202FB000701E04FF00007042B70
:109FD00050D8DFE813F0CA0040003B002200050023
:109FE00043F2B811C2F200010B6840F20007C0F65C
:109FF0000207FA1892F802E0D0784FEA006040EACF
:10A000000E40527840EA0220FA5C03F104030B6030
:10A010001043FEF7A3FFE8602CE043F2B812C2F24F
:10A020000002136840F20000C0F60200C11891F867
:10A0300001C0C05C4FEA004040EA0C208978084328
:10A0400003F1030313603F18EF6013E0FFF73AF9E1
:10A05000C219EA600EE043F2B813C2F200031868B6
:10A0600040F20001C0F602010A5CBF18EF6000F187
:10A0700001001860E37803F0070343F22400C2F202
:10A080000000017801F02002D0B230B1E17801F097
:10A090000802D0B208B14FEA4303E1784FEA9112C7
:10A0A000012A02D0022A0FD108E06E6996F8510009
:10A0B000E278C2F3011101FB000607E0E078C0F38B
:10A0C000011101FB066601E04FF00006042B4CD89D
:10A0D000DFE803F04B031318300043F2B813C2F269
:10A0E0000003186840F20001C0F602010A5CB618CD
:10A0F0002E6100F101001860F8BDFFF7E3F8821946
:10A100002A61F8BD43F2B812C2F20002136840F2AD
:10A110000000C0F60200C1184C78C05C4FEA004055
:10A1200040EA04208978084303F1030313603618DA
:10A130002E61F8BD43F2B811C2F200010B6840F283
:10A140000004C0F60204E2189678D0784FEA006066
:10A1500040EA0640527840EA0220E25C03F1040340
:10A160000B601043FEF7FAFE2861F8BD08B503281E
:10A170001ED8DFE800F0020910174CF23450C0F688
:10A18000050010F001F808BD4CF23850C0F605008B
:10A190000FF0FAFF08BD4CF24C50C0F605000FF06E
:10A1A000F3FF08BD4CF26450C0F605000FF0ECFF61
:10A1B00008BD00BF2DE9F8430546884616461F46F0
:10A1C00043F22803C2F20003B3F8009043F2345084
:10A1D000C2F20000016843F21C02C2F200021368DE
:10A1E000994201D0FFF77AFB072D6ED81F2E6CD84D
:10A1F00040F2A064C1F200044FF4117000FB094466
:10A2000043F26800C2F200004FF00001FCF7BEFA12
:10A21000217965F34711072D14BF00250125AA19DF
:10A2200062F304012171CBB22DB184F8058043445F
:10A230004FF0020001E04FF0010006F1FF3E5FFA2F
:10A240008EFE46B302463F1A0EF0010C3D5C04F14F
:10A25000040635545B1902F101020EF1FF31C9B257
:10A26000FF2934D114E0BD5C04F10406B5545B1938
:10A2700002F1010201F1FF3101F0FF01BD5CB554B3
:10A280005B1902F1010201F1FF31C9B2FF29EAD1E4
:10A2900000F1010070442218137100F10100C4F8AC
:10A2A00004014FF0FF33C4F8083121680B6A43F210
:10A2B0002800C2F2000000789847FCF795FC43F2B2
:10A2C0006800C2F20000FCF76FFBBDE8F8834FFAAC
:10A2D0008CF5002DC7D0BD5C04F10406B5545B19A4
:10A2E00002F1010201F1FF31C9B2FF29BBD1CFE771
:10A2F00000B583B040F6E573C2F200034FF00402EC
:10A300001A704FF002008DF8000043F25801C2F2BB
:10A3100000014B7A8DF801300A68ADF802204868D8
:10A32000ADF80400097A8DF806104FF007004FF0E1
:10A33000410102466B46FFF73DFF03B000BD00BF81
:10A3400008B540F6E573C2F20003197889B198B1F7
:10A35000042814D0042904D1FFF7CAFF4FF00100EC
:10A3600008BD40F6E572C2F2000210704FF0000026
:10A3700008BD4FF0000008BD4FF0000008BD4FF0D1
:10A38000000008BD38B5054642F6F074C2F200047C
:10A390002046FCF709FBF7F787FA2846FCF7ECFDA7
:10A3A00020464FF00001FCF7F1F938BD10B586B03A
:10A3B0000DF10700FFF7B0FA044618B19DF8073019
:10A3C00023B90FE044F20004C0F60004E2894FF61E
:10A3D000FF7082422BD048F20001C0F600018C428F
:10A3E00009D32AE0304821464FF00D020DF086FCDB
:10A3F000002848D0EAE74FF6FF7248F20000C0F6A6
:10A4000000006FEA0403C118C1F3001104F1100445
:10A41000E389934239D10AE004F110031C46D9893B
:10A42000914204D003F11004E389934239D148F2F8
:10A430000002C0F60002944207D344F20004C0F6C2
:10A44000000420462146F8F77FFA02A816494FF08B
:10A450000D020EF0A9F84FF0FF008DF815004FF631
:10A46000FF7002A94FF00D02FEF7E8FC4FF6FF71F6
:10A47000884212BFADF816000021ADF81610204634
:10A4800002A9FFF7DDFA06B010BD8442D5D200293B
:10A49000C2D004F11004E1899142C8D08442BBD3F8
:10A4A000CBE78442B8D3C8E7EE0F00202DE9F04F88
:10A4B00085B0884691461D46E2464FF00004264688
:10A4C0004FF0020B2DE007462846C047034670B305
:10A4D00024B9202822D0092802D11FE0012C05D15F
:10A4E0002B2B0DD02D2B0DD05C4601E0022C01D181
:10A4F0002E2B09D0A3F13002D0B2092817D805E0DD
:10A500005C4603E05C4601E04FF003040E2E05D8E4
:10A5100004A98A1902F8103C06F101062846C8472A
:10A520003846FF28CFD000F1FF370028CCD1012CCE
:10A5300012D98EB104ACA6194FF0000406F8104CE5
:10A54000684621460DF034FCDAF81410C864DAF8D5
:10A55000142082F8504005E0DAF814304FF0010082
:10A5600083F8500005B0BDE8F08F00BF10B586B08D
:10A5700040F20000C0F602003449F8F7E5F900287F
:10A580004BD1334B334A9A421DD240F20001C0F600
:10A5900002010B68B3F1FF3F42D102F104032E4ADE
:10A5A000D01A20F00302991812F0040F3FD1184678
:10A5B0008B420CD003F104021B68B3F1FF3F3ED085
:10A5C0004FF0000031E040F20000C0F6020040F21F
:10A5D0000003C0F60403984225D10DF10700FFF7F0
:10A5E0009BF90446B0B19DF80710022912D002A8C9
:10A5F00021464FF010020DF0D7FF9DF815006FF3C4
:10A6000007008DF81500204602A9FFF719FA4FF050
:10A6100001000AE04FF0010007E04FF0000004E005
:10A620004FF0000001E04FF0000006B010BD1846EA
:10A6300003F104030268B2F1FF3FB8D0C0E702F1B2
:10A6400004031068B0F1FF3FB1D0B9E7FFFF030882
:10A65000000004080000020803000408F8B50446DE
:10A66000002914BF4FF4803500250378D3B9427810
:10A67000C2B9C1B90BF04EFF43F21C06C2F200068C
:10A680003068FCF725FD4FF000033360FBF7FCFE5C
:10A690004CF28850C0F605000FF076FDFFF766FF1C
:10A6A00060B94EE051B1607840EA03214CF2985015
:10A6B000C0F6050069180FF067FD09E02678677895
:10A6C0004CF2A450C0F6050047EA06210FF05CFDED
:10A6D0006778214611F8022B05EB022540F20000B5
:10A6E000C0F602002E1840F6E875C2F20005E8191F
:10A6F0004FF080020DF058FF4FF68071CFF6FF71DA
:10A70000CB1BDAB2A818B1184FF080020DF04CFF45
:10A71000284631464FF48072F8F782F9A0B92846EE
:10A7200031464FF480720DF0E9FA80B94FF0010024
:10A730004FF000010A460B46FFF73CFD4FF00100C9
:10A74000F8BD4FF00000F8BD4FF00000F8BD4FF02D
:10A750000000F8BD2DE9F007034600284ED040F276
:10A760000022C0F6000292F8469092F8470043F2A9
:10A770003C04C2F2000494F8018092F848C02578A5
:10A7800043F25802C2F200021468177A567AD2F8DD
:10A7900004A04FF000021A7083F801909870DA70EC
:10A7A0004FF0FB0018714FF0060983F805909D717A
:10A7B00083F807804FF0040883F8088083F8098045
:10A7C00083F80AC0DD721A734FEA14255D739C7317
:10A7D000DF731E745A744FF01D029A744FF0020218
:10A7E000DA744FF0FE021A755A754FEA1A229A75FA
:10A7F00083F817A018764FF01F00587629B143F25E
:10A800003C03C2F200031A680A60BDE8F007704713
:10A8100010B14FF001020270704700BF034628B12B
:10A8200043F25802C2F200021068186043F2580165
:10A83000C2F20001087A704770B505460E4614460C
:10A840004FF000002946FEF747FF08B1F5F748FC36
:10A8500043F23803C2F200031A686260A560266002
:10A860001C6070BD08B539B143F22003C2F2000389
:10A870001A68426018601EE043F22003C2F200032F
:10A880001B6883420FD1586843F22001C2F20001D5
:10A89000086010E042685A6041605A688242F9D00C
:10A8A00013461BB907E033B14FF000015A688242EA
:10A8B000F0D01346F5E7FEF72BFE08BD08B539B119
:10A8C00043F25403C2F200031A68426018601EE0AB
:10A8D00043F25403C2F200031B6883420FD158684D
:10A8E00043F25401C2F20001086010E042685A606D
:10A8F00041605A688242F9D013461BB907E033B170
:10A900004FF000015A688242F0D01346F5E7FEF797
:10A91000FFFD08BD08B539B143F23403C2F20003AC
:10A920001A68426018601EE043F23403C2F200036A
:10A930001B6883420FD1586843F23401C2F2000110
:10A94000086010E042685A6041605A688242F9D05B
:10A9500013461BB907E033B14FF000015A68824239
:10A96000F0D01346F5E7FEF7D3FD08BD08B539B1C1
:10A9700043F21803C2F200031A68426018601EE036
:10A9800043F21803C2F200031B6883420FD15868D8
:10A9900043F21801C2F20001086010E042685A60F8
:10A9A00041605A688242F9D013461BB907E033B1BF
:10A9B0004FF000015A688242F0D01346F5E7FEF7E7
:10A9C000A7FD08BD01604360826043F26403C2F2E8
:10A9D00000031A68C2601860704700BF70B582B08B
:10A9E00006464FF000038DF807300D4601B10B709D
:10A9F00043F22000C2F20000046874B121684B6881
:10AA000043B130460DF107012A46984710B19DF831
:10AA1000070011E06468002CF0D1132E03D83046F3
:10AA2000FAF76EFC08E02DB14FF005022A704FF0E6
:10AA3000000001E04FF0000002B070BD70B582B0C0
:10AA400006464FF000038DF807300D4601B10B703C
:10AA500043F22000C2F20000046874B121688B68E0
:10AA600043B130460DF107012A46984710B19DF8D1
:10AA7000070019E06468002CF0D1132E0BD8304683
:10AA8000FAF754FC8DF8070010B13046FAF794FC41
:10AA90009DF8070008E02DB14FF005022A704FF035
:10AAA000000001E04FF0000002B070BD70B582B050
:10AAB00006464FF000038DF807300D4601B10B70CC
:10AAC00043F22000C2F20000046874B12168CB6830
:10AAD00043B130460DF107012A46984710B19DF861
:10AAE000070011E06468002CF0D1132E03D8304623
:10AAF000FAF7ECFB08E02DB14FF005022A704FF099
:10AB0000000001E04FF0000002B070BD70B582B0EF
:10AB100006464FF000038DF807300D4601B10B706B
:10AB200043F25400C2F2000004685CB121688B68F3
:10AB30002BB130460DF107012A46984758B9646891
:10AB4000002CF3D10F2E0CDC122E0AD83046F6F76B
:10AB5000CDF98DF807009DF80700003018BF0120DF
:10AB600008E02DB14FF006022A704FF0000001E01E
:10AB70004FF0000002B070BDF0B583B005460E4640
:10AB80004FF000038DF8073043F25400C2F200008A
:10AB90000468E4B14FF000072168CA681AB128467A
:10ABA00031469047F0B923689B6833B128460DF1D0
:10ABB00006010DF10702984700E038469DF807109E
:10ABC00099B9646814B10028E6D004E018B90F2DD3
:10ABD0000DDC122D0ED82846314607F073F94FF0E0
:10ABE000000009E04FF0000006E0084604E04FF0E6
:10ABF000060001E04FF0060003B0F0BD70B582B072
:10AC000005460E464FF000038DF8073012B1194685
:10AC1000FFF7B2FF43F25400C2F2000004686CB1C7
:10AC200021684B68284631460DF10702984710B15C
:10AC30009DF8070012E06468002CF1D10F2D08DCAC
:10AC4000122D09D828463146F6F772F94FF0000068
:10AC500004E04FF0060001E04FF0060002B070BDC6
:10AC600008B54FF0000001464FF00102FFF7C6FFA4
:10AC700008BD00BF70B582B005460E464FF0000318
:10AC80008DF8073043F23400C2F2000004689CB132
:10AC900021684B68284669460DF10702984728B19C
:10ACA0000EB1009830609DF8070014E064681CB194
:10ACB0009DF80720002AEBD0012D07D84EB1284679
:10ACC000F7F71AF830604FF0000004E04FF00F0083
:10ACD00001E04FF0000002B070BD00BF70B582B05F
:10ACE00005460E464FF000038DF8073043F218007A
:10ACF000C2F20000046884B121684B6828463146DE
:10AD00000DF10702984710B19DF8070010E0646844
:10AD10001CB19DF80720002AEED03DB94FF000008D
:10AD20003146F6F7C5FE4FF0000001E04FF00E008F
:10AD300002B070BD70B582B005460E464FF00003FC
:10AD40008DF8073043F21800C2F200000468A4B185
:10AD500021688B685BB1284669460DF10702984768
:10AD600028B10EB1009830609DF8070014E06468C7
:10AD70001CB19DF80720002AEAD045B956B14FF022
:10AD80000000F6F7DDFF30604FF0000004E04FF008
:10AD9000060001E04FF0000002B070BD00000000AE
:10ADA0002DE9F04F2DED048B8BB0834692469142F6
:10ADB00064D289464FF000089FED379A9FED328BA1
:10ADC000DFED369A32A7D7E900674FF000044FF065
:10ADD0000005C3F6E0758DED019ABBF1020F05D1B8
:10ADE0005FFA89F001A9FFF7A5FF04E05FFA89F097
:10ADF00001A9FFF73FFF08EB48030AAAD01800F8A3
:10AE0000209C01980CF034FA53EC182B0CF0A8FDA0
:10AE100008B1CDED019A01980CF02AFA32463B4672
:10AE20000CF0C4FB22462B460CF07CFA0CF0E6F941
:10AE300081B208EB48030AAAD31803F81E1C4FEA94
:10AE4000112003F81F0C08F10108B8F10A0F06D011
:10AE50000AF1FF3149450DD1B8F1000F0AD008EBD6
:10AE600048024FF007005946D2B202ABFFF7A2F9F1
:10AE70004FF0000809F10109CA45ACD80BB0BDEC90
:10AE8000048BBDE8F08F00BF9831CB64FE0F70409B
:10AE90000000000000E06F4000000000F37F8043EE
:10AEA0002DE9F04F9FB040F6C410FCF765F84FF065
:10AEB00002004FF0000143F23C03C2F20003DA78D3
:10AEC000FFF76EFF4FF0010002904FF0000BDA46E3
:10AED000D94607464CF6CD41CCF6CC4103914FF014
:10AEE0007D00FCF749F88DF83790C8464E464C4631
:10AEF00013E045F0800504F10804E4B216A9725C81
:10AF0000AA4202D016ABF554B84606F101069DF8E8
:10AF10003750002D50D1202E4ED020460DF1370154
:10AF2000FFF75CFD051C18BF012504F10102D0B23A
:10AF30000DF13701FFF752FD10B145F00205EDB2FA
:10AF400004F10203D8B20DF13701FFF747FD08B154
:10AF500045F0040504F10300C0B20DF13701FFF71D
:10AF60003DFD08B145F0080504F10401C8B20DF13A
:10AF70003701FFF733FD08B145F0100504F1050274
:10AF8000D0B20DF13701FFF729FD08B145F02005DA
:10AF900004F10603D8B20DF13701FFF71FFD08B128
:10AFA00045F0400504F10700C0B20DF13701FFF78D
:10AFB00015FD00289DD19EE7B8F1000F02D1BAF12E
:10AFC000000F0CD14FF002004946F2B216ABFFF76A
:10AFD000F1F84FF03200FBF7CFFF019701E0CDF819
:10AFE00004908DF83790C8464E464C4613E045F025
:10AFF000800504F10804E4B20EA8315CA94202D035
:10B000000EAAB554B84606F101069DF83750002D3A
:10B0100050D1202E4ED020460DF13701FFF776FD9E
:10B02000051C18BF012504F10100C0B20DF1370164
:10B03000FFF76CFD10B145F00201CDB204F1020240
:10B04000D0B20DF13701FFF761FD08B145F00405FD
:10B0500004F10303D8B20DF13701FFF757FD08B132
:10B0600045F0080504F10400C0B20DF13701FFF707
:10B070004DFD08B145F0100504F10501C8B20DF110
:10B080003701FFF743FD08B145F0200504F1060242
:10B09000D0B20DF13701FFF739FD08B145F0400599
:10B0A00004F10703D8B20DF13701FFF72FFD002897
:10B0B0009DD19EE7B8F1000F02D1BAF1010F0AD17C
:10B0C00048464946F2B20EABFFF774F84FF0320033
:10B0D000FBF752FF019743F23C03C2F200039A7858
:10B0E000B2B1039EA6FB0A044FEA141000EB8001E4
:10B0F000BAEB810F0CD138464946FFF751FE4FF0AD
:10B100003200FBF739FFBBF1000F40F0B88003E0DD
:10B11000BBF1000F40F09C8005A849464FF020028B
:10B120000DF066FA43F23C06C2F20006B478ACB306
:10B130004D466FEA0900011901F0010209F0070309
:10B1400007FA03F69DF8140046EA00018DF8141082
:10B1500005F10105A542C0F2B3801FE01EAB03EB71
:10B16000D50605F0070007FA00F216F8641C42EA5B
:10B17000010306F8643C05F101051EA800EBD502A9
:10B1800005F0070107FA01F312F8646C43EA0600C0
:10B1900002F8640C05F10105A542DFDB4FF0070062
:10B1A0004FF011014FF01E0205ABFFF703F84FF00F
:10B1B0003200FBF7E1FE05A849464FF020020DF0F2
:10B1C00017FA43F23C04C2F20004E578A5B34B46FB
:10B1D0006FEA0902511901F0010609F0070007FAA8
:10B1E00000F49DF8142044EA02018DF8141003F1D4
:10B1F00001039D4250DC1FE01EAC04EBD30203F0C0
:10B20000070007FA00F612F8641C46EA010402F887
:10B21000644C03F101031EAA02EBD30403F0070000
:10B2200007FA00F614F8641C46EA010204F8642CDC
:10B2300003F101039D42DFDC4FF007004FF01201E4
:10B240004FF01E0205ABFEF7B5FF4FF0060B16E000
:10B25000019AA2B9BBF1020F11D1029D7DB943F24F
:10B260003C03C2F20003DA784AB14FF002004946CB
:10B27000FFF796FD4FF03200FBF77EFE0297BAF122
:10B28000000F06D10BF1FF3BCDF808904FF0280AD4
:10B2900025E60AF1FF3A22E6002EADD01EAE06EBFF
:10B2A000D30403F0070007FA00F214F8641C42EA22
:10B2B000010604F8646C03F101039D429CDCBBE7CA
:10B2C000002A3FF44BAF1EAA02EBD50305F0070698
:10B2D00007FA06F013F8641C40EA010203F8642C34
:10B2E00005F10105A542FFF639AF57E72DE9F04F0B
:10B2F0002DED028B87B008EE100A0C4617469946D2
:10B30000129E1399B5EEC08AF1EE10FA54BF0025D3
:10B310000125A84604F1FF33D8B2082807D8092A26
:10B3200005D8A24601F1FF32944205D808E001F1A8
:10B33000FF339C4240F2CD8001F1FF34E4B2C8E01B
:10B3400018EE100A0CF068FB48B930464FF03F0188
:10B3500022460DF04DF94FF000013155C4E018EED2
:10B36000100A0CF0C5FB06EE900AF2EE047AF4EE39
:10B37000E76AF1EE10FA0DDB4FF00100B0EE677AEC
:10B3800000F1010067EE877AF4EEE76AF1EE10FA59
:10B39000F6DA03E04FF00100F2EE047A2146431999
:10B3A000A34200F39680C0EB040EC5EB0E0202F13F
:10B3B000FF3E4DF2840AC0F6050ADFED9C4AF6EE28
:10B3C000003AB2EE044AC0EB040CC5EB0C0303F0E8
:10B3D000010BBEF1000F00F38F808AE0BEF1000F79
:10B3E00004DDBE45B4BF72463A4601E04FF00002AC
:10B3F0005AF8223003EE103AB8EE430A20EE027AF1
:10B40000B4EEE47AF1EE10FA48BF37EE237ABDEEDF
:10B41000C73A13EE10CABCFBF3FB06EE10BAB8EE47
:10B42000C65AB4EEE75AF1EE10FA0DDB00F1010C4A
:10B4300087EE006A67EE847A0EF1FF3E6046BEF149
:10B44000000200F3C380BEE013EE105AB5FBF3F424
:10B4500003FB14542CB916EE107A002F08BF4FF0DE
:10B460000008B9F1000F07D0C8EB0103181A002A31
:10B4700018BF0138831A01E04FF0000301F1010108
:10B48000B8F1000F04D04CF2B057C0F6050703E046
:10B490004AF28427C0F6050722B14CF2B450C0F638
:10B4A000050003E04AF28420C0F605004CF2C855BE
:10B4B000C0F60505009501978DED026A0390049290
:10B4C000059430464CF2B852C0F605020CF05AFC16
:10B4D0000AE03046002D0CBF2B212D2122460DF015
:10B4E00087F84FF00000305507B0BDEC028BBDE887
:10B4F000F08F4FF0000203E0BE45B4BF72463A46FB
:10B500005AF8223000EE103AB8EE405A65EE260A9C
:10B51000F4EEE40AF1EE10FA48BF70EEA30ABDEEB5
:10B52000E03A13EE10CABCFBF3FC06EE10CAF8EECC
:10B53000C65AF4EEE75AF1EE10FA85DB00F101008D
:10B5400080EE852A67EE847A0EF1FF3E4219914221
:10B55000BFDBBBF1000F3FF441AFBEF1000F02DCD7
:10B560004FF0000203E0BE45B4BF72463A465AF8B7
:10B57000223001EE103AF8EE411A21EE822AB4EEA2
:10B58000E42AF1EE10FA48BF32EE232ABDEEC23AA9
:10B5900013EE10BABBFBF3FB06EE10BAF8EEC62AA8
:10B5A000F4EEE72AF1EE10FAFFF64EAF00F10100DB
:10B5B00082EE212A67EE847A0EF1FF3E431999420A
:10B5C000BFF60CAF85E74FF0000202E0BA42A8BF19
:10B5D0003A465AF8223006EE903AF8EE660A20EE25
:10B5E000861AB4EEE41AF1EE10FA48BF31EE231ACF
:10B5F000BDEEC13A13EE10BABBFBF3FB06EE10BA78
:10B60000F8EEC65AF4EEE75AF1EE10FAFFF61CAF68
:10B610000CF1010081EE202A67EE847A0EF1FF3EE4
:10B6200042199142BFF6DAAE53E700BF0000004B6B
:10B63000F8B505460F46F4F7A9FD064640F2A062AC
:10B64000C1F200024FF4117303FB05F014181158F6
:10B6500011B18A682846904784F820724FF000059F
:10B66000C4F81052C4F81452C4F80451C4F8085174
:10B670003046F4F795FD04F5097029464FF00802AD
:10B68000F4F73EFDF8BD00BF70B588B0054640F246
:10B69000A064C1F200044FF4117303FB004494F85A
:10B6A000200200284AD043F22801C2F200010A8891
:10B6B0004FF6FF76B24204D0D0B24FF00401FFF74C
:10B6C000B7FF28464FF00001FFF7B2FF43F228060C
:10B6D000C2F2000635804CF2D450C0F605004FF09F
:10B6E000070141F2F902C0F60502FBF707FCC4F8B6
:10B6F0001C02246830784FF0010300934FF00002E1
:10B70000019249F21971C0F60401029149F61153F0
:10B71000C0F60403039349F63141C0F604010491D5
:10B7200049F67923C0F604030593069264684FF442
:10B7300016514FF00803A047FEF7D0F808B070BDCF
:10B74000704700BF08B5B0F1FF3F04D040B90246D2
:10B75000F6F724FB08BD4FF000000246F6F71EFB8B
:10B7600008BD00BF38B506F0A1FB43F24003C2F2AA
:10B7700000034FF001021A704FF000042546E0B2BA
:10B7800029462A46FFF73AFA40B904F10104E0B22B
:10B7900029462A46FFF732FA002867D04FF0FF30DB
:10B7A0004FF00001FFF7CEFF4FF000004FF0000117
:10B7B000FFF794FA43F21801C2F200010C6834B1A9
:10B7C0002368DA6802B190476468002CF8D143F22C
:10B7D0003800C2F2000004683CB121680B680BB16C
:10B7E000A06898476468002CF7D1FAF793FAFEF73F
:10B7F00065F940F2A062C1F2000292F8200204282A
:10B8000006D028B14FF000004FF00401FFF710FF01
:10B8100040F2A061C1F2000191F86434042B06D01B
:10B820002BB14FF001004FF00401FFF701FF40F290
:10B83000A062C1F2000292F8A806042806D028B13E
:10B840004FF002004FF00401FFF7F2FE40F2A0615A
:10B85000C1F2000191F8EC38042B06D02BB14FF067
:10B8600003004FF00401FFF7E3FE38BD04F10104CB
:10B87000B4F5807F83D191E738B5054643F21C04C7
:10B88000C2F200042068FBF723FC4FF000032360A2
:10B890008DB14CF2E450C0F605004FF007014BF6B5
:10B8A000BD12C0F60402FBF729FB43F22C02C2F2E0
:10B8B0000002106038BD43F22C04C2F2000420687C
:10B8C000FBF706FC4FF00000206040F6E572C2F284
:10B8D00000021070FAF7D8FDFFF744FF0AF01AFED5
:10B8E00043F22801C2F2000108884FF6FF73984224
:10B8F00004D0C0B24FF00401FFF79AFE38BD00BF7C
:10B9000070B543F26800C2F200004CF2F451C0F688
:10B910000501FAF723FF43F22803C2F200034FF6B2
:10B92000FF721A8040F2A064C1F200044FF00406D6
:10B9300084F820624FF00005C4F81C522846FBF73B
:10B94000F7F8206084F86464C4F860544FF0010094
:10B95000FBF7EEF8C4F8440284F8A866C4F8A456CD
:10B960004FF00200FBF7E4F8C4F8880484F8EC68B0
:10B97000C4F8E8584FF00300FBF7DAF8C4F8CC0637
:10B9800042F6F070C2F200004CF20061C0F6050110
:10B99000FAF7E4FE43F24400C2F200004CF66811EC
:10B9A000C0F605012A462B46FFF70CF8FDF7B0FD5F
:10B9B0004FF00100FFF760FF70BD00BF2DE9F04FB1
:10B9C0002DED048BABB01CAF26AC4BF61065C0F66A
:10B9D000050595E80F0084E80F00A76049F29D4334
:10B9E000C0F60403E36020462AA9F7F711FF22AE50
:10B9F00095E80F0086E80F00B76049F2B940C0F63D
:10BA00000400F06030462146F7F702FF4FF00004D3
:10BA10001B9442F6F070C2F200002146FAF7B6FE1F
:10BA200043F25801C2F200010C72FFF79BFE0AF0CC
:10BA300071FD4FF00200FFF727FE43F2B812C2F289
:10BA4000000215680DBB0EF08FFBF0B9F5F72EFE66
:10BA500010F0C20F19D14FF00300FEF787FB4FF42F
:10BA60007A754FF032063046FBF786FAF5F71CFF81
:10BA700005F1FF343046FBF77FFAF5F715FF651E39
:10BA8000F1D14FF00000FEF771FB43F22403C2F244
:10BA900000034FF000041C604FF00100187040F2EA
:10BAA000A066C1F2000606F515652846214642F655
:10BAB00054220CF09DFD40F6E870C2F200002146D1
:10BAC0004FF400520CF094FD06F5116021464FF042
:10BAD00040020CF08DFD43F29000C2F200002146BE
:10BAE0004FF0FC020CF084FD21954FF00A01C6F8DE
:10BAF000741920462946FDF76DFC43F29012C2F2FC
:10BB00000002146043F23003C2F200031C6043F2EF
:10BB1000B815C2F200054FF030042C6040F200046A
:10BB2000C0F6020494F82F0000F1010094F82E10E2
:10BB300000EB0122101943F28C13C2F200031860CB
:10BB4000FBF79EFE0C902B68E15CFF2930D143F29D
:10BB50005800C2F200004FF0010101720360219A07
:10BB6000106A18B100F1010052F8203043F2580178
:10BB7000C2F200014B604FF0FF024A7243F22C0008
:10BB8000C2F200004FF00003036043F22801C2F24A
:10BB90000001088840F2A062C1F200024FF4117364
:10BBA00003FB0021D1F81C02FBF750F805F071BA35
:10BBB00006F05AF94FF000070A97B946BB4601E074
:10BBC0004FF0000BBBF1000F05D14FF00000FEF766
:10BBD000D9FB4FF0640B0BF1FF3B43F2B816C2F2F6
:10BBE0000006356840F20004C0F60204615D40F6CC
:10BBF000E572C2F200021378002B00F09180FE295A
:10BC000049D043F29810C2F200000068002839D0F1
:10BC1000854243D043F29817C2F20007786888B390
:10BC200085423ED043F29816C2F20006B06848B38F
:10BC3000854239D043F29814C2F20004E06808B398
:10BC4000854234D043F29812C2F200021069C8B1A2
:10BC500085422FD043F29810C2F20000406988B1AB
:10BC600085422AD043F29817C2F20007B86948B15A
:10BC7000854225D043F29816C2F20006F06908B159
:10BC8000854220D0022B14BF00200120032B1CD0A2
:10BC9000002845D019E04FF0000016E04FF00000FA
:10BCA00013E04FF0000010E04FF000000DE04FF007
:10BCB00000000AE04FF0000007E04FF0000004E051
:10BCC0004FF0000001E04FF0000040F6E574C2F2D2
:10BCD00000044FF003032370ADB28DF844008DF8DB
:10BCE0004510ADF84850ADF846504FF000018DF8C2
:10BCF0004A104FF007004FF04101024611ABFEF72A
:10BD000059FA2278032A0BD14FF0000740F6E57666
:10BD1000C2F200063846FEF735FB30780328F9D02A
:10BD200043F22404C2F20004237803F0E7056FF322
:10BD30004515257043F2B811C2F200010A68099254
:10BD400043F2B815C2F2000540F20006C0F6020642
:10BD500043F22407C2F200074CF68448C0F60508F7
:10BD60002868345C00F1010028603B7813F0010F73
:10BD70000ED109F1010940F2FF31894508D943F29A
:10BD80005801C2F200014FF036020A7205F01BB9E9
:10BD90000DF1700C20464146FDF7D8FF4BF624729A
:10BDA000C0F6050252F824304CF2287AC0F6050A93
:10BDB00043F0010000472B68F15C0B9103F1010394
:10BDC0002B600F2905F2F7800DF1700C08465146E3
:10BDD000FDF7BCFF4CF64430C0F605000B9A50F856
:10BDE0002230E5E72B68F15C0B9103F101032B6036
:10BDF000102902D90C4605F0DFB80DF1700C0B9834
:10BE00004CF2AC71C0F60501FDF7A0FF4CF2687072
:10BE1000C0F605000B9A50F82230C9E72B68F15C98
:10BE20000B9103F101032B600F2902D90C4605F099
:10BE3000C3B80DF1700C0B984CF62801C0F6050143
:10BE4000FDF784FF4CF66800C0F605000B9A50F829
:10BE50002230ADE72B68F15C0B9103F101032B60FD
:10BE60002F2902D90C4605F0A7B80DF1700C0B98DC
:10BE70004CF6A801C0F60501FDF768FF4CF67410FA
:10BE8000C0F605000B9A50F8223091E72B68F15C60
:10BE90000B9103F101032B603B2902D90C4605F0FD
:10BEA0008BB80DF1700C0B984BF63461C0F60501A0
:10BEB000FDF74CFF4CF23860C0F605000B9A50F8C5
:10BEC000223075E72B68F15C0B9103F101032B60C5
:10BED0003F2902D90C4605F06FB80DF1700C0B9894
:10BEE0004CF68431C0F60501FDF730FF4CF23440CA
:10BEF000C0F605000B9A50F8223059E72B68F15C28
:10BF00000B9103F101032B60432902D90C4605F084
:10BF100053B80DF1700C0B984CF22431C0F60501AA
:10BF2000FDF714FF4CF63420C0F605000B9A50F8CC
:10BF300022303DE7219F97F846600DF1700CFDF728
:10BF4000ABF9219C351894F8501001F001002A1823
:10BF50001C9284F84720FF2A94BF0022012284F813
:10BF600050202FE6219B93F846700DF1700CFDF7E1
:10BF700093F93E181C96219C84F84760FF2E94BFCD
:10BF80000026012684F850601CE60DF1700CFDF7C8
:10BF900083F930B1219991F84700051C18BF01259C
:10BFA00001E04FF00005219A82F847500AE60DF1B2
:10BFB000700CFDF771F9219B93F84770384083F8B6
:10BFC0004700FFE51D9EA6F1FB061C961AE11D9D8C
:10BFD000A5F1FB051C95A2E11D99A1F1FB011C91A6
:10BFE000D3E11D98A0F1FB001C9072E21D9AA2F112
:10BFF000FB021C924FF002031B9308E21D9EA6F168
:10C00000FB061C961E9D1B9533E21D99A1F1FB01B9
:10C010001C912BE11D98A0F1FB001C90B0E21D9A31
:10C02000A2F1FB021C92ECE21D9BA3F1FB031C930B
:10C030001E9E1B9629E31D9DA5F1FB051C951E99CF
:10C040001B914FF000008DF86A0000F001BC1D9AB2
:10C05000A2F1FB021C921E9B1B934FF001068DF870
:10C060006A60F5E31D9DA5F1FB051C9500F085BCFC
:10C070001D9CA4F1FB041C9400F0DABC9DF8740034
:10C080004FF00101FEF778FD8DF86B0000283FF4BA
:10C0900099AD43F25801C2F20001087204F093BF57
:10C0A0001D981C904FF001038DF86A301E46219AAE
:10C0B00092F847502B4205D09DF870003146FEF7AC
:10C0C0005BFD68B99DF86A304FEA43018DF86A104C
:10C0D0001C9800F101001C9011F0FE03E7D10CE068
:10C0E0009DF86A60012E08D19DF86B2043F2580537
:10C0F000C2F200052A7204F066BF0DF1700CFDF764
:10C10000CBF85FE59DF8740005F0A0FE5AE50DF14F
:10C11000700CFDF7C1F81C9043F2B810C2F2000099
:10C1200003681C9903EB41060660FDF7CBF81C90F1
:10C1300001F0F6BE43F22401C2F20001087810F0CB
:10C14000280F06D01D9BB3F5005F34BF00230123E9
:10C1500004E01D9BFA2B94BF0023012343B143F25B
:10C160005801C2F200014FF01300087204F02BBF17
:10C1700040F6E876C2F200061D9AB55C1C95CBE746
:10C18000219B93F852601C96C6E7219A92F8505072
:10C190001C95C1E74FF0000914E50DF1700CFDF797
:10C1A0007BF81C90219F97F847101B91FDF72AF907
:10C1B00087F8470006E5219C94F8470094F846105C
:10C1C000FDF720F984F85000FCE40DF1700CFDF748
:10C1D0008BF81E9D40F6E872C2F20002505D1D9B76
:10C1E00020EA03015155EDE443F29000C2F2000051
:10C1F0004FF000014FF0FB020CF0FAF9E2E44FF0CF
:10C2000000061C960DF1A80C1CF8385DFDF744F8EB
:10C210000146284608F0F8FB8DF86B0000283FF433
:10C22000D1AC43F25802C2F20002107204F0CBBE4D
:10C2300007F028F9C6E407F02DF98DF86B00002807
:10C240003FF4C0AC43F25803C2F20003187204F08A
:10C25000BABE43F28C17C2F200073C681D98201842
:10C2600007F004F9AEE44FF000011C911C9E40F26F
:10C27000A065C1F200054FF4117303FB065292F85A
:10C28000200203283FD140F2A067C1F2000703FB60
:10C2900006F606F588757919BB1903F104034FF00A
:10C2A0000000D1F80021FE2A94BF541C0024D1F8CC
:10C2B0000461B44214BF0024012464F30000B242BC
:10C2C00014BF0022012262F34100D3F80041FE2C8A
:10C2D00094BF013400240DF1A80C4CF8384DD3F86C
:10C2E0000471BC4214BF0024012464F38200D3F81B
:10C2F0000851D5F1010138BF002161F3C300C0B27C
:10C30000FCF7B2FF5EE443F25801C2F200014FF0C5
:10C3100048060E7204F057BE4FF000031C931C98A1
:10C3200040F2A062C1F200024FF4117606FB002534
:10C3300095F8201203291CD140F2A064C1F2000438
:10C3400006FB0047D7F81022D7F81462951BB5F505
:10C35000807F88BF05F580751C951C99FF2984BFD7
:10C36000FF211C910DF1A80C1CF8380DFCF77CFF87
:10C3700028E443F25803C2F200034FF04800187259
:10C3800004F021BE4FF000031C931C9840F2A06201
:10C39000C1F200024FF4117606FB002595F8201239
:10C3A000032925D140F2A064C1F2000406FB004736
:10C3B00007F58876D6F80021D6F80451511BB1F55F
:10C3C000807F88BF01F580711C910DF1700CFCF726
:10C3D00063FF8DF86A001C9B984238BF1C90D6F80A
:10C3E00004011C9C2718FAB2C6F80421FFF7EABB27
:10C3F00043F25803C2F200034FF04800187204F0F1
:10C40000E2BD4FF000061C964FF002051B951C9BE9
:10C4100040F2A060C1F200004FF4117101FB030271
:10C4200092F82062032E16D140F2A064C1F20004FB
:10C4300001FB03470DF1700C1B9849F21941C0F63E
:10C44000040149F22D42C0F6040207F58873FCF797
:10C450005DFFFFF7B7BB43F25805C2F200054FF08E
:10C4600048032B7204F0AFBD4FF000001C901D99E3
:10C470001B911C9E40F2A062C1F200024FF41175A4
:10C4800005FB062393F82002032816D140F2A0648E
:10C49000C1F2000405FB06470DF1700C1B9849F230
:10C4A0001941C0F6040149F22D42C0F6040207F515
:10C4B0008873FDF7FBFFFFF785BB43F25801C2F21B
:10C4C00000014FF048060E7204F07DBD4FF00002EF
:10C4D0001C921C9D40F2A063C1F200034FF4117046
:10C4E00000FB053191F82062032E3DD140F2A0649B
:10C4F000C1F2000400FB054707F588740DF1700CCC
:10C50000FCF7CAFE8DF86A00D4F804611C964FF05F
:10C5100000031B93D4F800113346B14207D0A55D48
:10C52000854219D04FF001024FF000050CE04FF0AA
:10C53000FF001B9010E002F10106E75C874202D188
:10C540001C931B9208E03246FF2B14BF01332B468D
:10C550008B42F0D11C93EAE70DF1700C9DF86C0052
:10C56000FCF782FEFFF72EBB43F25805C2F200052E
:10C570004FF048022A7204F026BD4FF000011C91D2
:10C580001C9B40F2A065C1F200054FF4117606FB3A
:10C59000035292F82002032827D140F2A064C1F28E
:10C5A000000406FB034707F58876D7F81452D7F83E
:10C5B0001022954212D00DF1700CFCF76DFE43195C
:10C5C000DCB21C940DF1700C305DFCF74DFE4FF0A9
:10C5D0000007219E86F85070FFF7F4BA4FF0010073
:10C5E000219981F85000FFF7EDBA43F25801C2F2E9
:10C5F00000014FF048030B7204F0E5BC4FF000055A
:10C600001C951C9840F2A062C1F200024FF4117117
:10C6100001FB002393F82062032E28D140F2A0648E
:10C62000C1F2000401FB004707F58876D6F8041133
:10C63000D6F80021914213D00DF1700C705CFCF71C
:10C6400013FED6F80401FF2814BF01300020C6F8FD
:10C6500004014FF00004219F87F85040FFF7B2BA61
:10C660004FF00105219B83F85050FFF7ABBA43F21E
:10C670005805C2F200054FF04800287204F0A3BC30
:10C680004FF000061C961D991B9143F28C12C2F2CA
:10C690000002D2F800A0DDF86C800AEB080540F239
:10C6A0000003C0F604039D4208D943F25801C2F2C8
:10C6B00000014FF01F050D7204F085BC1C98032883
:10C6C00008D943F25800C2F200004FF0370303725A
:10C6D00004F079BCEE780D2E08D943F25806C2F268
:10C6E00000064FF03702327204F06DBC40F2A062D7
:10C6F000C1F200024FF4117101FB002393F82002F4
:10C7000038B11AF8086026B113E03846FDF73AFE52
:10C7100007E04CF24F364FF09607CDF82CB0DDF81D
:10C7200030B0FBF7ADF8CBEB0002B242EDD9DDF84B
:10C730002CB01AF80830032B7BD8DFE803F002088E
:10C74000192A9DF87000FEF79FFFFFF73BBA9DF88E
:10C750007000294608F07AF900287FF433AA43F2E2
:10C760005801C2F200014FF037050D7204F02BBCE6
:10C770009DF87000294606F007FE00287FF422AAE3
:10C7800043F25800C2F200004FF03703037204F086
:10C790001ABC9DF87060AF7830464FF00301FEF789
:10C7A00047FF4FF4117101FB06F040F2A062C1F2A5
:10C7B0000002105800283FF405AA4BF62063C0F68B
:10C7C000050307EB470703EB070EED784CF2F0711A
:10C7D000C0F6050151F82510DA5D9EF801309EF88B
:10C7E000027000974FF00005019549F2E977C0F615
:10C7F0000407029749F62907C0F60407039749F68C
:10C800005907C0F60407049749F67927C0F60407CC
:10C810000597069545683046A84700287FF4D2A9B9
:10C8200043F25806C2F200064FF03702327204F0AB
:10C83000CABB9DF870004FF00401FEF7F9FEFFF748
:10C84000C1B94FF000061C961D9A1B928DF86A60C4
:10C850001C9D40F2A066C1F200064FF4117000FB6F
:10C86000056292F82032032B71D140F2A064C1F22C
:10C87000000400FB054707F5887843F28C16C2F2E6
:10C8800000063068219A936BC118C35CFF2B53D00C
:10C890000B914FF0010409944FF0000A0B9F7E7832
:10C8A00006EB032043F28C12C2F2000213681D183B
:10C8B000D8F804111C919DF86A401CB11F5C05F169
:10C8C000010500E0574605F1FF349DF86A600EB19E
:10C8D00037B901E0607818B91C9EC8F804612EE0F1
:10C8E0001C9BD8F800219A4218D014F8016F18F850
:10C8F00003501B9939B930460BF0E8F9C6B2284607
:10C900000BF0E4F9C5B2AE4208D11C98FF2814BF61
:10C91000013050461C9007F1FF37D6E7099C04F11F
:10C92000010409940B9A12F8023F0B92FF2BB5D128
:10C930004FF00001099102E04FF0000509950DF15B
:10C94000700C099DE8B2FCF78FFCFFF73BB943F28E
:10C950005801C2F200014FF048050D7204F033BBDC
:10C960004FF000001C901E9B1B934FF001018DF8AF
:10C970006A106DE74FF000001C901C9B40F2A06213
:10C98000C1F200024FF4117101FB032696F8205208
:10C99000032D31D140F2A067C1F2000701FB0374FF
:10C9A00004F588760DF1700CFCF776FC8DF86A00C2
:10C9B0004FF000021C92D6F80431D6F80071BB4249
:10C9C00012D0F15C81420FD14FF00004FF2B14BF55
:10C9D00001332346BB4202D1C6F8043104E0F55CC2
:10C9E0008542F3D0C6F804310DF1700C4FF0000011
:10C9F000FCF73AFCFFF7E6B843F25800C2F2000039
:10CA00004FF04803037204F0DEBAFAF739FF0C9EC8
:10CA1000801B0DF1700C4CF24F3290428CBF002005
:10CA20000120FCF721FCFFF7CDB84FF000001C906F
:10CA30001C9B40F2A067C1F200074FF4117101FB8B
:10CA4000037494F82052032D7FF4BCA840F2A06632
:10CA5000C1F2000601FB036000F10402D0F80831C6
:10CA6000D2F8007107F10107BB4238BF03F58073AC
:10CA7000D91BFF2934BF0C46FF240DF1700CE0B226
:10CA8000FCF7F2FBFFF79EB81D9D40F6E876C2F278
:10CA90000006705D00F1FF327255FFF793B843F264
:10CAA0002403C2F20003197811F0280F06D01D9D4F
:10CAB000B5F5005F34BF0025012504E01D9DFA2D6A
:10CAC00094BF0025012545B143F25806C2F2000685
:10CAD0004FF01300307204F076BA1D9E40F6E870F5
:10CAE000C2F20000825D02F1FF33D9B28155002904
:10CAF0003FF468A81E9D1C9501F012BA43F224026F
:10CB0000C2F20002137813F0280F06D01D99B1F578
:10CB1000005F34BF0021012104E01D99FA2994BF70
:10CB20000021012141B143F25801C2F200014FF04E
:10CB300013050D7204F047BA1D9D40F6E876C2F267
:10CB40000006705D00F1FF32D3B27355002B42F046
:10CB50000687FFF737B843F22406C2F200063078A2
:10CB600010F0280F06D01D9AB2F5005F34BF0022E6
:10CB7000012204E01D9AFA2A94BF0022012242B148
:10CB800043F25805C2F200054FF013022A7204F076
:10CB90001ABA1D9D40F6E871C2F200014B5D03F127
:10CBA000FF36F0B24855002802F0D986FFF70AB8E0
:10CBB000219F97F8514004F1FF3187F85110FFF79A
:10CBC00001B8219B93F8476006F1FF3083F84700D6
:10CBD000FEF7F8BF219DE86C0AF08AFF219AD06425
:10CBE000FEF7F0BF219F97ED137AD7ED127A37EE5B
:10CBF000270A87ED130A219DE86C0AF0EDFE30B19B
:10CC00004FF00202219E86F85020FEF7DBBF2198EC
:10CC1000C06C0AF0F1FE30B14FF00101219B83F8A6
:10CC20005010FEF7CFBF4FF00007219C84F85070E2
:10CC3000FEF7C8BF9DF87400219901F14C01FEF781
:10CC400019F88DF86B0000283EF4BCAF43F2580190
:10CC5000C2F20001087204F0B6B99DF87400219B7D
:10CC6000D96CFEF73BF88DF86B0000283EF4AAAFB4
:10CC700043F25806C2F20006307204F0A4B9219CB7
:10CC8000E06C0AF0B9FE20B92198806C0AF0B4FE7D
:10CC900030B14FF00306219C84F85060FEF792BF3C
:10CCA000219DD5ED138A95ED128A78EEC80A10EE13
:10CCB000900A0AF01DFF09EE100A18EE900A18EE0D
:10CCC000101A0AF0AFFE01464FF07E500AF0AAFE9D
:10CCD0009FEDCF1A01EE900A21EE812AB4EEC29A9E
:10CCE000F1EE10FA06D84FF00001219B83F85010A6
:10CCF000FEF768BF219FD7ED132A97ED123AF4EEA5
:10CD0000C32AF1EE10FA05DD4FF0010287F850203A
:10CD1000FEF758BFF4EEC32AF1EE10FA4CBF022220
:10CD2000032287F85020FEF74DBF2198D0ED133A2B
:10CD3000B7EE004A73EEC44AC0ED134A219FF86C67
:10CD40000AF05AFE30B14FF00306219D85F850607D
:10CD5000FEF738BF219CD4ED138A9FEDAE8A38EEE2
:10CD6000C89A19EE100A0AF0C3FE09EE100A18EE6E
:10CD7000900A18EE101A0AF055FE01464FF07E5048
:10CD80000AF050FEDFEDA23A04EE100A64EE234AE8
:10CD9000B4EEE49AF1EE10FA22D9219890ED138ABC
:10CDA000DFED9C8A38EE285A15EE100A0AF0A0FE34
:10CDB00008EE900A18EE100A6FF052510AF032FE97
:10CDC00001464FF07E500AF02DFEDFED915A06EE3F
:10CDD000100A66EE256AF4EEE68AF1EE10FA06D83D
:10CDE0004FF00404219880F85040FEF7EBBE219EDE
:10CDF000F56C28460AF07CFE08EE100A28464FF033
:10CE000000010AF00FFE01464FF07E500AF00AFEC4
:10CE1000DFED7F7A07EE100A27EE270AB4EEC08A0C
:10CE2000F1EE10FA06D84FF00007219B83F85070FE
:10CE3000FEF7C8BE2199D1ED130AF5EEC00AF1EE56
:10CE400010FA05DD4FF0010281F85020FEF7BABE5E
:10CE5000F5EEC00AF1EE10FA4CBF0222032281F86F
:10CE60005020FEF7AFBE219D95ED125AD5ED135A15
:10CE700085EE256A85ED136ABDE6219AD06C0AF02D
:10CE8000A7FD002841F04A80FEF79CBE2199CE6C98
:10CE900030460AF02DFE08EE100A30464FF0000131
:10CEA0000AF0C0FD01464FF07E500AF0BBFDDFEDF9
:10CEB000586A07EE100A67EE267AB4EEE78AF1EEBA
:10CEC00010FA01F32B80FEF77DBE219BD86C0AF08F
:10CED0007FFD002801F02280FEF774BE219890EDBE
:10CEE000130AD0ED120AB4EEE00AF1EE10FA81F264
:10CEF0001580FEF767BE219D95ED131AD5ED121A28
:10CF0000B4EEE11AF1EE10FA01F30880FEF75ABE12
:10CF1000219A92ED132AD2ED122AB4EEE22AF1EE12
:10CF200010FA40F2FB87FEF74DBE219991ED133ABE
:10CF3000D1ED123AB4EEE33AF1EE10FA00F1EE87D9
:10CF4000FEF740BE219EF56C28460AF0D1FD08EEA2
:10CF5000100A28464FF000010AF064FD01464FF028
:10CF60007E500AF05FFD9FED2A4A04EE900A24EEFF
:10CF7000845AB4EEC58AF1EE10FA40F2CF87FEF77C
:10CF800021BE219FF86CFBF7BFFFF8640DF1700C18
:10CF90004FF00000FCF754FAFEF714BE1D9BF62B71
:10CFA00008D943F25801C2F200014FF012050D7288
:10CFB00004F009B8219CE06C0AF00AFD38B9219A06
:10CFC00092ED136AF6EE006A36EE268A06E02198A4
:10CFD00090ED138AF6EE005A38EE658A18EE100AC4
:10CFE0000AF0F6FC00BB9FED0C7AB4EEC78AF1EEB6
:10CFF00010FA04DC18EE100A0AF0EEFCA0B14FF0B3
:10D000000102219E86F850206FF000463BE000BFF1
:10D0100000000034FFFF7F4BFEFFFF4AFEFFFFCA08
:10D0200000008043000080C318EE100A0AF0D0FC14
:10D0300098B15FED067AB4EEE78AF1EE10FA04D407
:10D0400018EE100A0AF0C8FC38B14FF0010421981C
:10D0500080F850404FF0004615E018EE100A0AF034
:10D06000CBFC38B14FF00207219B83F850704FF092
:10D07000000608E0BDEEC88A18EE106A4FF0000105
:10D08000219D85F850104FEA066141EA166506F4C5
:10D090007F4745EA072406F47F0344EA132043F25E
:10D0A0009002C2F200021D9E9051FEF78BBD1D9BA7
:10D0B000F62B08D943F25806C2F200064FF01202CE
:10D0C000327203F080BF43F29007C2F20007FC58AF
:10D0D0004FEA046040EA146204F47F4642EA062103
:10D0E00004F47F0541EA152300EE103AF8EEC00A79
:10D0F000219FC7ED130A1FED381AF4EEC10AF1EEB5
:10D1000010FA06DC5FED3B1AF4EEE10AF1EE10FADC
:10D1100005D54FF0010087F85000FEF753BD4FF0E2
:10D12000000487F85040FEF74DBD0DF1700C4FF034
:10D130000100FCF785F92199C86CFBF70FFF219DD1
:10D14000E864FEF73FBD219B93ED132AF7EE002A1A
:10D1500032EE223A83ED133AF0E52199C86C0AF0D9
:10D160004BFC50B1219C4FF0000084F847004FF079
:10D17000040684F85060FEF725BD219A92ED131A3B
:10D18000B5EEC01AF1EE10FA23DB1FED5B3AB4EEF8
:10D19000C31AF1EE10FA0FD5FCEEC13A13EE902A45
:10D1A0000DF1700CD0B2FCF75FF84FF00007219B37
:10D1B00083F85070FEF706BD0DF1700C4FF0FF00C4
:10D1C000FCF752F84FF00205219981F85050FEF714
:10D1D000F9BCB5EEC01AF1EE10FA7EF5F3AC5FEDD6
:10D1E0006F1AB4EEE11AF1EE10FA11DDB1EE412A38
:10D1F000FCEEC22A12EE904A0DF1700CE0B2FCF780
:10D2000033F84FF00100219E86F85000FEF7DABC9B
:10D210000DF1700C4FF0FF00FCF726F84FF00307FC
:10D22000219B83F85070FEF7CDBC43F22405C2F277
:10D230000005297811F0280F08D01D9A02F101028B
:10D24000B2F5005F34BF0022012206E01D9A02F110
:10D250000102FA2A94BF0022012242B143F258038C
:10D26000C2F200034FF01300187203F0ACBE219F0E
:10D2700097ED134AFDEEC44A14EE903A1CB21C948A
:10D28000A0B2C3F3072646EA002540F6E871C2F2D1
:10D2900000011D9A8D52FEF795BC43F22406C2F29E
:10D2A0000006357815F0280F08D01D9901F101010D
:10D2B000B1F5005F34BF0021012106E01D9901F1A5
:10D2C0000101FA2994BF0021012141B143F2580123
:10D2D000C2F200014FF013030B7203F074BE219FE2
:10D2E00097ED135AFCEEC55A15EE904AA3B21C9363
:10D2F0004FEA132242EA032040F6E876C2F2000623
:10D300001D9D7053FEF75EBC1D9F219CA764FEF718
:10D3100059BC1D9A2198C264FEF754BC0DF1700CE3
:10D32000FBF7BAFF06EE100AF8EE466A219EC6ED3C
:10D33000136AFEF747BC43F22405C2F200052978C0
:10D3400011F0280F08D01D9B03F10103B3F5005F16
:10D3500034BF0023012306E01D9B03F10103FA2BD8
:10D3600094BF0023012343B143F25803C2F20003E8
:10D370004FF01300187203F026BE40F6E877C2F2B1
:10D3800000071D9C385B4FEA102242EA0026B5B226
:10D3900007EE905AB8EE670A219981ED130A9FEDC6
:10D3A000C97AB4EEC70AF1EE10FAFEF60BACDFED67
:10D3B000C60A30EE601A81ED131AFEF703BC43F281
:10D3C0002402C2F20002167816F0280F08D01D9D24
:10D3D00005F10105B5F5005F34BF0025012506E024
:10D3E0001D9D05F10105FA2D94BF0025012545B1CC
:10D3F00043F25805C2F200054FF01301297203F001
:10D40000E2BD40F6E877C2F200071D9C395B4FEAA7
:10D41000112343EA012082B201EE902AB8EE612A7C
:10D42000219E86ED132AFEF7CDBB1D98072808D94B
:10D4300043F25803C2F200034FF00800187203F0E1
:10D44000C2BDFCF77DFB02EE900AB8EE623A219F66
:10D4500087ED133AFEF7B6BB219CD4ED133A94ED59
:10D46000124A63EE844AC4ED134AFFF7C4BB219A03
:10D4700092ED135AF1EE455AC2ED135AFEF7A2BBD4
:10D480004FF000004FF001010A46FDF7B7FB219E67
:10D4900096ED136AF1EE046A66EE267A4FF0000507
:10D4A0000095019543F2D010C2F20000BCEEE70AED
:10D4B00010EE101A4FF0FF024AF66143C0F6040363
:10D4C000FAF7A8F9FEF77EBB43F22401C2F200018D
:10D4D0000B7813F0280F08D01D9800F10300B0F569
:10D4E000005F34BF0020012006E01D9800F103001A
:10D4F000FA2894BF0020012040B143F25806C2F23E
:10D5000000064FF01305357203F05DBD40F6E87775
:10D51000C2F200071D9C3859FBF720FD219A906448
:10D52000FEF750BB43F22401C2F200010B7813F066
:10D53000280F08D01D9800F10300B0F5005F34BF3C
:10D540000020012006E01D9800F10300FA2894BF96
:10D550000020012040B143F25806C2F200064FF00D
:10D560001305357203F02FBD40F6E877C2F20007CD
:10D570001D9C3859FBF7F2FC219AD064FEF722BBC0
:10D580001D99072908D943F25803C2F200034FF04E
:10D5900008021A7203F017BD219BD3ED130AF5EEB2
:10D5A000C00AF1EE10FA0FDB9FED487AF4EEC70ADD
:10D5B000F1EE10FA08D8FCEEE01ACDED1C1A4FF08F
:10D5C000000083F8500021E09FED401AF4EEC10AFC
:10D5D000F1EE10FA07DD6FF07F451C954FF0010169
:10D5E00083F8501012E04FF000001C9010EE900AEB
:10D5F0000AF0EEF928B14FF00202219E86F8502081
:10D6000004E04FF00307219C84F850701D981C998A
:10D61000FCF768FAFEF7D6BA219FF86C0AF0ECF92D
:10D6200000287EF4CFAA219C94ED132AB5EEC02ADF
:10D63000F1EE10FA04DD4FF07E55E564FEF7C2BA54
:10D64000B5EEC02AF1EE10FA7EF5BCAA4FF0000646
:10D65000CBF68076E664FEF7B5BA2199886AC8B140
:10D66000FAF70EF9219FBA6AC2F1040426184CF6A3
:10D67000CD45CCF6CC45A5FB06104FEA90017B6A60
:10D68000B1FBF3F202EE902AB8EE623A87ED133A5C
:10D69000FEF798BA4FF6FF73C7F67F73CB64FEF7B9
:10D6A00091BA43F22406C2F20006357815F0280F2D
:10D6B00010D01D9800F10300B0F5005F34BF0020CA
:10D6C00001200EE00000004700008047FFFF7F4B75
:10D6D000000000341D9800F10300FA2894BF0020D8
:10D6E000012040B143F25803C2F200034FF013028D
:10D6F0001A7203F068BC1D9F219CE06CFBF704FCD0
:10D7000040F6E871C2F20001C851FEF75BBA219EF3
:10D71000D6ED123A96ED134A73EEC44AC6ED134A9B
:10D72000FFF769BA219DE86C1C90AF6CEF64A864A8
:10D73000FEF748BA219CE06C0AF05EF930B14FF078
:10D740000306219B83F85060FEF73CBA2199C86C10
:10D750000AF042F930B14FF00404219981F85040A9
:10D76000FEF730BA219BDE6C30460AF0C1F908EEB4
:10D77000100A30464FF000010AF054F901464FF00C
:10D780007E500AF04FF91FED2E5A05EE900A25EE55
:10D79000856AB4EEC68AF1EE10FA06D84FF00000A2
:10D7A000219F87F85000FEF70DBA219DD5ED136A31
:10D7B000F5EEC06AF1EE10FA05DD4FF0010285F8D2
:10D7C0005020FEF7FFB9F5EEC06AF1EE10FA4CBF3B
:10D7D0000222032285F85020FEF7F4B9219DD5EDF1
:10D7E000138A95ED128A38EEC89A19EE100A0AF0DB
:10D7F0007FF909EE100A18EE900A18EE101A0AF0D6
:10D8000011F901464FF07E500AF00CF95FED507AA5
:10D8100000EE100A60EE270AB4EEE09AF1EE10FA7C
:10D820000DF1700C8CBF00200120FBF71DFDFEF7F1
:10D83000C9B9219AD76C38460AF05AF908EE100A8D
:10D8400038464FF000010AF0EDF801464FF07E50E7
:10D850000AF0E8F81FED621A07EE100A67EE011AE7
:10D86000B4EEE18AF1EE10FA0DF1700C8CBF0020DD
:10D870000120FBF7F9FCFEF7A5B9219890ED132ADA
:10D88000D0ED122AB4EEE22AF1EE10FA0DF1700C8E
:10D89000B4BF00200120FBF7E7FCFEF793B9219C01
:10D8A00094ED133AB5EEC03AF1EE10FA0DF1700CAA
:10D8B000B4BF00200120FBF7D7FCFEF783B9219904
:10D8C000D1ED133A91ED124AF4EEC43AF1EE10FAAA
:10D8D0000DF1700CD4BF00200120FBF7C5FCFEF752
:10D8E00071B9219ED6ED134A96ED125AF4EEC54A4F
:10D8F000F1EE10FA0DF1700C8CBF00200120FBF747
:10D90000B3FCFEF75FB9219BD3ED135A93ED126A76
:10D91000F4EEC65AF1EE10FA0DF1700C54BF00206F
:10D920000120FBF7A1FCFEF74DB9219DD5ED136A4F
:10D93000F5EEC06AF1EE10FA0DF1700C54BF002044
:10D940000120FBF791FCFEF73DB9219AD2ED138A35
:10D9500092ED128A38EEC89A19EE100A0AF0C8F849
:10D9600009EE100A18EE900A18EE101A0AF05AF88A
:10D9700001464FF07E500AF055F85FEDAB7A00EEAD
:10D98000100A60EE270AB4EEE09AF1EE10FA0DF1FB
:10D99000700CD4BF00200120FBF766FCFEF712B923
:10D9A000219FFC6C20460AF0A3F808EE100A2046DE
:10D9B0004FF000010AF036F801464FF07E500AF0B1
:10D9C00031F81FEDBD1A07EE100A67EE011AB4EE2A
:10D9D000E18AF1EE10FA0DF1700CD4BF00200120A5
:10D9E000FBF742FCFEF7EEB843F22400C2F200005F
:10D9F000017811F0280F08D01D9E06F10206B6F539
:10DA0000005F34BF0026012606E01D9E06F10206D7
:10DA1000FA2E94BF0026012646B143F25803C2F203
:10DA200000034FF01300187203F0CDBAF9F728FF86
:10DA3000219B00F104004CF6CD45CCF6CC45A5FB6E
:10DA400000124FEA92075C6AB7FBF4F61D9A40F6A3
:10DA5000E870C2F2000081184D78875C4FEA0744F5
:10DA600044EA05208A7840EA02011B91761A26F0E2
:10DA70007F451C9502EE105AF8EE422AC3ED132A98
:10DA8000FEF7A0B8219FFC6CBC64FEF79BB8219AFE
:10DA900092F85110002940F04182FEF793B8219E80
:10DAA00096F85150002D00F03982FEF78BB843F202
:10DAB0002403C2F20003187810F0280F06D01D9A34
:10DAC000B2F5005F34BF0022012204E01D9AFA2A59
:10DAD00094BF0022012242B143F25800C2F200007A
:10DAE0004FF01302027203F06EBA40F6E871C2F210
:10DAF00000011D9E8D5D002D7EF464A81E9B1C936D
:10DB00000EE243F22401C2F200010E7816F0280F53
:10DB100006D01D9DB5F5005F34BF0025012504E04A
:10DB20001D9DFA2D94BF0025012545B143F25806ED
:10DB3000C2F200064FF01305357203F044BA40F606
:10DB4000E870C2F200001D9BC25C002A3EF43AA8B5
:10DB50001E991C91E4E143F25800C2F200004FF01C
:10DB60000103037203F02FBA1D99F92908D943F272
:10DB70005803C2F200034FF01201197203F023BAE6
:10DB800043F29002C2F20002565C1E9D2E427EF4C9
:10DB900019A81F981C90C3E11D9EF92E08D943F2C5
:10DBA0005801C2F200014FF012060E7203F00BBAD8
:10DBB00043F29002C2F20002955D1E9805423EF4C7
:10DBC00001A81F9B1C93ABE143F22402C2F20002A6
:10DBD000157815F0280F06D01D98B0F5005F34BFFA
:10DBE0000020012004E01D98FA2894BF00200120A5
:10DBF00040B143F25805C2F200054FF013002872FD
:10DC000003F0E1B940F6E871C2F200011D9BCE5C61
:10DC1000002E7DF4D7AF1E9A1C92B2E143F224018C
:10DC2000C2F200010B7813F0280F06D01D9EB6F546
:10DC3000005F34BF0026012604E01D9EFA2E94BF2B
:10DC40000026012646B143F25803C2F200034FF00A
:10DC500013061E7203F0B7B940F6E872C2F2000272
:10DC60001D9D505D00283DF4ADAF1E991C9188E1CB
:10DC700043F22402C2F20002157815F0280F06D0F4
:10DC80001D98B0F5005F34BF0020012004E01D980E
:10DC9000FA2894BF0020012040B143F25800C2F29C
:10DCA00000004FF01301017203F08DB940F6E871E6
:10DCB000C2F200011D9BCE5C1E9A96427DF682AF99
:10DCC0001F9D1C952CE143F22403C2F200031E7831
:10DCD00016F0280F06D01D9AB2F5005F34BF00225F
:10DCE000012204E01D9AFA2A94BF0022012242B1C7
:10DCF00043F25805C2F200054FF013022A7203F0F6
:10DD000062B940F6E875C2F200051D98295C1E9BB9
:10DD10009942FDF457AF1F9E1C9601E143F2240087
:10DD2000C2F20000017811F0280F06D01D9BB3F558
:10DD3000005F34BF0023012304E01D9BFA2B94BF36
:10DD40000023012343B143F25803C2F200034FF012
:10DD500013061E7203F037B940F6E876C2F20006E9
:10DD60001D9D725D1E9882427DF42CAF1F991C91FF
:10DD7000D6E043F22405C2F200052A7812F0280FFB
:10DD800006D01D98B0F5005F34BF0020012004E0EC
:10DD90001D98FA2894BF0020012040B143F258009A
:10DDA000C2F200004FF01301017203F00CB940F60B
:10DDB000E871C2F200011D9BCE5C1E9DAE423DF497
:10DDC00001AF1F9A1C92ABE043F22403C2F200039E
:10DDD0001E7816F0280F06D01D9DB5F5005F34BFE4
:10DDE0000025012504E01D9DFA2D94BF0025012585
:10DDF00045B143F25805C2F200054FF013022A72F2
:10DE000003F0E1B840F6E872C2F200021D98115C1E
:10DE10001E9B99423DF6D6AE1F9E1C9680E043F2B3
:10DE20002400C2F20000017811F0280F06D01D9BDB
:10DE3000B3F5005F34BF0023012304E01D9BFA2BE0
:10DE400094BF0023012343B143F25803C2F20003FD
:10DE50004FF013061E7203F0B6B840F6E876C2F231
:10DE600000061D9D725D1E988242BDF4ABAE1F99E7
:10DE70001C9155E0219D95F847201D9882427DF424
:10DE8000A1AE1E991C917CE0219B93F847601D9DDB
:10DE9000AE423DF497AE1E9A1C9272E0219890F823
:10DEA00047101D9B99427DF68DAE1E9E1C9668E024
:10DEB000219D95F847201D988242FDF483AE1E995E
:10DEC0001C915EE0219B93F847601D9DAE42BDF41E
:10DED00079AE1E9A1C9254E0219890F847101D9B31
:10DEE00099423DF66FAE1E9E1C964AE09DF8740066
:10DEF0000DF16B01FCF7A2FD8DF86A009DF86B50E7
:10DF000035B143F25800C2F20000057203F05BB86D
:10DF100000283DF457AE1E9A1C9201E01D991C91F9
:10DF20001C9E40F20000C0F6020090F82E1090F8FF
:10DF30002F3043EA0122B24208D243F25805C2F21E
:10DF400000054FF009062E7203F03DB843F2B817F2
:10DF5000C2F200073E60FDF735BE0DF1700CFBF715
:10DF60009BF91C900028D9D0FDF72CBE0DF1700C48
:10DF7000FBF792F91C900028D0D1FDF723BE1D9B22
:10DF80001C93219A166A052E08D943F25806C2F24C
:10DF900000064FF00A02327203F015B806F10200D3
:10DFA00043F2B811C2F200010D6842F8205006F1A8
:10DFB0000106219B1E62B3E70DF1700CFBF76CF9B3
:10DFC0001C900028DBD0FDF7FDBD0DF1700CFBF7B8
:10DFD00063F91C900028D2D1FDF7F4BD0DF1700C4F
:10DFE000FBF75AF91C901D9EB0427DF4EBAD1E9DCF
:10DFF0001C9595E70DF1700CFBF74EF91C901D9ADE
:10E0000090423DF4DFAD1E981C9089E70DF1700C35
:10E01000FBF742F91C901D9988427DF6D3AD1E9BFB
:10E020001C937DE70DF1700CFBF736F91C901D9EDB
:10E03000B042FDF4C7AD1E9D1C9571E70DF1700C4B
:10E04000FBF72AF91C901D9A9042BDF4BBAD1E98B7
:10E050001C9065E70DF1700CFBF71EF91C901D99E3
:10E0600088423DF6AFAD1E9B1C9359E79DF87400A6
:10E070000DF16B01FCF7B2FC8DF86A009DF86B6046
:10E0800036B143F25802C2F20002167202F09BBF90
:10E0900000283DF497AD1E9D1C9541E79DF8740046
:10E0A0000DF16B01FCF79AFC8DF86A009DF86B107E
:10E0B00031B143F25803C2F20003197202F083BF78
:10E0C00000287DF47FAD1E981C9029E70DF1700C9F
:10E0D000FBF70AF940F6E876C2F200061E9D725D73
:10E0E0001D990A423DF46EAD1F981C9018E70DF182
:10E0F000700CFBF7F9F840F6E876C2F200061E9BBA
:10E10000F55C1D9A15427DF45DAD1F991C9107E7E2
:10E110000DF1700CFBF7E8F840F6E870C2F2000071
:10E120001E9E855D1D9B1D427DF44CAD1F9A1C9269
:10E1300027E70DF1700CFBF7D7F840F6E871C2F253
:10E1400000011E980E5C1D9D2E423DF43BAD1F9BB1
:10E150001C9316E73C7844F008003870FDF700BEC9
:10E160000DF1700CFBF798F88DF86A00219991F881
:10E1700051501D9BEE181C9643F22402C2F200027D
:10E18000117811F0280F09D01E9A02F1FF318E1973
:10E19000B6F5005F34BF0026012607E01E9D05F19D
:10E1A000FF339E19FA2E94BF0026012646B143F292
:10E1B0005803C2F200034FF013051D7202F003BFB3
:10E1C0004FF000071B971E9CE4B11C9E40F6E875BB
:10E1D000C2F20005AB5D834232D004F1FF3240F65B
:10E1E000E871C2F200018B1940F6E877C2F200072D
:10E1F000C7F10104C6F10106F51B12F0010F18D09A
:10E2000002F067BF4FF0FF001B9019E013F8018F79
:10E2100002F1FF37404503D11C911B961E920FE07F
:10E220003A46E118EE1813F801CF604542F05D87D9
:10E23000F2E7E118EE18002AE8D11C911E92E1E7FE
:10E240000DF1700C9DF86C00FBF70EF8FDF7BABCF1
:10E250000DF1700CFBF720F843F2BC110E46C2F230
:10E26000000630704FF001021C92B246BAE02198CD
:10E2700090F851501D9BE9181C9143F22406C2F2FC
:10E280000006327812F0280F07D001F10101B1F534
:10E29000005F34BF0021012105E001F10101FA29ED
:10E2A00094BF0021012141B143F25800C2F20000A5
:10E2B0004FF01305057202F086BE1E981B900DF1FB
:10E2C000700C26AC44F0010122AF47F001024FF080
:10E2D0000003FBF71BF8FDF775BC219B93F8511069
:10E2E0001D9E88191C9043F22402C2F20002157888
:10E2F00015F0280F05D0B0F5005F34BF00200120D5
:10E3000003E0FA2894BF0020012040B143F25801F5
:10E31000C2F200014FF013060E7202F054BE1F9CB1
:10E320001E98A04228BF20461B900DF1700C26AF0E
:10E3300047F0010122AB43F001024FF00003FCF76C
:10E34000B5F8FDF73FBC0DF1700CFAF7A5FF0346D9
:10E3500043F2BC100546C2F2000528464FF01001FA
:10E360004CF20862C0F6050209F00CFD1C90AA46AA
:10E3700038E01E9A1C921F9B1B934FF0000A31E05D
:10E380004FF0FF311C918A462CE0219EF06C9DF8E5
:10E3900078109DF87C2043F2BC15C2F20005009570
:10E3A0004FF0100301934FF00103FCF79FFF4FF074
:10E3B000FF301C90AA4615E0219AD06C9DF8781089
:10E3C0009DF87C2043F2BC16C2F2000600964FF086
:10E3D000100501954FF00003FCF788FF4FF0FF3167
:10E3E0001C91B2461D9BA3F1FB018AB20D92A3F1D1
:10E3F000FB06032E23D840F2A065C1F200054FF4BE
:10E4000011730D9903FB015292F82002032808D0E2
:10E4100043F25803C2F200034FF04800187202F0B2
:10E42000D2BD40F2A067C1F200074FF411760D9DF6
:10E4300006FB057606F104064FF0000505E0219F76
:10E4400097F85100C5184FF000061C9B0B93B3F1D1
:10E45000FF3F10D14FF0FF010B914FF000084746EE
:10E4600043F22400C2F200000E9040F6E873C2F2BC
:10E4700000030F9305E00B9A002AEED14FF000083D
:10E4800070E01D99A1F1FB01032910D8D6F80051C5
:10E49000FF2D14BF01353D46D6F80421954206D123
:10E4A0003846FBF76FFFD6F804018542F8D0BAF181
:10E4B000FF3F14D1219850F8342F1368D3F800C0CF
:10E4C000414610AA4FF00103E0478DF86B0088B178
:10E4D00043F25805C2F20005287202F074BDBAF189
:10E4E000000F04D01AF808108DF8401002E01B9BB2
:10E4F0008DF840301C98B0F1FF3F02D19DF84010DC
:10E5000081B31D9AA2F1FB02032A07D8D6F8003185
:10E510009DF84000F054C6F800511EE00E9B18789C
:10E5200010F0280F05D0B5F5005F34BF00200120A2
:10E5300003E0FA2D94BF0020012040B143F25806B9
:10E54000C2F200064FF01305357202F03CBD9DF893
:10E5500040100F9A515505F1010508F101080B997A
:10E5600088458ED31D9CA4F1FB04032C05D80D9E79
:10E57000F0B2FBF721F9FDF725BB219F97F8512059
:10E5800008EB020E87F851E0FDF71CBB1D9AA2F1C3
:10E59000FB03032B58D89FB240F2A060C1F20000E9
:10E5A0004FF4117101FB070292F82032032B08D0BF
:10E5B00043F25806C2F200064FF04800307202F0F3
:10E5C00002BD40F2A065C1F200054FF4117404FBD6
:10E5D000075404F104041E9E06F1FF301E9076B32A
:10E5E0004FF0000643F2B818C2F2000840F20001F2
:10E5F0008A46C0F6020AD4F80051FF2D14BF013537
:10E600003546D4F80421954206D13046FBF7BAFED0
:10E61000D4F804319D42F8D0D8F80000D4F8002195
:10E620001AF80010A15400F10100C8F80000C4F865
:10E6300000511E9D05F1FF331E93002DDBD1F8B272
:10E64000FBF7BAF8FDF7BEBA1E9E1C96219991F809
:10E65000510082181B9243F22405C2F200052B7868
:10E6600013F0280F08D006F1FF339A18B2F5005FB7
:10E6700034BF0022012206E006F1FF35AA18FA2A6B
:10E6800094BF0022012242B143F25805C2F20005B4
:10E690004FF013062E7202F096BC841981F8514097
:10E6A0001C9A02F1FF341C94002A3DF48BAA43F219
:10E6B000B817C2F200073D681B9E40F6E871C2F22F
:10E6C0000001891940F20000C0F6020028184FF03E
:10E6D000000304F0010710F8038001F8038003F140
:10E6E0000103934242F0E98409E0C75CCF5403F18F
:10E6F0000103C75CCF5403F101039342F5D1A01984
:10E70000611901F1010143F2B812C2F20002116075
:10E710004FF0FF331C9300F101001B90FDF752BA3C
:10E720004FF000028DF86A20219D95F851601D9BE5
:10E73000F1181C911E9A1B9243F22400C2F20000B1
:10E74000067816F0280F08D002F1FF304218B2F513
:10E75000005F34BF0022012206E002F1FF335A18A5
:10E76000FA2A94BF0022012242B143F25805C2F2B4
:10E7700000054FF013022A7202F025BC40F6E8773C
:10E78000C2F2000707EB01089DF87CA043F28C144D
:10E79000C2F200042668AD6B7119755DFF2D50D073
:10E7A0000B914FF0010209920B98477807EB052473
:10E7B00043F28C16C2F2000633681D194FF00001B7
:10E7C0001C919DF86A20002A02F04D841C5D05F121
:10E7D000010502F04ABC9DF86A600EB14CB901E037
:10E7E0006B7833B9219F97F85130C61887F851607C
:10E7F0002AE015F8016F18F800A047B9304609F073
:10E8000065FAC6B2504609F061FA5FFA80FA5645D9
:10E8100008D11C9800F101001C9004F1FF341B99F1
:10E820008142D8D2BA46099A02F1010209920B9CA0
:10E8300014F8025F0B94FF2DB6D14FF00000099041
:10E8400002E04FF0000309930DF1700C0999C8B272
:10E85000FAF70AFDFDF7B6B94FF001018DF86A101D
:10E8600062E70DF1700CFAF717FD034643F2BC1096
:10E870000646C2F2000630464FF010014CF210621C
:10E88000C0F6050209F07EFA1C90B246AAE50DF129
:10E89000700CFAF701FD034643F2BC110D46C2F2BB
:10E8A000000528464FF010014CF21862C0F6050230
:10E8B00009F068FA1C90AA4694E50DF1700CFAF77D
:10E8C000EBFC034643F2BC121646C2F20006304689
:10E8D0004FF010014CF21C62C0F6050209F052FA2A
:10E8E0001C90B2467EE50DF1700CFAF7D5FC03469C
:10E8F00043F2BC100546C2F2000528464FF0100155
:10E900004CF22462C0F6050209F03CFA1C90AA46BB
:10E9100068E5219991F8514004F1010481F85140D2
:10E92000FDF750B91D9F40F6E872C2F20002D65DB5
:10E9300006F10106D655FDF745B9219D95F84730FA
:10E9400003F1010385F84730FDF73CB99DF87400E9
:10E950000DF16B01FCF742F80DF1700C002814BFAB
:10E96000FF200020FAF780FC9DF86B0000283DF4A2
:10E9700029A943F25801C2F20001087202F023BB38
:10E980009DF874000DF16B01FCF790F80DF1700C1F
:10E99000002814BFFF200020FAF766FC9DF86B608A
:10E9A000002E3DF40FA943F25802C2F20002167283
:10E9B00002F009BB1D9D1C954FF000031B934FF007
:10E9C00001008DF86A009DF870000DF16B01FCF7F5
:10E9D00005F89DF86B1099B920B19DF86A601B9AF3
:10E9E00032431B929DF86A504FEA45038DF86A3016
:10E9F0001C9800F101001C9013F0FE0FE3D10AE017
:10EA00009DF86A60012E06D143F25802C2F200025C
:10EA1000117202F0D8BA0DF1700C9DF86C00FAF783
:10EA200023FCFDF7CFB81D991C914FF000051B95F5
:10EA30004FF001038DF86A309DF870000DF16B0105
:10EA4000FCF734F89DF86B609EB920B19DF86A0020
:10EA50001B9A02431B929DF86A104FEA41058DF8FC
:10EA60006A501C9B03F101031C9315F0FE0FE3D1C8
:10EA70000AE09DF86A00012806D143F25802C2F26A
:10EA80000002167202F09FBA0DF1700C9DF86C0036
:10EA9000FAF7EAFBFDF796B89DF874000DF16B01EB
:10EAA000FBF7CCFF8DF86A009DF86B6036B143F23E
:10EAB0005801C2F200010E7202F085BA0DF1700C1D
:10EAC000002814BFFF200020FAF7CEFBFDF77AB82C
:10EAD0001D9D1C954FF000031B934FF001068DF810
:10EAE0006A60219890F8472016420ED09DF8700079
:10EAF0000DF16B01FBF7A2FF9DF86B609EB920B191
:10EB00009DF86A101B9D0D431B959DF86A304FEAD6
:10EB100043008DF86A001C9A02F101021C9210F069
:10EB2000FE06DED10AE09DF86A10012906D143F203
:10EB30005805C2F200052E7202F045BA1B9C219FB7
:10EB400087F84740FDF73EB89DF874000DF16B0162
:10EB5000FBF7DCFF0DF1700C002814BFFF20002034
:10EB6000FAF782FB9DF86B30002B3DF42BA843F2A3
:10EB70005800C2F20000037202F025BA1D9A1C92DE
:10EB8000D0B20DF16B01FBF7C1FF1B909DF86B60DC
:10EB900036B143F25802C2F20002167202F013BA02
:10EBA0004FF001018DF86A101C9C60181C90C0B2D7
:10EBB0000DF16B01FBF7AAFF9DF86A7000FA07F0F0
:10EBC0001B9D05431B9507F101078DF86A701C9882
:10EBD00000F101001C90FBB2072BE8D90DF1700C7D
:10EBE0009DF86C00FAF740FBFCF7ECBF0DF1700CE0
:10EBF000219E96F85100FAF737FBFCF7E3BFFCF7CC
:10EC0000E1BF43F24001C2F200014FF001040C7079
:10EC1000FCF7D8BF43F24007C2F200074FF00005EF
:10EC20003D70FCF7CFBF21984FF000014FF0540228
:10EC300009F0DEFC4FF00000219043F29013C2F285
:10EC400000031A6802F1FF361E6002F028B943F291
:10EC50009010C2F2000003687F2B08D943F25800DD
:10EC6000C2F200004FF03003037202F0ACB94FF073
:10EC700001041C9440F2A067C1F20007D7F8A8294C
:10EC8000002A42F0FD8105E0D6F8AC50002D4ED1AF
:10EC90001C9301E04FF001031D9F40F2A065C1F2FB
:10ECA00000054FF0540404FB03F3EA18C2F850794E
:10ECB000C2F854791E9E82F8A2694FF00A01C2F888
:10ECC000741905F51567F81800F13400219901F160
:10ECD00034014FF0100209F067FC1C9804FB00702F
:10ECE00000F14400219901F144014FF0040209F0C0
:10ECF0005BFC1C9B04FB037000F14800219901F1AF
:10ED000048014FF0080209F04FFC219A92F8516037
:10ED10001C9904FB015585F8A16943F29014C2F2D5
:10ED20000004276807F101072760FCF74BBF03F1D8
:10ED30000104234606F15406D6F8AC00002842F040
:10ED4000B381A5E71C93FCF73DBF219991F8525080
:10ED50001E957CE70DF1700CFAF79EFA1E9076E78F
:10ED60001D9A219E86F85120FCF72CBF0DF1700CE6
:10ED70009DF87400FAF778FAFCF724BF21998D6AA0
:10ED8000002D3CF41FAFF8F77BFD219B9A6A801A97
:10ED90005E6A1D9906FB01F101EB8105A842BCF4F6
:10EDA00011AF1E9B1C93FFF7BBB8F8F769FD219CC0
:10EDB000A062FCF707BF43F29002C2F2000292F891
:10EDC000FB201E9E9019FB2808D943F25801C2F27D
:10EDD00000014FF012050D7202F0F5B843F2240164
:10EDE000C2F200010D7815F0280F09D01D9D5319AE
:10EDF00003F1FF31B1F5005FB4BF0021012107E04D
:10EE00001D9BD01800F1FF31FA29D4BF0021012148
:10EE100041B143F25800C2F200004FF013020272F7
:10EE200002F0D1B843F29007C2F20007B81940F6D9
:10EE3000E874C2F200041D9EA11909F0B5FBFCF7AD
:10EE4000C1BE3B7843F010043C70FCF789BF219FA2
:10EE500097F84760002E0CBFFF20002087F847007E
:10EE6000FCF7B0BE219991F847206FEA020581F8BE
:10EE70004750FCF7A7BE0DF1700CFAF735FA1E9B50
:10EE800040F6E874C2F20004E75C1D9E7E40E65442
:10EE9000FCF798BE2198816B1D9A55181C95BDE111
:10EEA000219BDE6B986B31181C91B7E1219D2A6C78
:10EEB00042B943F25803C2F200034FF020061E721B
:10EEC00002F081B802F1FF342C64FCF77BBE21987C
:10EED000016C01F10101016400297CF473AE43F27D
:10EEE0005805C2F200054FF020022A7202F06BB8FA
:10EEF000219B5E6B3068416841B943F25800C2F211
:10EF000000004FF01E01017202F05DB80DF1700CAF
:10EF1000FAF7C2F91C90219850F8345F2A685668B5
:10EF20001D991CAA4FF00103B0478DF86B00002813
:10EF30003CF448AE43F25803C2F20003187202F0E8
:10EF400042B80DF1700CFAF7A7F91C9054E10DF1DD
:10EF5000700CFAF7A1F9219FF863FCF733BE0DF1AD
:10EF6000700CFAF799F9219C2064FCF72BBE2198CC
:10EF700050F8345F2A6816681D991CAA4FF00103E7
:10EF8000B0478DF86B0030B143F25803C2F2000372
:10EF9000187202F018B80DF1A80C1CF8380DFAF729
:10EFA00063F9FCF70FBE2198416B0DF1700C087AE4
:10EFB000FAF75AF9FCF706BE0DF1700C219F97F88D
:10EFC0003C00FAF751F9FCF7FDBD219D2A6CFF2AA0
:10EFD00008D943F25806C2F200064FF020033372FC
:10EFE00001F0F1BF0DF1700CD0B2FAF73DF9FCF76A
:10EFF000E9BD219850F8344F21688F68B84703EE77
:10F00000100AF8EE433A2198C0ED133AFCF7DABD46
:10F01000219D95ED0E4AF8EE444AC5ED134AFCF7E2
:10F02000D1BD219A92ED105AF8EE455AC2ED135A0D
:10F03000FCF7C8BD219E96ED136AFCEEC66ACDEDC5
:10F040001C6AEBE0219BD3ED137A9FEDB40AF4EE3A
:10F05000C07AF1EE10FA08DB43F25801C2F2000167
:10F060004FF02000087201F0AEBFFCEEE70AC3EDDE
:10F07000100AFCF7A7BD219850F8345F2A6816687B
:10F080001D991CAA4FF00403B0478DF86B0030B1F6
:10F0900043F25803C2F20003187201F094BF1C98A7
:10F0A000F9F75CFF219CA064FCF78CBD219850F817
:10F0B000341F0D682E681D991CAA4FF00403B04739
:10F0C0008DF86B0030B143F25802C2F200021072A8
:10F0D00001F079BF1C98F9F741FF219FF864FCF714
:10F0E00071BD2198436B19684D6845B943F25800CA
:10F0F000C2F200004FF01E01017201F064BFC06C4B
:10F10000F9F702FF1C90219850F8346F3268556867
:10F110001D991CAA4FF00403A8478DF86B00002826
:10F120003CF450AD43F25803C2F20003187201F0F0
:10F130004ABF43F22406C2F20006327812F0280FCA
:10F140000BD0219AD56B1D98431903F1FF36B6F504
:10F15000005F34BF0026012609E0219DE86B1D9B5E
:10F16000191801F1FF36FA2E94BF0026012646B188
:10F1700043F25800C2F200004FF01301017201F097
:10F1800022BF219B184650F8341F0E6835684FF097
:10F19000000140F6E876C2F200061D9AB218DB6B59
:10F1A000A8478DF86B0000283CF40CAD43F25803DF
:10F1B000C2F20003187201F006BF219850F8345FC4
:10F1C0002E6835681D991BAA4FF00403A8478DF8D7
:10F1D0006B0030B143F25805C2F20005287201F00D
:10F1E000F2BE1B9B9AB2C3F3072040EA02218EB203
:10F1F0001C9613E01D9B1C931C982199FAF7EAF8C2
:10F200008DF86B0000283CF4DDAC43F25802C2F2EA
:10F210000002107201F0D7BE1D981C901C99B1F528
:10F22000803F08D343F25806C2F200064FF01F0594
:10F23000357201F0C8BE219CA163FCF7C3BC1D9CC4
:10F24000219FFC63FCF7BEBC1D99219E3164FCF735
:10F25000B9BC219DAA6B1D9BD01A1C90DEE71E9A9B
:10F26000219BD96B8818FB2808D943F25803C2F2B6
:10F2700000034FF01200187201F0A5BE43F2900691
:10F28000C2F2000686F8FB10184650F8345F296871
:10F290000D681D99B218DB6BA8478DF86B0000282C
:10F2A0003CF490AC43F25802C2F20002107201F03A
:10F2B0008ABE219B5E6B31684D6845B943F25801A7
:10F2C000C2F200014FF01E060E7201F07CBE43F246
:10F2D0002402C2F20002107810F0280F0AD0DE6B70
:10F2E0001D998A1902F1FF30B0F5005F34BF00208C
:10F2F000012008E0DE6B1D998A1902F1FF30FA281F
:10F3000094BF0020012058B143F25805C2F2000515
:10F310004FF01300287201F056BE00BF0000804776
:10F3200003F134004FF0000140F6E876C2F2000627
:10F330001D9AB218DB6BA8478DF86B0000283CF4CF
:10F3400041AC43F25803C2F20003187201F03BBE15
:10F35000F6F7EEFD00287CF435AC1D9A1C92FEF702
:10F36000DFBDF6F7E5FD00283CF42CAC1D9B1C939B
:10F37000FEF7D6BD1D9D132D08D943F25800C2F2E9
:10F3800000004FF00501017201F01DBEE8B24FF020
:10F390000001F6F78BFD01EE100AB8EE417A219FCD
:10F3A00087ED137AFCF70EBC1D9E132E08D943F28D
:10F3B0005803C2F200034FF005021A7201F003BEB7
:10F3C000F0B24FF00101F6F771FD01EE900AB8EED0
:10F3D000612A219C84ED132AFCF7F4BB1D9D132D9B
:10F3E00008D943F25800C2F200004FF00501017243
:10F3F00001F0E9BDE8B24FF00001F6F7C7FCFCF7F9
:10F40000E1BB1D9E132E08D943F25803C2F200033C
:10F410004FF005021A7201F0D6BDF0B24FF00101B3
:10F42000F6F7B4FCFCF7CEBB1D9D132D08D943F2B3
:10F430005800C2F200004FF00501017201F0C3BD97
:10F44000E8B24FF00001F6F7F1FCFCF7BBBB1D9EE4
:10F45000132E08D943F25803C2F200034FF00502FD
:10F460001A7201F0B0BDF0B24FF00101F6F7DEFC08
:10F47000FCF7A8BB9DF87400F2F732F800287CF482
:10F48000A1AB43F25805C2F200054FF028002872E4
:10F4900001F099BD9DF87400219901F14C01F2F73A
:10F4A0003FF800287CF48EAB43F25801C2F2000111
:10F4B0004FF028060E7201F086BD219BD3ED132A72
:10F4C0009DF87400BCEEE23A13EE101AF2F75AF807
:10F4D00000287CF477AB43F25805C2F200054FF0E8
:10F4E00028022A7201F06FBDFCF76CBB0DF1700CA5
:10F4F000F9F7D2FE30B9219F97F84740201C18BF7A
:10F50000012001E04FF00100219981F84700FCF74C
:10F5100059BB9DF874600DF1700CF9F7BDFE014602
:10F5200030464FF00102FBF769FB8DF86B000028B5
:10F530003CF448AB43F25803C2F20003187201F0E6
:10F5400042BD0DF1700CF9F7A7FE01468DF86A0077
:10F550009DF87400FBF710FB8DF86B0000283CF45D
:10F5600031AB43F25805C2F20005287201F02BBD01
:10F570001D9A1C924FF001038DF86A301E462198A7
:10F5800090F847100B420AD090F846109DF8700092
:10F5900019403246FBF732FB8DF86B0068B99DF8D5
:10F5A0006A304FEA43058DF86A501C9A02F1010255
:10F5B0001C9215F0FE03E2D10AE09DF86A60012E6C
:10F5C00006D143F25801C2F20001087201F0FBBCFF
:10F5D0004FF000078DF86B700DF1700CF9F75CFEC1
:10F5E0000DF1700CF9F758FEFCF7ECBA9DF87400B9
:10F5F0004FF001010A46FBF701FB8DF86B00002874
:10F600003CF4E0AA43F25805C2F20005287201F06A
:10F61000DABC9DF874004FF000014FF00102FBF7D7
:10F62000EDFA8DF86B0000283CF4CCAA43F25802A6
:10F63000C2F20002107201F0C6BC0DF1700CF9F7B5
:10F640002BFE219C94F84730184384F84700FCF7C0
:10F65000B9BA1D980DF1A80C4CF8380DFAF7CAFA92
:10F6600000287CF4AFAA43F2B810C2F20000099E51
:10F67000066001F02BBC10A8FAF74EF9014640B124
:10F680009DF84070022F04D0C2484FF00D0208F0E0
:10F690008BFF0DF1700C9DF84000F9F7E5FDFCF7CC
:10F6A00091BAFAF783FEFCF78DBA0DF1700CF9F7F9
:10F6B000F3FDFCF787BA1D9DFA2D08D943F25803D4
:10F6C000C2F200034FF012021A7201F07CBC0DF17D
:10F6D000700CF9F7E1FD43F29001C2F200014855C8
:10F6E000FCF770BA0DF1700CF9F7D6FD43F29004F7
:10F6F000C2F2000484F8FB00FCF764BA0DF1700C50
:10F70000219890F84700F9F7AFFDFCF75BBA1D9E12
:10F71000FA2E08D943F25805C2F200054FF0120143
:10F72000297201F050BC0DF1700C43F29007C2F247
:10F730000007B85DF9F798FDFCF744BA0DF1700CBD
:10F7400043F29003C2F2000393F8FB00F9F78CFD3B
:10F75000FCF738BA1D9EF62E08D943F25800C2F2C3
:10F7600000004FF01205057201F02DBC219A906C3B
:10F77000F9F7CAFB43F29004C2F20004A051FCF76F
:10F7800021BA43F22401C2F200010B7813F0280FD2
:10F7900006D01D9EB6F5005F34BF0026012604E0AA
:10F7A0001D9EFA2E94BF0026012646B143F2580052
:10F7B000C2F200004FF01305057201F004BC0DF118
:10F7C000700C40F6E877C2F200071D9AB85CF9F7B2
:10F7D0004BFDFCF7F7B90DF1700CF9F785FD40F61C
:10F7E000E874C2F200041E99665C1D9B1E420DF176
:10F7F000700C0CBF0020FF20F9F736FDFCF7E2B9D2
:10F8000043F22402C2F20002107810F0280F08D050
:10F810001D9D05F10105B5F5005F34BF00250125EB
:10F8200006E01D9D05F10105FA2D94BF0025012577
:10F8300045B143F25800C2F200004FF013010172CB
:10F8400001F0C1BB1D9E40F6E871C2F20001885D67
:10F850008B195A7842EA00251C95002D3CF4B2A978
:10F86000FEF75EBB43F22403C2F200031A7812F0E3
:10F87000280F06D01D9DB5F5005F34BF002501257A
:10F8800004E01D9DFA2D94BF0025012545B143F2EA
:10F890005803C2F200034FF013021A7201F093BB37
:10F8A00040F6E876C2F200061D98315C002956D178
:10F8B000FCF788B943F22405C2F200052E7816F051
:10F8C000280F06D01D98B0F5005F34BF002001203E
:10F8D00004E01D98FA2894BF0020012040B143F2B3
:10F8E0005805C2F200054FF013062E7201F06BBBF3
:10F8F00040F6E871C2F200011D9BCA5C7AB3FCF7C6
:10F9000061B90DF1700CF9F7C7FC1C9038BBFCF71E
:10F9100059B90DF1700CF9F7E7FC40F6E870C2F246
:10F9200000001E99425C1D9B1A4218D0FCF74AB990
:10F930000DF1700CF9F7D8FC40F6E875C2F200053D
:10F940001E9EA85D1D99084209D1FCF73BB90DF137
:10F95000700CF9F7A1FC1C9000287CF433A9219EBF
:10F96000336A43B943F25800C2F200004FF0030279
:10F97000027201F028BB03F1FF34346203F101038A
:10F9800056F8237043F2B815C2F200052F60FCF759
:10F9900019B900BFEE0F00203C7844F020023A7005
:10F9A000FCF7DEB9219F97F847304FEAD31545EAB7
:10F9B000430687F84760FCF705B9219890F847405F
:10F9C0004FEA540141EAC41280F84720FCF7FAB824
:10F9D000FAF774F8FCF7F6B842F6E877C2F20007D7
:10F9E000FB784FF0010505FA03F53E7926EA050696
:10F9F0003E71FCF7E7B843F25800C2F200004FF046
:10FA00000101017201F0DFBA42F6E874C2F20004AB
:10FA1000E27842B942F6E875C2F200054FF00606F8
:10FA2000EE70FCF7CFB802F1FF3742F6E873C2F28E
:10FA30000003DF70FCF7C6B842F6E870C2F20000BF
:10FA4000017801F1FF34E7B207700279FF2A0BD188
:10FA5000632F7CF6B7A842F6E876C2F200064FF0B4
:10FA600063003070FCF7AEB8172F7CF6ABA842F6F7
:10FA7000E873C2F200034FF017051D70FCF7A2B83F
:10FA800042F6E871C2F200014C7804F1FF37FBB294
:10FA90004B700A79FF2A0BD1002B7CF493A842F615
:10FAA000E870C2F200004FF00C014170FCF78AB818
:10FAB0003B2B7CF687A842F6E875C2F200054FF0B2
:10FAC0003B066E70FCF77EB843F25803C2F20003A7
:10FAD0004FF001021A7201F076BA43F25805C2F2F1
:10FAE00000054FF001062E7201F06DBA43F2580086
:10FAF000C2F200004FF00101017201F064BA43F25A
:10FB00005803C2F200034FF001021A7201F05BBA0F
:10FB100042F6E874C2F20004E778052F08D942F6ED
:10FB2000E876C2F200064FF00000F070FCF74AB829
:10FB300007F1010742F6E875C2F20005EF70FCF725
:10FB400041B842F6E871C2F200010B7803F10103FB
:10FB5000DCB20C700A79FF2A0BD1632C7CF632A838
:10FB600042F6E876C2F200064FF000003070FCF773
:10FB700029B8172C7CF626A842F6E877C2F20007CF
:10FB80004FF000053D70FCF71DB842F6E871C2F277
:10FB900000014B7803F10103DCB24C700A79FF2AB3
:10FBA0000BD10C2C7CF60EA842F6E876C2F20006C9
:10FBB0004FF001007070FCF705B83B2C7CF602A8F2
:10FBC00042F6E877C2F200074FF000057D70FBF7C0
:10FBD000F9BF43F25801C2F200014FF001030B726A
:10FBE00001F0F1B942F6E874C2F20004E2784FF095
:10FBF000010707FA02F7257987EA05062671FBF760
:10FC0000E1BF0DF1700CF9F747FB42F6E871C2F263
:10FC100000010871FBF7D6BF0DF1700CF9F73CFB42
:10FC2000062842F6E873C2F2000392BFD8700020A3
:10FC3000D870FBF7C7BF0DF1700CF9F72DFB42F63A
:10FC4000E874C2F200042070FBF7BCBF0DF1700C29
:10FC5000F9F722FB42F6E872C2F200025070FBF79D
:10FC6000B1BF0DF1700CF9F717FB42F6E877C2F25D
:10FC70000007B870FBF7A6BF0DF1700C42F6E875EF
:10FC8000C2F200052879F9F7EFFAFBF79BBF0DF1F7
:10FC9000700C42F6E876C2F20006F078F9F7E4FA62
:10FCA000FBF790BF0DF1700C42F6E871C2F2000153
:10FCB0000878F9F7D9FAFBF785BF0DF1700C42F619
:10FCC000E873C2F200035878F9F7CEFAFBF77ABF6F
:10FCD0000DF1700C42F6E870C2F200008078F9F77E
:10FCE000C3FAFBF76FBF43F25805C2F200054FF0AD
:10FCF00001022A7201F067B91D9E0F2E08D943F246
:10FD00005806C2F200064FF02701317201F05BB9CC
:10FD1000CC4C04EB860742F6E871C2F2000114F8FD
:10FD200026300B70787848704FF000058D70CD70DC
:10FD3000BA780A71FBF746BF43F25803C2F20003D8
:10FD40004FF00100187201F03EB942F6E874C2F2B9
:10FD50000004E7784FF0010505FA07F5227945EA36
:10FD600002062671FBF72EBF43F25801C2F20001D2
:10FD70004FF001030B7201F026B943F25800C2F2B2
:10FD800000004FF00105057201F01DB94FF00004AD
:10FD9000139412941194199442F6E877C2F2000772
:10FDA0003A7802F1640216927E7806F1FF311591DD
:10FDB000BB78149311A808F01DFA179818B100F138
:10FDC000FF34E5B201E04FF0060542F6E877C2F2F3
:10FDD0000007FD70FBF7F6BE1D9A0F2A08D943F203
:10FDE0005806C2F200064FF02702327201F0EBB85B
:10FDF000944E06EB820142F6E873C2F200031878D3
:10FE000006F822005D784D701C798C70FBF7DABE25
:10FE100043F25801C2F200014FF001030B7201F0EE
:10FE2000D2B80DF1700C219F97F85000F9F71CFA29
:10FE3000FBF7C8BE43F22400C2F20000057815F0BB
:10FE4000010F08D143F25800C2F200004FF0300514
:10FE5000057201F0B8B843F29016C2F2000632689B
:10FE600042B943F25801C2F200014FF031030B7264
:10FE700001F0A9B843F22401C2F200010B7803F0AB
:10FE8000FE0040F004050D7043F23006C2F2000699
:10FE90004FF00002326001F002B843F22406C2F2D1
:10FEA0000006327812F0010F08D143F25806C2F270
:10FEB00000064FF03002327201F085B843F2901123
:10FEC000C2F200010B6843B943F25800C2F20000CD
:10FED0004FF03405057201F076B843F22400C2F207
:10FEE0000000057805F0FE0646F00202027043F2BB
:10FEF0003001C2F200014FF000030B6000F0CFBFF1
:10FF0000219C94F846700DF1700CF9F7C5F9219910
:10FF10003B1A91F8500000F001055E1B1C9681F819
:10FF20004760FF2E94BF0026012681F85060FBF742
:10FF300049BE43F22402C2F20002117811F0280FE8
:10FF400006D01D9BB3F5005F34BF0023012304E0FE
:10FF50001D9BFA2B94BF0023012343B143F25805A4
:10FF6000C2F200054FF013062E7201F02CB840F6D5
:10FF7000E874C2F200041E9F1D982754FBF722BEAE
:10FF80004FF000021C921AE04FF001011C9116E0A4
:10FF90004FF002031C9312E04FF003041C940EE098
:10FFA0004FF004071C970AE04FF005001C9006E094
:10FFB0004FF006051C9502E04FF007061C961D99B0
:10FFC0001B911C98F9F78EFDFBF7FCBD0DF1700C31
:10FFD000F9F78AF91E9B40F6E872C2F20002D45C7F
:10FFE0001D992143D154FBF7EDBD1D98F92808D97F
:10FFF00043F25806C2F200064FF01203337200F0CB
:020000040805ED
:10000000E2BF43F29007C2F200071E9D3D54FBF78A
:10001000D9BD43F29002C2F200021D9C82F8FB405F
:10002000FBF7D0BD43F2A421C2F20001086858B921
:1000300043F25800C2F200004FF00105057200F0D3
:10004000C2BF00BF443A001045681D981E994FF08A
:1000500001020DF16A03A8478DF86B009DF86A60F4
:10006000D6F1010238BF0022219B83F850200028DE
:100070003BF4A8AD43F25801C2F20001087200F04F
:10008000A2BF43F2A426C2F20006326842B943F28C
:100090005800C2F200004FF00105057200F093BF56
:1000A00013681D981E9998478DF86B0000283BF443
:1000B00089AD43F25801C2F20001087200F083BF1B
:1000C00043F2A426C2F20006326842B943F2580055
:1000D000C2F200004FF00105057200F074BF5568D0
:1000E0001D981E994FF000020DF16A03A8478DF884
:1000F0006B009DF86A30D3F1010138BF0021219EC9
:1001000086F8501000283BF45DAD43F25802C2F26D
:100110000002107200F057BF0A981E99F9F7DCFA36
:100120000A9040B943F25801C2F200014FF017069D
:100130000E7200F048BF0A9B19688E6A46B943F2F6
:100140005800C2F200004FF01503037200F03BBFED
:100150000A9A90689DF8741043F29002C2F200026D
:10016000B0478DF86B0000283BF42CAD43F25805E6
:10017000C2F20005287200F026BF0A981E99F9F70E
:10018000ABFA0A9040B943F25805C2F200054FF0AD
:1001900017032B7200F017BF0A9A15686B6943B9F1
:1001A00043F25806C2F200064FF01502327200F018
:1001B0000ABF0A9880689DF8741043F29002C2F258
:1001C000000298478DF86B0000283BF4FBAC43F22B
:1001D0005801C2F20001087200F0F5BE0A981E999B
:1001E000F9F77AFA0A9040B943F25805C2F20005CD
:1001F0004FF017022A7200F0E6BE0A9801688E6975
:1002000046B943F25800C2F200004FF015060672DC
:1002100000F0D9BE43F29005C2F200050A9A906838
:100220009DF874102A460DF16A03B0478DF86B00F3
:100230009DF86A302B7000283BF4C4AC43F258019F
:10024000C2F20001087200F0BEBE0A981E99F9F7CA
:1002500043FA0A901D997F2909D1071C18BF01276D
:1002600043F29004C2F200042770FBF7ABBC0A9B78
:1002700043B943F25806C2F200064FF01705357233
:1002800000F0A1BE0A980668756845B943F25803A4
:10029000C2F200034FF01500187200F094BE0A9AE3
:1002A0009068C9B243F29002C2F20002A8478DF8EA
:1002B0006B0000283BF486AC43F25801C2F2000107
:1002C000087200F080BE0A981E99F9F705FA0A90A4
:1002D00040B943F25805C2F200054FF017032B72E4
:1002E00000F071BE0A9A11688E6846B943F2580050
:1002F000C2F200004FF01506067200F064BE43F231
:100300009005C2F200050A9B98689DF874102A783F
:100310000DF16A03B0478DF86B009DF86A202A70D2
:1003200000283BF44FAC43F25801C2F200010872BE
:1003300000F049BE0A981E99F9F7CEF90A9040B923
:1003400043F25805C2F200054FF01700287200F082
:100350003ABE0A9A1168CE6846B943F25801C2F211
:1003600000014FF015060E7200F02DBE43F290050D
:10037000C2F200050A9880689DF874102A460DF1B3
:100380006A03B0478DF86B009DF86A302B70002827
:100390003BF418AC43F25802C2F20002107200F0B3
:1003A00012BE0A981E99F9F797F90A9040B943F2DC
:1003B0005806C2F200064FF01705357200F003BE72
:1003C0000A9B1A68166946B943F25800C2F2000047
:1003D0004FF01502027200F0F6BD0A9FD7F80880B0
:1003E0009DF8747043F29005C2F200052868F8F792
:1003F000B5FD0246404639460DF16A03B0478DF817
:100400006B009DF86A10297000283BF4DBAB43F2C7
:100410005803C2F20003187200F0D5BD0A984FF0DD
:100420000001F9F759F90A9040B943F25803C2F2B2
:1004300000034FF017061E7200F0C5BD0A990B6845
:10044000DE6A46B943F25805C2F200054FF01501C5
:10045000297200F0B8BD0A9880689DF87410B04702
:100460008DF86B0000283BF4ADAB43F25802C2F2AA
:100470000002107200F0A7BD0A981E99F9F72CF936
:100480000A9040B943F25805C2F200054FF0170236
:100490002A7200F098BD0A980268D56945B943F2FE
:1004A0005806C2F200064FF01500307200F08BBD06
:1004B0000A9988689DF8741043F29002C2F2000213
:1004C000A8478DF86B0000283BF47CAB43F258033F
:1004D000C2F20003187200F076BD0A981E99F9F76F
:1004E000FBF80A9040B943F25803C2F200034FF000
:1004F00017061E7200F067BD0A990B681E6A46B99E
:1005000043F25801C2F200014FF015020A7200F0E6
:100510005ABD0A9880689DF8741043F29002C2F2A6
:100520000002B0478DF86B0000283BF44BAB43F260
:100530005805C2F20005287200F045BD0A981E99C0
:10054000F9F7CAF80A9040B943F25801C2F2000123
:100550004FF017020A7200F036BD0A9805686B6A00
:1005600043B943F25805C2F200054FF015032B7250
:1005700000F029BD0A9988689DF8741010AA984760
:100580008DF86B001098F8F7BFFC43F29002C2F2AE
:10059000000210609DF86B60002E3BF413AB43F239
:1005A0005800C2F20000067200F00DBD0A984FF02C
:1005B0000001F9F791F80A9040B943F25800C2F2ED
:1005C00000004FF01705057200F0FDBC0A9E306870
:1005D000056B45B943F25806C2F200064FF015020A
:1005E000327200F0F0BC0A9B98689DF8741043F2D8
:1005F0009002C2F20002A8478DF86B0000283BF47D
:10060000E1AA43F25801C2F20001087200F0DBBC1B
:100610001D9B072B08D943F25800C2F200004FF08F
:100620000803037200F0CFBC40F2A064C1F20004E2
:1006300004EBC307D7F8101900297BF4C3AAF7F716
:100640001FF9002808BF012040F2A066C1F2000691
:100650001D9A06EBC205C5F81009FBF7B3BA1D9940
:10066000072908D943F25803C2F200034FF00801EA
:10067000197200F0A8BC40F2A064C1F2000404EBBF
:10068000C107D7F81069002E3BF49CAAF7F7F8F8D9
:100690001D9D40F2A062C1F2000202EBC503D3F837
:1006A0001019401A1C90D3F81449A0428CBF0024A2
:1006B000C0EB04041B9440F2A067C1F2000707EBF3
:1006C000C5061B9DC6F814594FF00002C6F8102944
:1006D000FBF778BA43F22400C2F20000067816F065
:1006E000280F06D01D9DB5F5005F34BF00250125FC
:1006F00004E01D9DFA2D94BF0025012545B143F26C
:100700005803C2F200034FF013021A7200F05BBCF0
:100710001D9C0DF1700CF8F7BFFD40F6E877C2F2B2
:1007200000073855FBF74EBA0DF1700CF8F7DCFDF9
:100730000DF1700CF8F7B0FD1C9050B11E9F40F603
:10074000E873C2F20003DA5D1D9E1643DE55FBF727
:1007500039BA1E9E40F6E875C2F20005A85D1D99E3
:1007600020EA0104AC55FBF72DBA1D9D1E9A5019C5
:10077000C1B243F29003C2F2000383F8FB10FA29DE
:1007800008D943F25803C2F200034FF012061E725A
:1007900000F019BC43F2B814C2F20004276843F217
:1007A0009006C2F20006701940F20005C0F602057C
:1007B000791907F0F9FE22681E9811182160FBF7DD
:1007C00001BA43F22405C2F200052A7812F0280F7C
:1007D00008D01D9800F10200B0F5005F34BF002082
:1007E000012006E01D9800F10200FA2894BF0020C5
:1007F000012038B143F25803C2F200034FF0130650
:100800001E72E0E3F7F73CF800F104004CF6CD442B
:10081000CCF6CC44A4FB00174FEA9701219B5E6AFB
:10082000B1FBF6F51C951D9A40F6E874C2F200047F
:100830004FEA1540A054A7184FEA15217970BD70F2
:10084000FBF7C0B943F22405C2F200052A7812F082
:10085000280F08D01D9800F10200B0F5005F34BFEA
:100860000020012006E01D9800F10200FA2894BF44
:100870000020012038B143F25801C2F200014FF0CC
:1008800013030B729FE3F6F7FBFF00F104004CF635
:10089000CD44CCF6CC44A4FB00274FEA9701219B22
:1008A0005E6AB1FBF6F51D9840F6E877C2F20007E4
:1008B0003A185478395C4FEA014343EA04269078A9
:1008C00046EA00071B97ED1B25F07F421C920DF1B5
:1008D000700C1E9882422CBF00200120F8F7C4FC47
:1008E000FBF770B9219C94F846600DF1700CF8F795
:1008F000D3FC301A1C90219F87F84700FF2894BF33
:100900000020012087F85000FBF75CB943F2240572
:10091000C2F200052A7812F0280F08D01D9901F1C3
:100920000101B1F5005F34BF0021012106E01D99EE
:1009300001F10101FA2994BF0021012139B143F2EB
:100940005801C2F200014FF013060E723BE31D9EE8
:1009500043F2B813C2F200031D6840F6E872C2F217
:1009600000024FEA1520905591194D70FEF7F7BF20
:10097000219B93F847401C9493F8467083F8477086
:1009800083F84640FBF71EB91D98072807D943F2A4
:100990005805C2F200054FF00800287213E3F9F77A
:1009A000CFF80DF1A80C4CF8380D003018BF01201D
:1009B000F8F75AFCFBF706B9219A92F8470092F82B
:1009C00046100DF1700C884214BF00200120F8F78A
:1009D0004BFCFBF7F7B8219E96F8474096F8463057
:1009E0000DF1700CE01A18BF0120F8F73DFCFBF781
:1009F000E9B8219F97F8470097F846500DF1700C21
:100A0000A8422CBF00200120F8F72EFCFBF7DAB833
:100A1000219A92F8470092F846100DF1700C884226
:100A200094BF00200120F8F71FFCFBF7CBB8219EF4
:100A300096F8470096F846400DF1700CA0428CBF26
:100A400000200120F8F710FCFBF7BCB8219B93F8BD
:100A5000470093F846700DF1700CB84234BF002087
:100A60000120F8F701FCFBF7ADB81D98F62807D96F
:100A700043F25801C2F200014FF012060E72A2E2D8
:100A800043F29005C2F200052858F8F767FA219A58
:100A9000D064FBF797B81D9BF62B07D943F258009B
:100AA000C2F200004FF0120505728CE243F290048E
:100AB000C2F20004E058F8F751FA219FB864FBF73E
:100AC00081B843F29002C2F2000292F8FB201D9E10
:100AD0009119FB2907D943F25803C2F200034FF0E2
:100AE000120018726FE243F22403C2F20003187876
:100AF00010F0280F09D01E98151805F1FF33B3F533
:100B0000005FB4BF0023012307E01E9D511901F1CE
:100B1000FF33FA2BD4BF002301233BB143F2580625
:100B2000C2F200064FF0130232724CE240F6E87453
:100B3000C2F200041E9FE01943F29001C2F20001CC
:100B4000891907F031FDFBF73DB82198456B2968FD
:100B50004D683DB943F25801C2F200014FF01E0248
:100B60000A7230E21E9A43F29006C2F2000696F82C
:100B7000FB309918FB2907D943F25800C2F2000054
:100B80004FF0120505721EE200F134001D9943F288
:100B90009006C2F20006B218A8478DF86B00002834
:100BA0003BF410A843F25803C2F2000318720AE2A1
:100BB00043F25806C2F200064FF00103337202E21C
:100BC0000DF1700CF8F790FB40F6E874C2F20004E7
:100BD0001E9FE05D1D9D28423AF4F4AF43F2B81227
:100BE000C2F200020999116070E10DF1700CF8F782
:100BF0007BFB40F6E876C2F200061E9BF45C1D9F6C
:100C00003C427AF4DFAF43F2B810C2F20000099D13
:100C100005605BE19DF874000DF16B01F9F7DEFEF4
:100C20008DF86A009DF86B1029B143F25803C2F2A7
:100C300000031972C7E100283AF4C4AF43F2B812B6
:100C4000C2F20002099E166040E19DF874000DF1A9
:100C50006B01F9F7C3FED0F1010038BF00208DF819
:100C60006A009DF86B602EB143F25803C2F2000394
:100C70001E72A8E1219CE76A17B98DF86A7002E03C
:100C80009DF86A3063B90DF1700C1E98F8F7B2FF49
:100C900030B943F2B815C2F200050999296015E18F
:100CA0000DF1700C9DF86A00F8F7DEFA4FF00002C3
:100CB0002198C262FAF786BF9DF874000DF16B01AE
:100CC000F9F78CFE8DF86A009DF86B502DB143F258
:100CD0005801C2F200010D7275E100287AF472AF7A
:100CE00043F2B814C2F20004099F2760EEE09DF8B9
:100CF00074000DF16B01F9F7A1FE8DF86A009DF803
:100D00006B602EB143F25800C2F2000006725AE145
:100D100000287AF457AF43F2B813C2F20003099ADD
:100D20001A60D3E09DF874000DF16B01F9F786FEAF
:100D3000051C18BF01258DF86A5092E79DF87400D4
:100D40000DF16B01F9F74AFE011C18BF01218DF866
:100D50006A1086E71D9EF62E07D943F25800C2F2AC
:100D600000004FF0120202722DE1219CE06CF8F7B6
:100D7000CBF843F29007C2F20007B851FAF722BF4E
:100D80000DF1700CF8F788FA219D95F84710D1F114
:100D9000010338BF0023002814BF1E4683F001065C
:100DA00085F84760FAF70EBF0DF1700CF8F774FA8A
:100DB000219C94F84770784084F84700FAF702BF06
:100DC0000DF1700CF8F768FA219A82F85100FAF7E1
:100DD000F9BE06F04BF80DF1A80C4CF8380DFF28C1
:100DE00028BFFF20C0B2F8F73FFAFAF7EBBE06F0D3
:100DF00033F80DF1A80C4CF8380DFF2828BFFF2060
:100E0000C0B2F8F731FAFAF7DDBE06F039F80DF1A5
:100E1000A80C4CF8380DFF2828BFFF20C0B2F8F707
:100E200023FAFAF7CFBE06F00DF80DF1700C00288A
:100E30000CBFFF200020F8F717FAFAF7C3BE43F201
:100E40008C10C2F2000005681D99681805F034FB8B
:100E50008DF86B0000283AF4B5AE43F25803C2F2A5
:100E600000031872AFE01D9805F0E4FAFAF7AABE85
:100E70000DF1700CF8F710FA05F0D6FAFAF7A2BEE9
:100E800043F28C16C2F2000634681D9FE01905F08B
:100E9000EDFAFAF797BE05F0D1FAFAF793BE43F2EE
:100EA0009012C2F20002106880B943F22405C2F227
:100EB0000005297801F00203DEB23EB143F2580387
:100EC000C2F200034FF0350119727CE043F22404B2
:100ED000C2F20004277817F0010F7AF471AE21985E
:100EE00028B143F2B812C2F200021568456043F21D
:100EF0003001C2F200010B687F2B00F2BD8003F1CC
:100F000001031B931C9313B94FF001041B94794EFA
:100F10004FF0540543F22404C2F2000443F2901748
:100F2000C2F200071C9B05FB036021909BB921784E
:100F300001F00402D1B209B93A6842B9217841F00E
:100F400001026FF382022270426842B115E04FF055
:100F500001001C90E6E742687AB9802B02D003F1C9
:100F6000010301E04FF000031C931B988342D9D189
:100F70004FF00000F9F706FAD4E743F23006C2F268
:100F80000006336043F2B815C2F200052A604FF044
:100F90000009CB46FAF716BE219C276A47F00042AB
:100FA0002263FAF70FBE4FF00006219D2E63FAF779
:100FB00009BEFAF707BE0B9C43F25800C2F20000CC
:100FC0004FF00103037243F25806C2F20006099D76
:100FD00035602198036A23B103F1010350F823100F
:100FE000099143F25806C2F20006099A72607472BF
:100FF000F0F75AFCF0F758FC219C256A7DB14FF0C0
:1010000000001C90219B196A49B1F0F74DFC1C9E11
:1010100006F101061C96219A146AB442F5D840F6EE
:10102000E575C2F20005287828B94FF00000F9F7FD
:10103000A9F9FAF7FABCF9F75BF940F6E573C2F2E1
:101040000003197804297AF4F0AC4FF0000640F65A
:10105000E574C2F200043046F9F794F92278042AC4
:10106000F9D0FAF7E2BC4FF0000405F1FF354FF07C
:1010700000005746FDF7AFBB4FF000061C9643E754
:101080004FF002031C931B4ED6F8AC1031B9FDF79C
:10109000FFBD2BB0BDEC048BBDE8F08F03F1010365
:1010A00006F15406FDF7F0BD04F1010306F1540604
:1010B000812B7DF4E9ADFDF745BE002F3DF415AB66
:1010C000C75CCF5403F1010393427DF40EABFDF7EF
:1010D00016BBE118EE1813F801CF02F1FF37604597
:1010E0003DF49AA83A46FDF7A4B807F1FF32FDF7A0
:1010F000A0B800BFF00F00102DE9F04F2DED028BCE
:1011000091B04FF000020592904643F22C07C2F2D4
:10111000000743F21C03C2F20003049343F2280BBE
:10112000C2F2000B40F2A066C1F200069FEDBC8B3C
:1011300039684FF0FF3041B9F0F7B6FB3868002846
:101140000CBFFA204FF0FF30FFE7F5F715FF28B18D
:10115000B8F1320F09D808F1010806E0B8F1330FF1
:101160000CBF4FF034084FF000083C681CBBF0F790
:101170009BFBB8F1320F11D1049B1868F5F7A8FF5B
:101180004FF0000104980160F5F77EF94FF002007E
:10119000F8F7ECFF4FF0020405940CE0B8F1340FBF
:1011A00009D1059D012D06D04FF00100F8F7DEFFB3
:1011B0004FF001020592BBF800504FF4117202FB90
:1011C0000563D3F818120029B2D04FF4117000FB58
:1011D00005F505F5887406EB0409355DE02D40F052
:1011E000A58499F801200E2A00F09584212A40F068
:1011F0009D8400F090BC19F80310501A03F1FF35DC
:1012000019F80520821A05F1FF33002DF3D112F0F1
:10121000FF0F40F07C84335D4FEA5311072900F241
:101220006E84DFE811F008006C046C043500AB003C
:101230006C048F005A01335D09F1010413F01F00A3
:1012400000F0658409F1020904F1020400F1FF32A3
:1012500054FA82F503954FF000054FF0010A15E0AE
:1012600019F8011CE8B221405246F9F7C7FC0028E2
:1012700040F04D8405F101054FEA4404FF2CEFD9FD
:1012800009F101090399894500F041845446E7E7D3
:1012900099F80150386898B1F5F71AFF4FF000003F
:1012A000386040F6E572C2F200021070F5F7ECF813
:1012B000FAF758FA4FF00100F8F758FFF0F7F4FA90
:1012C000049B196869B94CF22860C0F605004FF01C
:1012D00007014AF6A162C0F60402F5F70FFE049C6E
:1012E000206007A84FF00001F9F734FA7DB9F6F74E
:1012F000C7FAC1B201F1FF33DCB2FD2C43F2941006
:10130000C2F2000092BF01700122027009E043F2B4
:101310009410C2F20000027802FB05F505EB1525DA
:10132000057043F29415C2F20005297810AB03F85A
:10133000241D4FF003004FF000014FF01A02F8F7A0
:1013400039FFF5E60DF11B00F8F7E6FA01469DF8C6
:101350001B408DF81C40012C06D828B10DF11D0052
:101360004FF00D0207F020F94FF006004FF000019A
:101370004FF00E0207ABF8F71DFFD9E6BBF80030BF
:101380004FF4117101FB03F499F80100052800F2F4
:10139000A180DFE800F00A2F495B037D40F6E5738A
:1013A000C2F200034FF0010119704FF00100FAF78B
:1013B00063FA4FF0000510AB03F8255D4FF0040011
:1013C00029464FF00102F8F7F5FE4FF0C800F7F795
:1013D0001DFD31599BF800004FF001040094019568
:1013E000D1F80CC04FF416512A464FF00803E047DD
:1013F000204689E34FF0000143F25803C2F2000394
:1014000019724FF0010410AB03F8254D4FF00400A2
:101410002246F8F7CFFE204676E300BFAFF3008008
:101420000000000000E06F40F8F7C0FF10AB4FF085
:10143000020203F8252D4FF004004FF000014FF099
:101440000102F8F7B7FE4FF001005DE310AB4FF07B
:10145000120003F8250D4FF004004FF000014FF08B
:101460000102F8F7A7FE4FF0C800F7F7CFFC355997
:101470009BF800004FF0010400944FF0000201922D
:10148000ED684FF416414FF00803A84720463BE3B0
:1014900010AB4FF0120203F8252D4FF004004FF06F
:1014A00000014FF00102F8F785FE4FF0C800F7F792
:1014B000ADFC35599BF800004FF0010400944FF04B
:1014C00000020192ED684FF4E1314FF00803A847A4
:1014D000204619E34FF0000016E399F802E099F86E
:1014E000035005EB0E201FFA80FC99F80130A3F1A0
:1014F0000203412B00F20683DFE813F042009D0057
